:040000000DEF00F010
:0400080083EF50F042
:0A001800FF0011EECFF1D3EF5FF00F
:10100000000200000100E652E652E652FB0E6F00BD
:101010008FFFE6FF6F008FFFE6FF25EC63F0FE0E0B
:101020006000BFF0E3FFFD0E6000BBF0E3FFFD0ECC
:101030006F008FFFF6FFFE0E6F008FFFF7FF000EB1
:10104000F86E0F0EF76403D00800F55007D06F005C
:10105000DBFFE9FF6F00DFFFEAFFEF50396EFF0EA5
:101060006000E7F0E3FFFB0E6F008FFFE6FF6F000D
:101070008FFFE6FFE5EC63F0FB0E6F008FFFE6FFEE
:101080006F008FFFE6FF87EC62F0F80EE126FF0E9F
:10109000E22230EF0DF0FD0EE350010F386EFE0E30
:1010A0006F008CFF39F0000E39226000E3F0E6FF9C
:1010B0006000E7F0E6FFDBEC54F0FB0E6F008FFF03
:1010C000D9FFFC0E6F008FFFDAFFDF50140AD8A49F
:1010D0006CEF08F06EEF08F087EF08F0FD0E6F0080
:1010E0008FFFF6FFFE0E6F008FFFF7FF000EF86E0A
:1010F0000F0EF76404D0150EF56E0C0008D06F00CB
:10110000DBFFE9FF6F00DFFFEAFF150EEF6EFB0E5E
:101110006F008FFFD9FFFC0E6F008FFFDAFFDF50EB
:10112000150AD8A496EF08F098EF08F06FEF0DF0CD
:10113000FD0E6F008FFFF6FFFE0E6F008FFFF7FFB3
:10114000000EF86E0F0EF76404D0190EF56E0C0049
:1011500008D06F00DBFFE9FF6F00DFFFEAFF190E29
:10116000EF6E000EE66E000EE66E000EE66E000EEE
:10117000E66E000EE66E000EE66E000EE66E000EE7
:10118000E66EF50EE3501E0F386EF60E6F008CFF04
:1011900039F0000E39226000E3F0F6FF6000E7F05E
:1011A000F7FF000EF86E0F0EF76403D00800F5503D
:1011B00007D06F00DBFFE9FF6F00DFFFEAFFEF50B2
:1011C0000A0D6F00CCFF38F06F00D0FF39F06000DF
:1011D000E3F0E6FF6000E7F0E6FFF30E6F008FFF3D
:1011E000E6FF6F008FFFE6FF29EC5FF06FEF0DF079
:1011F000FB0E6F008FFFD9FFFC0E6F008FFFDAFF31
:10120000DF50160AD8A407EF09F009EF09F06FEFD5
:101210000DF0FD0E6F008FFFF6FFFE0E6F008FFFCB
:10122000F7FF000EF86E0F0EF76404D0160EF56E81
:101230000C0008D06F00DBFFE9FF6F00DFFFEAFF63
:10124000160EEF6E6FEF0DF0FB0E6F008FFFD9FFE4
:10125000FC0E6F008FFFDAFFDF50170AD8A433EFC0
:1012600009F035EF09F06FEF0DF0FD0E6F008FFF05
:10127000F6FFFE0E6F008FFFF7FF000EF86E0F0EE9
:10128000F76404D0170EF56E0C0008D06F00DBFF7A
:10129000E9FF6F00DFFFEAFF170EEF6E000EE66E4C
:1012A000000EE66E000EE66E000EE66E000EE66EB6
:1012B000000EE66E000EE66E000EE66EF50EE350D2
:1012C0001E0F386EF60E6F008CFF39F0000E3922BB
:1012D0006000E3F0F6FF6000E7F0F7FF000EF86E45
:1012E0000F0EF76403D00800F55007D06F00DBFF46
:1012F000E9FF6F00DFFFEAFFEF50140D6F00CCFF36
:1013000038F06F00D0FF39F06000E3F0E6FF6000D6
:10131000E7F0E6FFF30E6F008FFFE6FF6F008FFF31
:10132000E6FF29EC5FF06FEF0DF0FB0E6F008FFF13
:10133000D9FFFC0E6F008FFFDAFFDF50180AD8A428
:10134000A4EF09F0A6EF09F06FEF0DF0FD0EE350EA
:101350001E0F386EFE0E6F008CFF39F0000E392222
:101360006000E3F0F6FF6000E7F0F7FF000EF86EB4
:101370000F0EF76403D00800F55007D06F00DBFFB5
:10138000E9FF6F00DFFFEAFFEF500009D8A4CBEFC1
:1013900009F0CDEF09F00FEF0AF0FD0EE3501D0F3D
:1013A000386EFE0E6F008CFF39F0000E392260009F
:1013B000E3F0F6FF6000E7F0F7FF000EF86E0F0EA7
:1013C000F76403D00800F55007D06F00DBFFE9FF9A
:1013D0006F00DFFFEAFFEF500009D8B4F2EF09F029
:1013E000F4EF09F0AFEF0AF0FD0E6F008FFFF6FF8C
:1013F000FE0E6F008FFFF7FF000EF86E0F0EF76402
:1014000004D01A0EF56E0C0008D06F00DBFFE9FF68
:101410006F00DFFFEAFF1A0EEF6EAFEF0AF0FD0E6E
:10142000E3501A0F386EFE0E6F008CFF39F0000E7D
:1014300039226000E3F0F6FF6000E7F0F7FF000EEE
:10144000F86E0F0EF76403D00800F55007D06F0058
:10145000DBFFE9FF6F00DFFFEAFFEF500009D8B4C0
:1014600034EF0AF036EF0AF096EF0AF0FD0E6F0047
:101470008FFFF6FFFE0E6F008FFFF7FF000EF86E76
:101480000F0EF76404D0170EF56E0C0008D06F0035
:10149000DBFFE9FF6F00DFFFEAFF170EEF6E000EC4
:1014A000E66E000EE66E000EE66E000EE66E000EB4
:1014B000E66E000EE66E000EE66E000EE66EF50EAF
:1014C000E3501E0F386EF60E6F008CFF39F0000EE1
:1014D00039226000E3F0F6FF6000E7F0F7FF000E4E
:1014E000F86E0F0EF76403D00800F55007D06F00B8
:1014F000DBFFE9FF6F00DFFFEAFFEF50140D6F0025
:10150000CCFF38F06F00D0FF39F06000E3F0E6FF69
:101510006000E7F0E6FFF30E6F008FFFE6FF6F005D
:101520008FFFE6FF29EC5FF0AFEF0AF0FD0E6F00D2
:101530008FFFF6FFFE0E6F008FFFF7FF000EF86EB5
:101540000F0EF76404D0180EF56E0C0008D06F0073
:10155000DBFFE9FF6F00DFFFEAFF180EEF6EFD0E05
:10156000E3501A0F386EFE0E6F008CFF39F0000E3C
:1015700039226000E3F0F6FF6000E7F0F7FF000EAD
:10158000F86E0F0EF76404D0000EF56E0C0008D054
:101590006F00DBFFE9FF6F00DFFFEAFF000EEF6E79
:1015A0006FEF0DF0FB0E6F008FFFD9FFFC0E6F0089
:1015B0008FFFDAFFDF501A0AD8A4E1EF0AF0E3EF59
:1015C0000AF06FEF0DF0FD0E6F008FFFF6FFFE0EBD
:1015D0006F008FFFF7FF000EF86E0F0EF76404D058
:1015E000150EF56E0C0008D06F00DBFFE9FF6F00F1
:1015F000DFFFEAFF150EEF6E6FEF0DF0FB0E6F00D1
:101600008FFFD9FFFC0E6F008FFFDAFFDF50180A43
:10161000D8A40DEF0BF00FEF0BF06FEF0DF0FD0EF8
:10162000E3502F0F386EFE0E6F008CFF39F0000E66
:1016300039226000E3F0F6FF6000E7F0F7FF000EEC
:10164000F86E0F0EF76409D009006F00D4FF38F070
:1016500009006F00D4FF39F00CD06F00DBFFE9FF09
:101660006F00DFFFEAFF6F00B8FF38F06F00B8FFD0
:1016700039F038503910D8B440EF0BF042EF0BF08E
:10168000A8EF0BF0FD0EE350310F386EFE0E6F0029
:101690008CFF39F0000E39226000E3F0F6FF6000A5
:1016A000E7F0F7FF000EF86E0F0EF76409D009009F
:1016B0006F00D4FF38F009006F00D4FF39F00CD070
:1016C0006F00DBFFE9FF6F00DFFFEAFF6F00B8FF8D
:1016D00038F06F00B8FF39F06000E3F0E6FF60001B
:1016E000E7F0E6FFFB0EE3502F0F386EFC0E6F00A5
:1016F0008CFF39F0000E39226000E3F0F6FF600045
:10170000E7F0F7FF000EF86E0F0EF76409D009003E
:101710006F00D4FF38F009006F00D4FF39F00CD00F
:101720006F00DBFFE9FF6F00DFFFEAFF6F00B8FF2C
:1017300038F06F00B8FF39F002D8A8EF0BF00500C1
:10174000FA6E3850FD6E3950FE6EFF6AFA50120084
:10175000FD0EE3501E0F386EFE0E6F008CFF39F049
:10176000000E39226000E3F0F6FF6000E7F0F7FFBB
:10177000000EF86E0F0EF76403D00800F55007D086
:101780006F00DBFFE9FF6F00DFFFEAFFEF500009AA
:10179000D8A4CDEF0BF0CFEF0BF011EF0CF0FD0E56
:1017A000E3501D0F386EFE0E6F008CFF39F0000EF7
:1017B00039226000E3F0F6FF6000E7F0F7FF000E6B
:1017C000F86E0F0EF76403D00800F55007D06F00D5
:1017D000DBFFE9FF6F00DFFFEAFFEF500009D8B43D
:1017E000F4EF0BF0F6EF0BF06FEF0DF0FD0E6F0066
:1017F0008FFFF6FFFE0E6F008FFFF7FF000EF86EF3
:101800000F0EF76404D01A0EF56E0C0008D06F00AE
:10181000DBFFE9FF6F00DFFFEAFF1A0EEF6E6FEFED
:101820000DF0000EE66E000EE66E000EE66E000E87
:10183000E66E000EE66E000EE66E000EE66E000E20
:10184000E66EF50EE3501E0F386EF60E6F008CFF3D
:1018500039F0000E39226000E3F0F6FF6000E7F097
:10186000F7FF000EF86E0F0EF76403D00800F55076
:1018700007D06F00DBFFE9FF6F00DFFFEAFFEF50EB
:10188000140D6F00CCFF38F06F00D0FF39F060000E
:10189000E3F0E6FF6000E7F0E6FFF30E6F008FFF76
:1018A000E6FF6F008FFFE6FF29EC5FF06FEF0DF0B2
:1018B000FB0E6F008FFFD9FFFC0E6F008FFFDAFF6A
:1018C000DF50190AD8A467EF0CF069EF0CF06FEF46
:1018D0000DF0000EE66E000EE66E000EE66E000ED7
:1018E000E66E000EE66E000EE66E000EE66E000E70
:1018F000E66EF50EE3501E0F386EF60E6F008CFF8D
:1019000039F0000E39226000E3F0F6FF6000E7F0E6
:10191000F7FF000EF86E0F0EF76403D00800F550C5
:1019200007D06F00DBFFE9FF6F00DFFFEAFFEF503A
:101930000A0D6F00CCFF38F06F00D0FF39F0600067
:10194000E3F0E6FF6000E7F0E6FFF30E6F008FFFC5
:10195000E6FF6F008FFFE6FF29EC5FF0FD0EE3501E
:101960001B0F386EFE0E6F008CFF39F0000E39220F
:101970006000E3F0F6FF6000E7F0F7FF000EF86E9E
:101980000F0EF76403D00800F55007D06F00DBFF9F
:10199000E9FF6F00DFFFEAFFEF500009D8B4D3EF93
:1019A0000CF0D5EF0CF0EEEF0CF0FD0E6F008FFF9A
:1019B000F6FFFE0E6F008FFFF7FF000EF86E0F0EA2
:1019C000F76404D0170EF56E0C0008D06F00DBFF33
:1019D000E9FF6F00DFFFEAFF170EEF6EFD0EE35029
:1019E0001C0F386EFE0E6F008CFF39F0000E39228E
:1019F0006000E3F0F6FF6000E7F0F7FF000EF86E1E
:101A00000F0EF76403D00800F55007D06F00DBFF1E
:101A1000E9FF6F00DFFFEAFFEF500009D8B413EFD2
:101A20000DF015EF0DF06FEF0DF0FD0E6F008FFF55
:101A3000F6FFFE0E6F008FFFF7FF000EF86E0F0E21
:101A4000F76404D0190EF56E0C0008D06F00DBFFB0
:101A5000E9FF6F00DFFFEAFF190EEF6E6FEF0DF089
:101A6000FD0E6F008FFFF6FFFE0E6F008FFFF7FF7A
:101A7000000EF86E0F0EF76403D00800F55007D083
:101A80006F00DBFFE9FF6F00DFFFEAFFEF50386E0A
:101A9000396A3950000AD8B450EF0DF06FEF0DF0ED
:101AA0003850140AD8B44BEF08F0010AD8B4F8EF54
:101AB00008F0030AD8B424EF09F0010AD8B495EF6E
:101AC00009F00F0AD8B4D2EF0AF0010AD8B4FEEF39
:101AD0000AF0030AD8B458EF0CF06FEF0DF0FF0EC8
:101AE0006F008CFF39F0FD0E6F008FFFF6FFFE0ECA
:101AF0006F008FFFF7FF000EF86E0F0EF76403D034
:101B00000800F55007D06F00DBFFE9FF6F00DFFF33
:101B1000EAFFEF503918D8B490EF0DF092EF0DF0C6
:101B2000C0EF11F0BCEF0DF0FD0EE350020F386E68
:101B3000FE0E6F008CFF39F0000E39226000E3F0DA
:101B4000E6FF6000E7F0E6FF40EC61F081EF11F0A6
:101B5000FD0EE350020F386EFE0E6F008CFF39F061
:101B6000000E39226000E3F0E6FF6000E7F0E6FFD8
:101B700040EC61F081EF11F0FF0EE350386E396AEE
:101B80003950000AD8B4C7EF0DF081EF11F038508A
:101B9000140AD8B481EF11F0010AD8B481EF11F022
:101BA000030AD8B481EF11F0010AD8B494EF0DF014
:101BB0000F0AD8B481EF11F0010AD8B4A8EF0DF0E4
:101BC000030AD8B481EF11F081EF11F0FD0EE3505C
:101BD0001B0F386EFE0E6F008CFF39F0000E39229D
:101BE0006000E3F0F6FF6000E7F0F7FF000EF86E2C
:101BF0000F0EF76404D0010EF56E0C0008D06F00D4
:101C0000DBFFE9FF6F00DFFFEAFF010EEF6EFD0E65
:101C1000E3501F0F386EFE0E6F008CFF39F0000E80
:101C200039226000E3F0F6FF6000E7F0F7FF000EF6
:101C3000F86E0F0EF76409D009006F00D4FF38F07A
:101C400009006F00D4FF39F00CD06F00DBFFE9FF13
:101C50006F00DFFFEAFF6F00B8FF38F06F00B8FFDA
:101C600039F038503910D8B438EF0EF03AEF0EF0A2
:101C7000C0EF11F0FD0EE350210F386EFE0E6F0025
:101C80008CFF39F0000E39226000E3F0F6FF6000AF
:101C9000E7F0F7FF000EF86E0F0EF76409D00900A9
:101CA0006F00D4FF38F009006F00D4FF39F00CD07A
:101CB0006F00DBFFE9FF6F00DFFFEAFF6F00B8FF97
:101CC00038F06F00B8FF39F06000E3F0E6FF600025
:101CD000E7F0E6FFFB0EE3501F0F386EFC0E6F00BF
:101CE0008CFF39F0000E39226000E3F0F6FF60004F
:101CF000E7F0F7FF000EF86E0F0EF76409D0090049
:101D00006F00D4FF38F009006F00D4FF39F00CD019
:101D10006F00DBFFE9FF6F00DFFFEAFF6F00B8FF36
:101D200038F06F00B8FF39F002D8A0EF0EF00500D0
:101D3000FA6E3850FD6E3950FE6EFF6AFA5012008E
:101D4000C0EF11F0FD0EE350230F386EFE0E6F0052
:101D50008CFF39F0000E39226000E3F0F6FF6000DE
:101D6000E7F0F7FF000EF86E0F0EF76409D00900D8
:101D70006F00D4FF38F009006F00D4FF39F00CD0A9
:101D80006F00DBFFE9FF6F00DFFFEAFF6F00B8FFC6
:101D900038F06F00B8FF39F038503910D8B4D3EFAD
:101DA0000EF0D5EF0EF0C0EF11F0FD0EE350250F51
:101DB000386EFE0E6F008CFF39F0000E3922600085
:101DC000E3F0F6FF6000E7F0F7FF000EF86E0F0E8D
:101DD000F76409D009006F00D4FF38F009006F00E4
:101DE000D4FF39F00CD06F00DBFFE9FF6F00DFFF9D
:101DF000EAFF6F00B8FF38F06F00B8FF39F06000FD
:101E0000E3F0E6FF6000E7F0E6FFFB0EE350230F90
:101E1000386EFC0E6F008CFF39F0000E3922600026
:101E2000E3F0F6FF6000E7F0F7FF000EF86E0F0E2C
:101E3000F76409D009006F00D4FF38F009006F0083
:101E4000D4FF39F00CD06F00DBFFE9FF6F00DFFF3C
:101E5000EAFF6F00B8FF38F06F00B8FF39F002D822
:101E60003BEF0FF00500FA6E3850FD6E3950FE6EF4
:101E7000FF6AFA501200C0EF11F0FD0EE350010F9F
:101E8000386EFE0E6F008CFF39F0000E39226000B4
:101E9000E3F0E6FF6000E7F0E6FF4FEC55F0000EE0
:101EA000E66E000EE66EFB0EE350020F386EFC0E7F
:101EB0006F008CFF39F0000E39226000E3F0E6FF7E
:101EC0006000E7F0E6FF29EC60F0FD0EE350270F1D
:101ED000386EFE0E6F008CFF39F0000E3922600064
:101EE000E3F0F6FF6000E7F0F7FF000EF86E0F0E6C
:101EF000F76409D009006F00D4FF38F009006F00C3
:101F0000D4FF39F00CD06F00DBFFE9FF6F00DFFF7B
:101F1000EAFF6F00B8FF38F06F00B8FF39F03850B3
:101F20003910D8B496EF0FF098EF0FF0C0EF11F022
:101F3000FD0EE350290F386EFE0E6F008CFF39F056
:101F4000000E39226000E3F0F6FF6000E7F0F7FFD3
:101F5000000EF86E0F0EF76409D009006F00D4FF71
:101F600038F009006F00D4FF39F00CD06F00DBFFB0
:101F7000E9FF6F00DFFFEAFF6F00B8FF38F06F0086
:101F8000B8FF39F06000E3F0E6FF6000E7F0E6FF3D
:101F9000FB0EE350270F386EFC0E6F008CFF39F0FC
:101FA000000E39226000E3F0F6FF6000E7F0F7FF73
:101FB000000EF86E0F0EF76409D009006F00D4FF11
:101FC00038F009006F00D4FF39F00CD06F00DBFF50
:101FD000E9FF6F00DFFFEAFF6F00B8FF38F06F0026
:101FE000B8FF39F002D8FEEF0FF00500FA6E385056
:101FF000FD6E3950FE6EFF6AFA501200C0EF11F00C
:10200000FD0EE3502B0F386EFE0E6F008CFF39F083
:10201000000E39226000E3F0F6FF6000E7F0F7FF02
:10202000000EF86E0F0EF76409D009006F00D4FFA0
:1020300038F009006F00D4FF39F00CD06F00DBFFDF
:10204000E9FF6F00DFFFEAFF6F00B8FF38F06F00B5
:10205000B8FF39F038503910D8B431EF10F033EF01
:1020600010F0C0EF11F0FD0EE3502D0F386EFE0E94
:102070006F008CFF39F0000E39226000E3F0F6FFAC
:102080006000E7F0F7FF000EF86E0F0EF76409D05E
:1020900009006F00D4FF38F009006F00D4FF39F059
:1020A0000CD06F00DBFFE9FF6F00DFFFEAFF6F007E
:1020B000B8FF38F06F00B8FF39F06000E3F0E6FFDA
:1020C0006000E7F0E6FFFB0EE3502B0F386EFC0ECE
:1020D0006F008CFF39F0000E39226000E3F0F6FF4C
:1020E0006000E7F0F7FF000EF86E0F0EF76409D0FE
:1020F00009006F00D4FF38F009006F00D4FF39F0F9
:102100000CD06F00DBFFE9FF6F00DFFFEAFF6F001D
:10211000B8FF38F06F00B8FF39F002D899EF10F02F
:102120000500FA6E3850FD6E3950FE6EFF6AFA50A7
:102130001200C0EF11F0FD0EE350010F386EFE0EDD
:102140006F008CFF39F0000E39226000E3F0E6FFEB
:102150006000E7F0E6FF4FEC55F0000EE66E000E73
:10216000E66EFB0EE350020F386EFC0E6F008CFF24
:1021700039F0000E39226000E3F0E6FF6000E7F07E
:10218000E6FF29EC60F0FD0EE3501C0F386EFE0EEA
:102190006F008CFF39F0000E39226000E3F0F6FF8B
:1021A0006000E7F0F7FF000EF86E0F0EF76404D042
:1021B000010EF56E0C0008D06F00DBFFE9FF6F0029
:1021C000DFFFEAFF010EEF6EC0EF11F0FD0EE350EE
:1021D000330F386EFE0E6F008CFF39F0000E39227F
:1021E0006000E3F0F6FF6000E7F0F7FF000EF86E26
:1021F0000F0EF76409D009006F00D4FF38F0090012
:102200006F00D4FF39F00CD06F00DBFFE9FF6F00E7
:10221000DFFFEAFF6F00B8FF38F06F00B8FF39F05A
:1022200038503910D8B417EF11F019EF11F0C0EF92
:1022300011F0FD0EE350350F386EFE0E6F008CFF6F
:1022400039F0000E39226000E3F0F6FF6000E7F09D
:10225000F7FF000EF86E0F0EF76409D009006F004B
:10226000D4FF38F009006F00D4FF39F00CD06F00B4
:10227000DBFFE9FF6F00DFFFEAFF6F00B8FF38F018
:102280006F00B8FF39F06000E3F0E6FF6000E7F0B0
:10229000E6FFFB0EE350330F386EFC0E6F008CFF31
:1022A00039F0000E39226000E3F0F6FF6000E7F03D
:1022B000F7FF000EF86E0F0EF76409D009006F00EB
:1022C000D4FF38F009006F00D4FF39F00CD06F0054
:1022D000DBFFE9FF6F00DFFFEAFF6F00B8FF38F0B8
:1022E0006F00B8FF39F002D87FEF11F00500FA6EE9
:1022F0003850FD6E3950FE6EFF6AFA501200C0EF82
:1023000011F0FD0E6F008FFFF6FFFE0E6F008FFFC6
:10231000F7FF000EF86E0F0EF76403D00800F550BB
:1023200007D06F00DBFFE9FF6F00DFFFEAFFEF5030
:10233000386E396A3950000AD8B4A1EF11F0C0EFF5
:1023400011F03850140AD8B4C0EF11F0010AD8B413
:10235000E6EF0DF0030AD8B4A2EF0EF0010AD8B4EC
:102360003DEF0FF00F0AD8B400EF10F0010AD8B417
:102370009BEF10F0030AD8B4E6EF10F0C0EF11F0B5
:10238000FB0EE126FF0EE2221200E652E6526F003B
:102390003CFE39F00F0E3916FE0E6000E7F0E3FF49
:1023A000FF0E6F0047FEE3FFFE0EE350100F911289
:1023B00098EF1AF080AEDFEF11F0E1EF11F0C6EF09
:1023C0001AF082A6E6EF11F0E8EF11F018EF12F024
:1023D000FC0E6F008FFFD9FFFD0E6F008FFFDAFF3D
:1023E000020EDF6E8250E66E8150E66E8450E66E1D
:1023F0008350E66E97EC49F0FC0E6F008CFF38F0CE
:10240000FD0E6F008CFF39F0010E3824D96E000EDE
:102410003920DA6E6000BBF0DEFF6000BFF0DEFF47
:102420006000C3F0DEFF6000C7F0DEFF42EF12F095
:10243000FC0E6F008FFFD9FFFD0E6F008FFFDAFFDC
:10244000010EDF6E8250E66E8150E66EC3EC55F0F1
:10245000FC0E6F008CFF38F0FD0E6F008CFF39F022
:10246000010E3824D96E000E3920DA6E6000BBF000
:10247000DEFF6000BFF0DEFF6000C3F0DEFF600043
:10248000C7F0DEFFFC0E6F008CFF38F0FD0E6F0012
:102490008CFF39F0050E3824D96E000E3920DA6E23
:1024A00085500F0BDF6EFC0E6F008CFF38F0FD0EB9
:1024B0006F008CFF39F00E0E3824D96E000E3920D3
:1024C000DA6E8544E846030BDF6EFC0E6F008CFF6E
:1024D00038F0FD0E6F008CFF39F0060E3824D96EEF
:1024E000000E3920DA6E6F001BFEDFFFFC0E6F005E
:1024F0008CFF38F0FD0E6F008CFF39F0070E38248A
:10250000D96E000E3920DA6E6F001FFEDFFFFC0E61
:102510006F008CFF38F0FD0E6F008CFF39F0080E55
:102520003824D96E000E3920DA6E6F0023FEDFFFEB
:10253000FC0E6F008CFF38F0FD0E6F008CFF39F041
:10254000090E3824D96E000E3920DA6E6F0027FE8E
:10255000DFFFFC0E6F008CFF38F0FD0E6F008CFF6C
:1025600039F00A0E3824D96E000E3920DA6E6F0069
:102570002BFEDFFFFC0E6F008CFF38F0FD0E6F00AE
:102580008CFF39F00B0E3824D96E000E3920DA6E2C
:102590006F002FFEDFFFFC0E6F008CFF38F0FD0E8A
:1025A0006F008CFF39F00C0E3824D96E000E3920E4
:1025B000DA6E6F0033FEDFFFFC0E6F008CFF38F029
:1025C000FD0E6F008CFF39F00D0E3824D96E000E11
:1025D0003920DA6E6F0037FEDFFF809EC6EF1AF0FB
:1025E0003701F0AFF6EF12F0F8EF12F0C6EF1AF085
:1025F00082A6FDEF12F0FFEF12F02FEF13F0FC0EAA
:102600006F008FFFD9FFFD0E6F008FFFDAFF020E04
:10261000DF6E8250E66E8150E66E8450E66E835027
:10262000E66E97EC49F0FC0E6F008CFF38F0FD0E63
:102630006F008CFF39F0010E3824D96E000E39205E
:10264000DA6E6000BBF0DEFF6000BFF0DEFF60000E
:10265000C3F0DEFF6000C7F0DEFF59EF13F0FC0EA1
:102660006F008FFFD9FFFD0E6F008FFFDAFF010EA5
:10267000DF6E8250E66E8150E66EC3EC55F0FC0EC4
:102680006F008CFF38F0FD0E6F008CFF39F0010EEB
:102690003824D96E000E3920DA6E6000BBF0DEFF00
:1026A0006000BFF0DEFF6000C3F0DEFF6000C7F037
:1026B000DEFFFC0E6F008CFF38F0FD0E6F008CFF0C
:1026C00039F0050E3824D96E000E3920DA6E8550A7
:1026D0000F0BDF6EFC0E6F008CFF38F0FD0E6F00ED
:1026E0008CFF39F00E0E3824D96E000E3920DA6EC8
:1026F0008544E846030BDF6EFC0E6F008CFF38F05C
:10270000FD0E6F008CFF39F0060E3824D96E000ED6
:102710003920DA6E6F001BFEDFFFFC0E6F008CFFAE
:1027200038F0FD0E6F008CFF39F0070E3824D96E9B
:10273000000E3920DA6E6F001FFEDFFFFC0E6F0007
:102740008CFF38F0FD0E6F008CFF39F0080E382436
:10275000D96E000E3920DA6E6F0023FEDFFFFC0E0B
:102760006F008CFF38F0FD0E6F008CFF39F0090E02
:102770003824D96E000E3920DA6E6F0027FEDFFF95
:10278000FC0E6F008CFF38F0FD0E6F008CFF39F0EF
:102790000A0E3824D96E000E3920DA6E6F002BFE37
:1027A000DFFFFC0E6F008CFF38F0FD0E6F008CFF1A
:1027B00039F00B0E3824D96E000E3920DA6E6F0016
:1027C0002FFEDFFFFC0E6F008CFF38F0FD0E6F0058
:1027D0008CFF39F00C0E3824D96E000E3920DA6ED9
:1027E0006F0033FEDFFFFC0E6F008CFF38F0FD0E34
:1027F0006F008CFF39F00D0E3824D96E000E392091
:10280000DA6E6F0037FEDFFF3701F09FEEEF12F058
:10281000370140AF0EEF14F010EF14F0C6EF1AF0CE
:1028200082A615EF14F017EF14F047EF14F0FC0E2A
:102830006F008FFFD9FFFD0E6F008FFFDAFF020ED2
:10284000DF6E8250E66E8150E66E8450E66E8350F5
:10285000E66E97EC49F0FC0E6F008CFF38F0FD0E31
:102860006F008CFF39F0010E3824D96E000E39202C
:10287000DA6E6000BBF0DEFF6000BFF0DEFF6000DC
:10288000C3F0DEFF6000C7F0DEFF71EF14F0FC0E56
:102890006F008FFFD9FFFD0E6F008FFFDAFF010E73
:1028A000DF6E8250E66E8150E66EC3EC55F0FC0E92
:1028B0006F008CFF38F0FD0E6F008CFF39F0010EB9
:1028C0003824D96E000E3920DA6E6000BBF0DEFFCE
:1028D0006000BFF0DEFF6000C3F0DEFF6000C7F005
:1028E000DEFFFC0E6F008CFF38F0FD0E6F008CFFDA
:1028F00039F0050E3824D96E000E3920DA6E855075
:102900000F0BDF6EFC0E6F008CFF38F0FD0E6F00BA
:102910008CFF39F00E0E3824D96E000E3920DA6E95
:102920008544E846030BDF6EFC0E6F008CFF38F029
:10293000FD0E6F008CFF39F0060E3824D96E000EA4
:102940003920DA6E6F001BFEDFFFFC0E6F008CFF7C
:1029500038F0FD0E6F008CFF39F0070E3824D96E69
:10296000000E3920DA6E6F001FFEDFFFFC0E6F00D5
:102970008CFF38F0FD0E6F008CFF39F0080E382404
:10298000D96E000E3920DA6E6F0023FEDFFFFC0ED9
:102990006F008CFF38F0FD0E6F008CFF39F0090ED0
:1029A0003824D96E000E3920DA6E6F0027FEDFFF63
:1029B000FC0E6F008CFF38F0FD0E6F008CFF39F0BD
:1029C0000A0E3824D96E000E3920DA6E6F002BFE05
:1029D000DFFFFC0E6F008CFF38F0FD0E6F008CFFE8
:1029E00039F00B0E3824D96E000E3920DA6E6F00E4
:1029F0002FFEDFFFFC0E6F008CFF38F0FD0E6F0026
:102A00008CFF39F00C0E3824D96E000E3920DA6EA6
:102A10006F0033FEDFFFFC0E6F008CFF38F0FD0E01
:102A20006F008CFF39F00D0E3824D96E000E39205E
:102A3000DA6E6F0037FEDFFF3701409FEEEF12F0D6
:102A4000370150AF26EF15F028EF15F0C6EF1AF05A
:102A500082A62DEF15F02FEF15F05FEF15F0FC0EAD
:102A60006F008FFFD9FFFD0E6F008FFFDAFF020EA0
:102A7000DF6E8250E66E8150E66E8450E66E8350C3
:102A8000E66E97EC49F0FC0E6F008CFF38F0FD0EFF
:102A90006F008CFF39F0010E3824D96E000E3920FA
:102AA000DA6E6000BBF0DEFF6000BFF0DEFF6000AA
:102AB000C3F0DEFF6000C7F0DEFF89EF15F0FC0E0B
:102AC0006F008FFFD9FFFD0E6F008FFFDAFF010E41
:102AD000DF6E8250E66E8150E66EC3EC55F0FC0E60
:102AE0006F008CFF38F0FD0E6F008CFF39F0010E87
:102AF0003824D96E000E3920DA6E6000BBF0DEFF9C
:102B00006000BFF0DEFF6000C3F0DEFF6000C7F0D2
:102B1000DEFFFC0E6F008CFF38F0FD0E6F008CFFA7
:102B200039F0050E3824D96E000E3920DA6E855042
:102B30000F0BDF6EFC0E6F008CFF38F0FD0E6F0088
:102B40008CFF39F00E0E3824D96E000E3920DA6E63
:102B50008544E846030BDF6EFC0E6F008CFF38F0F7
:102B6000FD0E6F008CFF39F0060E3824D96E000E72
:102B70003920DA6E6F001BFEDFFFFC0E6F008CFF4A
:102B800038F0FD0E6F008CFF39F0070E3824D96E37
:102B9000000E3920DA6E6F001FFEDFFFFC0E6F00A3
:102BA0008CFF38F0FD0E6F008CFF39F0080E3824D2
:102BB000D96E000E3920DA6E6F0023FEDFFFFC0EA7
:102BC0006F008CFF38F0FD0E6F008CFF39F0090E9E
:102BD0003824D96E000E3920DA6E6F0027FEDFFF31
:102BE000FC0E6F008CFF38F0FD0E6F008CFF39F08B
:102BF0000A0E3824D96E000E3920DA6E6F002BFED3
:102C0000DFFFFC0E6F008CFF38F0FD0E6F008CFFB5
:102C100039F00B0E3824D96E000E3920DA6E6F00B1
:102C20002FFEDFFFFC0E6F008CFF38F0FD0E6F00F3
:102C30008CFF39F00C0E3824D96E000E3920DA6E74
:102C40006F0033FEDFFFFC0E6F008CFF38F0FD0ECF
:102C50006F008CFF39F00D0E3824D96E000E39202C
:102C6000DA6E6F0037FEDFFF3701509FEEEF12F094
:102C7000370160AF3EEF16F040EF16F0C6EF1AF0E6
:102C800082A645EF16F047EF16F077EF16F0FC0E30
:102C90006F008FFFD9FFFD0E6F008FFFDAFF020E6E
:102CA000DF6E8250E66E8150E66E8450E66E835091
:102CB000E66E97EC49F0FC0E6F008CFF38F0FD0ECD
:102CC0006F008CFF39F0010E3824D96E000E3920C8
:102CD000DA6E6000BBF0DEFF6000BFF0DEFF600078
:102CE000C3F0DEFF6000C7F0DEFFA1EF16F0FC0EC0
:102CF0006F008FFFD9FFFD0E6F008FFFDAFF010E0F
:102D0000DF6E8250E66E8150E66EC3EC55F0FC0E2D
:102D10006F008CFF38F0FD0E6F008CFF39F0010E54
:102D20003824D96E000E3920DA6E6000BBF0DEFF69
:102D30006000BFF0DEFF6000C3F0DEFF6000C7F0A0
:102D4000DEFFFC0E6F008CFF38F0FD0E6F008CFF75
:102D500039F0050E3824D96E000E3920DA6E855010
:102D60000F0BDF6EFC0E6F008CFF38F0FD0E6F0056
:102D70008CFF39F00E0E3824D96E000E3920DA6E31
:102D80008544E846030BDF6EFC0E6F008CFF38F0C5
:102D9000FD0E6F008CFF39F0060E3824D96E000E40
:102DA0003920DA6E6F001BFEDFFFFC0E6F008CFF18
:102DB00038F0FD0E6F008CFF39F0070E3824D96E05
:102DC000000E3920DA6E6F001FFEDFFFFC0E6F0071
:102DD0008CFF38F0FD0E6F008CFF39F0080E3824A0
:102DE000D96E000E3920DA6E6F0023FEDFFFFC0E75
:102DF0006F008CFF38F0FD0E6F008CFF39F0090E6C
:102E00003824D96E000E3920DA6E6F0027FEDFFFFE
:102E1000FC0E6F008CFF38F0FD0E6F008CFF39F058
:102E20000A0E3824D96E000E3920DA6E6F002BFEA0
:102E3000DFFFFC0E6F008CFF38F0FD0E6F008CFF83
:102E400039F00B0E3824D96E000E3920DA6E6F007F
:102E50002FFEDFFFFC0E6F008CFF38F0FD0E6F00C1
:102E60008CFF39F00C0E3824D96E000E3920DA6E42
:102E70006F0033FEDFFFFC0E6F008CFF38F0FD0E9D
:102E80006F008CFF39F00D0E3824D96E000E3920FA
:102E9000DA6E6F0037FEDFFF3701609FEEEF12F052
:102EA000370170AF56EF17F058EF17F0C6EF1AF072
:102EB00082A65DEF17F05FEF17F08FEF17F0FC0EB3
:102EC0006F008FFFD9FFFD0E6F008FFFDAFF020E3C
:102ED000DF6E8250E66E8150E66E8450E66E83505F
:102EE000E66E97EC49F0FC0E6F008CFF38F0FD0E9B
:102EF0006F008CFF39F0010E3824D96E000E392096
:102F0000DA6E6000BBF0DEFF6000BFF0DEFF600045
:102F1000C3F0DEFF6000C7F0DEFFB9EF17F0FC0E74
:102F20006F008FFFD9FFFD0E6F008FFFDAFF010EDC
:102F3000DF6E8250E66E8150E66EC3EC55F0FC0EFB
:102F40006F008CFF38F0FD0E6F008CFF39F0010E22
:102F50003824D96E000E3920DA6E6000BBF0DEFF37
:102F60006000BFF0DEFF6000C3F0DEFF6000C7F06E
:102F7000DEFFFC0E6F008CFF38F0FD0E6F008CFF43
:102F800039F0050E3824D96E000E3920DA6E8550DE
:102F90000F0BDF6EFC0E6F008CFF38F0FD0E6F0024
:102FA0008CFF39F00E0E3824D96E000E3920DA6EFF
:102FB0008544E846030BDF6EFC0E6F008CFF38F093
:102FC000FD0E6F008CFF39F0060E3824D96E000E0E
:102FD0003920DA6E6F001BFEDFFFFC0E6F008CFFE6
:102FE00038F0FD0E6F008CFF39F0070E3824D96ED3
:102FF000000E3920DA6E6F001FFEDFFFFC0E6F003F
:103000008CFF38F0FD0E6F008CFF39F0080E38246D
:10301000D96E000E3920DA6E6F0023FEDFFFFC0E42
:103020006F008CFF38F0FD0E6F008CFF39F0090E39
:103030003824D96E000E3920DA6E6F0027FEDFFFCC
:10304000FC0E6F008CFF38F0FD0E6F008CFF39F026
:103050000A0E3824D96E000E3920DA6E6F002BFE6E
:10306000DFFFFC0E6F008CFF38F0FD0E6F008CFF51
:1030700039F00B0E3824D96E000E3920DA6E6F004D
:103080002FFEDFFFFC0E6F008CFF38F0FD0E6F008F
:103090008CFF39F00C0E3824D96E000E3920DA6E10
:1030A0006F0033FEDFFFFC0E6F008CFF38F0FD0E6B
:1030B0006F008CFF39F00D0E3824D96E000E3920C8
:1030C000DA6E6F0037FEDFFF3701709FEEEF12F010
:1030D000370180AF6EEF18F070EF18F0C6EF1AF0FE
:1030E00082A675EF18F077EF18F0A7EF18F0FC0E36
:1030F0006F008FFFD9FFFD0E6F008FFFDAFF020E0A
:10310000DF6E8250E66E8150E66E8450E66E83502C
:10311000E66E97EC49F0FC0E6F008CFF38F0FD0E68
:103120006F008CFF39F0010E3824D96E000E392063
:10313000DA6E6000BBF0DEFF6000BFF0DEFF600013
:10314000C3F0DEFF6000C7F0DEFFD1EF18F0FC0E29
:103150006F008FFFD9FFFD0E6F008FFFDAFF010EAA
:10316000DF6E8250E66E8150E66EC3EC55F0FC0EC9
:103170006F008CFF38F0FD0E6F008CFF39F0010EF0
:103180003824D96E000E3920DA6E6000BBF0DEFF05
:103190006000BFF0DEFF6000C3F0DEFF6000C7F03C
:1031A000DEFFFC0E6F008CFF38F0FD0E6F008CFF11
:1031B00039F0050E3824D96E000E3920DA6E8550AC
:1031C0000F0BDF6EFC0E6F008CFF38F0FD0E6F00F2
:1031D0008CFF39F00E0E3824D96E000E3920DA6ECD
:1031E0008544E846030BDF6EFC0E6F008CFF38F061
:1031F000FD0E6F008CFF39F0060E3824D96E000EDC
:103200003920DA6E6F001BFEDFFFFC0E6F008CFFB3
:1032100038F0FD0E6F008CFF39F0070E3824D96EA0
:10322000000E3920DA6E6F001FFEDFFFFC0E6F000C
:103230008CFF38F0FD0E6F008CFF39F0080E38243B
:10324000D96E000E3920DA6E6F0023FEDFFFFC0E10
:103250006F008CFF38F0FD0E6F008CFF39F0090E07
:103260003824D96E000E3920DA6E6F0027FEDFFF9A
:10327000FC0E6F008CFF38F0FD0E6F008CFF39F0F4
:103280000A0E3824D96E000E3920DA6E6F002BFE3C
:10329000DFFFFC0E6F008CFF38F0FD0E6F008CFF1F
:1032A00039F00B0E3824D96E000E3920DA6E6F001B
:1032B0002FFEDFFFFC0E6F008CFF38F0FD0E6F005D
:1032C0008CFF39F00C0E3824D96E000E3920DA6EDE
:1032D0006F0033FEDFFFFC0E6F008CFF38F0FD0E39
:1032E0006F008CFF39F00D0E3824D96E000E392096
:1032F000DA6E6F0037FEDFFF3701809FEEEF12F0CE
:10330000370190AF86EF19F088EF19F0C6EF1AF089
:1033100082A68DEF19F08FEF19F0BFEF19F0FC0EB8
:103320006F008FFFD9FFFD0E6F008FFFDAFF020ED7
:10333000DF6E8250E66E8150E66E8450E66E8350FA
:10334000E66E97EC49F0FC0E6F008CFF38F0FD0E36
:103350006F008CFF39F0010E3824D96E000E392031
:10336000DA6E6000BBF0DEFF6000BFF0DEFF6000E1
:10337000C3F0DEFF6000C7F0DEFFE9EF19F0FC0EDE
:103380006F008FFFD9FFFD0E6F008FFFDAFF010E78
:10339000DF6E8250E66E8150E66EC3EC55F0FC0E97
:1033A0006F008CFF38F0FD0E6F008CFF39F0010EBE
:1033B0003824D96E000E3920DA6E6000BBF0DEFFD3
:1033C0006000BFF0DEFF6000C3F0DEFF6000C7F00A
:1033D000DEFFFC0E6F008CFF38F0FD0E6F008CFFDF
:1033E00039F0050E3824D96E000E3920DA6E85507A
:1033F0000F0BDF6EFC0E6F008CFF38F0FD0E6F00C0
:103400008CFF39F00E0E3824D96E000E3920DA6E9A
:103410008544E846030BDF6EFC0E6F008CFF38F02E
:10342000FD0E6F008CFF39F0060E3824D96E000EA9
:103430003920DA6E6F001BFEDFFFFC0E6F008CFF81
:1034400038F0FD0E6F008CFF39F0070E3824D96E6E
:10345000000E3920DA6E6F001FFEDFFFFC0E6F00DA
:103460008CFF38F0FD0E6F008CFF39F0080E382409
:10347000D96E000E3920DA6E6F0023FEDFFFFC0EDE
:103480006F008CFF38F0FD0E6F008CFF39F0090ED5
:103490003824D96E000E3920DA6E6F0027FEDFFF68
:1034A000FC0E6F008CFF38F0FD0E6F008CFF39F0C2
:1034B0000A0E3824D96E000E3920DA6E6F002BFE0A
:1034C000DFFFFC0E6F008CFF38F0FD0E6F008CFFED
:1034D00039F00B0E3824D96E000E3920DA6E6F00E9
:1034E0002FFEDFFFFC0E6F008CFF38F0FD0E6F002B
:1034F0008CFF39F00C0E3824D96E000E3920DA6EAC
:103500006F0033FEDFFFFC0E6F008CFF38F0FD0E06
:103510006F008CFF39F00D0E3824D96E000E392063
:10352000DA6E6F0037FEDFFF3701909FEEEF12F08B
:10353000FE0EE350386E396A3950000AD8B4A3EF52
:103540001AF0C6EF1AF03850000AD8B4DAEF11F0CA
:10355000010AD8B4F0EF12F0030AD8B408EF14F05F
:10356000010AD8B420EF15F0070AD8B438EF16F0E6
:10357000010AD8B450EF17F0030AD8B468EF18F076
:10358000010AD8B480EF19F0C6EF1AF0FF0E6F00F1
:103590008FFF91FFE552E552E552E5521200240EED
:1035A000E126000EE222DA0E6F008FFFE6FF6F00C9
:1035B0008FFFE6FF25EC63F0FC0E6000BFF0E3FF39
:1035C000FB0E6000BBF0E3FFFB0E6F008FFFF6FF0A
:1035D000FC0E6F008FFFF7FF000EF86E0F0EF76402
:1035E00003D00800F55007D06F00DBFFE9FF6F0044
:1035F000DFFFEAFFEF50396EFF0E6000E7F0E3FFF8
:10360000DA0E6F008FFFE6FF6F008FFFE6FFE5EC3D
:1036100063F0DA0E6F008FFFE6FF6F008FFFE6FFAB
:1036200087EC62F0E5526F009CFF45F0E5526F00B9
:103630009CFF44F0E5526F009CFF43F0E5526F00A1
:103640009CFF42F0E5526F009CFF41F0E5526F0095
:103650009CFF40F0E5526F009CFF3FF0E5526F0089
:103660009CFF3EF0EB0E6000FBF0E3FFEC0E600011
:10367000FFF0E3FFED0E600003F1E3FFEE0E6000EC
:1036800007F1E3FFEF0E60000BF1E3FFF00E6000C7
:103690000FF1E3FFF10E600013F1E3FFF20E6000A3
:1036A00017F1E3FFEB0E6F008CFF36F0EC0E6F00AE
:1036B0008CFF37F0ED0E6F008CFF38F0EE0E6F00D0
:1036C0008CFF39F0F70E6000DBF0E3FFF80E6000CE
:1036D000DFF0E3FFF90E6000E3F0E3FFFA0E6000B5
:1036E000E7F0E3FF85EF22F0DA0E6F008FFFD9FFDE
:1036F000DB0E6F008FFFDAFFDF500A0AD8A483EFDA
:103700001BF085EF1BF0B0EF22F0FB0E6F008FFF78
:10371000F6FFFC0E6F008FFFF7FF000EF86E0F0E26
:10372000F76404D00B0EF56E0C0008D06F00DBFFC1
:10373000E9FF6F00DFFFEAFF0B0EEF6EB0EF22F044
:10374000DA0E6F008FFFD9FFDB0E6F008FFFDAFFFD
:10375000DF500B0AD8A4AFEF1BF0B1EF1BF0BFEFA7
:103760001CF0FB0EE350020F386EFC0E6F008CFF56
:1037700039F0000E39226000E3F0F6FF6000E7F058
:10378000F7FF000EF86E0F0EF76409D009006F0006
:10379000D4FF38F009006F00D4FF39F00CD06F006F
:1037A000DBFFE9FF6F00DFFFEAFF6F00B8FF38F0D3
:1037B0006F00B8FF39F038503910D8B4E2EF1BF081
:1037C000E4EF1BF0BFEF1CF0EF0EE124D96EFF0E0B
:1037D000E220DA6E6F0078FF36F06F0078FF37F086
:1037E0006F0078FF38F06F0078FF39F036503E6E8A
:1037F00037503F6E3850406E3950416E426A436ACE
:10380000446A456AEB0E6000FBF0E3FFEC0E6000DB
:10381000FFF0E3FFED0E600003F1E3FFEE0E60004A
:1038200007F1E3FFEF0E60000BF1E3FFF00E600025
:103830000FF1E3FFF10E600013F1E3FFF20E600001
:1038400017F1E3FFEB0E6F008CFF36F0EC0E6F000C
:103850008CFF37F0ED0E6F008CFF38F0EE0E6F002E
:103860008CFF39F0F30E6000DBF0E3FFF40E600034
:10387000DFF0E3FFF50E6000E3F0E3FFF60E60001B
:10388000E7F0E3FFF30E6F008CFF2EF0FD0E6000FB
:10389000BBF0E3FFE150FD0FD96EE250DA6EFF0E90
:1038A000DA22DF3A0F0EDF16FD0E6F008CFF2EF0CE
:1038B0000F0E2E16FD0E6000BBF0E3FFF40EE124A8
:1038C000D96EFF0EE220DA6EDF50396EFE0E600018
:1038D000E7F0E3FFE150FE0FD96EE250DA6EFF0E23
:1038E000DA22DF3A0F0EDF16F70E6F008FFFE6FFCA
:1038F0006F008FFFE6FF6F008FFFE6FF6F008FFF07
:10390000E6FF000EE66EF80EE350E66EF80EE350AA
:10391000E66EF40EE350020F386EF50E6F008CFF6A
:1039200039F0000E39226000E3F0F6FF6000E7F0A6
:10393000F7FF000EF86E0F0EF76409D009006F0054
:10394000D4FF38F009006F00D4FF39F00CD06F00BD
:10395000DBFFE9FF6F00DFFFEAFF6F00B8FF38F021
:103960006F00B8FF39F002D8BFEF1CF00500FA6E07
:103970003850FD6E3950FE6EFF6AFA501200DA0EB2
:103980006F008FFFD9FFDB0E6F008FFFDAFFDF5074
:103990000C0AD8A4CEEF1CF0D0EF1CF0DEEF1DF027
:1039A000FB0EE350020F386EFC0E6F008CFF39F0F7
:1039B000000E39226000E3F0F6FF6000E7F0F7FF49
:1039C000000EF86E0F0EF76409D009006F00D4FFE7
:1039D00038F009006F00D4FF39F00CD06F00DBFF26
:1039E000E9FF6F00DFFFEAFF6F00B8FF38F06F00FC
:1039F000B8FF39F038503910D8B401EF1DF003EF9B
:103A00001DF0DEEF1DF0EF0EE124D96EFF0EE22077
:103A1000DA6E6F0078FF36F06F0078FF37F06F00D6
:103A200078FF38F06F0078FF39F036503E6E37502F
:103A30003F6E3850406E3950416E426A436A446A64
:103A4000456AEB0E6000FBF0E3FFEC0E6000FFF058
:103A5000E3FFED0E600003F1E3FFEE0E600007F1FF
:103A6000E3FFEF0E60000BF1E3FFF00E60000FF1DB
:103A7000E3FFF10E600013F1E3FFF20E600017F1B7
:103A8000E3FFEB0E6F008CFF36F0EC0E6F008CFF47
:103A900037F0ED0E6F008CFF38F0EE0E6F008CFFEC
:103AA00039F0F30E6000DBF0E3FFF40E6000DFF0AE
:103AB000E3FFF50E6000E3F0E3FFF60E6000E7F0D1
:103AC000E3FFF30E6F008CFF2EF0FD0E6000BBF0E5
:103AD000E3FFE150FD0FD96EE250DA6EFF0EDA22FD
:103AE000DF3A0F0EDF16FD0E6F008CFF2EF00F0E6B
:103AF0002E16FD0E6000BBF0E3FFF40EE124D96E3C
:103B0000FF0EE220DA6EDF50396EFE0E6000E7F045
:103B1000E3FFE150FE0FD96EE250DA6EFF0EDA22BB
:103B2000DF3A0F0EDF16F70E6F008FFFE6FF6F0014
:103B30008FFFE6FF6F008FFFE6FF6F008FFFE6FF4E
:103B4000010EE66EF80EE350E66EF80EE350E66EF8
:103B5000F40EE350020F386EF50E6F008CFF39F053
:103B6000000E39226000E3F0F6FF6000E7F0F7FF97
:103B7000000EF86E0F0EF76409D009006F00D4FF35
:103B800038F009006F00D4FF39F00CD06F00DBFF74
:103B9000E9FF6F00DFFFEAFF6F00B8FF38F06F004A
:103BA000B8FF39F002D8DEEF1DF00500FA6E38508C
:103BB000FD6E3950FE6EFF6AFA501200DA0E6F0089
:103BC0008FFFD9FFDB0E6F008FFFDAFFDF500D0A8A
:103BD000D8A4EDEF1DF0EFEF1DF0CCEF1EF0DC0EE2
:103BE000E36AE32AE10EE124D96EFF0EE220DA6EE9
:103BF000040EDF6EEA0EE124D96EFF0EE220DA6ECB
:103C0000DF6AE20EE124D96EFF0EE220DA6EEB0EDF
:103C10006F008FFFDFFF080E396EE150EB0FD96E9A
:103C2000E250DA6EFF0EDA223928DE5227EF1EF05C
:103C3000DE52DE52DE52DE52DE52DE52D890DD32ED
:103C4000DD32DD32DD32DD32DD32DD32DE32E82EF4
:103C500018EF1EF0E30EE124D96EFF0EE220DA6EBB
:103C6000EB0E6F008FFFDFFF080E396EE150EB0F98
:103C7000D96EE250DA6EFF0EDA223928DE5250EFAA
:103C80001EF0DE52DE52DE52DE52DE52DE52D8909E
:103C9000DD32DD32DD32DD32DD32DD32DD32DE32AB
:103CA000E82E41EF1EF0E40EE124D96EFF0EE22073
:103CB000DA6EEB0E6F008FFFDFFF080E396EE150FA
:103CC000EB0FD96EE250DA6EFF0EDA223928DE529F
:103CD00079EF1EF0DE52DE52DE52DE52DE52DE524E
:103CE000D890DD32DD32DD32DD32DD32DD32DD3203
:103CF000DE32E82E6AEF1EF0E50EE124D96EFF0EEB
:103D0000E220DA6EEB0E6F008FFFDFFF080E396ED8
:103D1000E150EB0FD96EE250DA6EFF0EDA2239284D
:103D2000DE52A2EF1EF0DE52DE52DE52DE52DE52D4
:103D3000DE52D890DD32DD32DD32DD32DD32DD3291
:103D4000DD32DE32E82E93EF1EF0E150EB0FD96E3C
:103D5000E250DA6EFF0EDA22DD0EE124E96EFF0E8C
:103D6000E220EA6E6F007BFFEEFF6F007BFFEEFF4D
:103D70006F007BFFEEFF6F007BFFEEFFDC0EE124A8
:103D80002E6EFF0EE2202F6E6000BBF0E6FF60009B
:103D9000BFF0E6FFF6EC37F0DA0E6F008FFFD9FFC9
:103DA000DB0E6F008FFFDAFFDF500E0AD8A4DBEFC7
:103DB0001EF0DDEF1EF0BAEF1FF0DC0EE36AE32A1F
:103DC000E10EE124D96EFF0EE220DA6E020EDF6E04
:103DD000EA0EE124D96EFF0EE220DA6EDF6AE20E0F
:103DE000E124D96EFF0EE220DA6EEB0E6F008FFF3A
:103DF000DFFF080E396EE150EB0FD96EE250DA6E3C
:103E0000FF0EDA223928DE5215EF1FF0DE52DE52A5
:103E1000DE52DE52DE52DE52D890DD32DD32DD324D
:103E2000DD32DD32DD32DD32DE32E82E06EF1FF02C
:103E3000E30EE124D96EFF0EE220DA6EEB0E6F0086
:103E40008FFFDFFF080E396EE150EB0FD96EE250A5
:103E5000DA6EFF0EDA223928DE523EEF1FF0DE5214
:103E6000DE52DE52DE52DE52DE52D890DD32DD32DC
:103E7000DD32DD32DD32DD32DD32DE32E82E2FEFB3
:103E80001FF0E40EE124D96EFF0EE220DA6EEB0E95
:103E90006F008FFFDFFF080E396EE150EB0FD96E18
:103EA000E250DA6EFF0EDA223928DE5267EF1FF099
:103EB000DE52DE52DE52DE52DE52DE52D890DD326B
:103EC000DD32DD32DD32DD32DD32DD32DE32E82E72
:103ED00058EF1FF0E50EE124D96EFF0EE220DA6EF6
:103EE000EB0E6F008FFFDFFF080E396EE150EB0F16
:103EF000D96EE250DA6EFF0EDA223928DE5290EFE8
:103F00001FF0DE52DE52DE52DE52DE52DE52D8901A
:103F1000DD32DD32DD32DD32DD32DD32DD32DE3228
:103F2000E82E81EF1FF0E150EB0FD96EE250DA6E10
:103F3000FF0EDA22DD0EE124E96EFF0EE220EA6ECA
:103F40006F007BFFEEFF6F007BFFEEFF6F007BFFDC
:103F5000EEFF6F007BFFEEFFDC0EE1242E6EFF0E06
:103F6000E2202F6E6000BBF0E6FF6000BFF0E6FFCE
:103F7000F6EC37F0DA0E6F008FFFD9FFDB0E6F0023
:103F80008FFFDAFFDF500F0AD8A4C9EF1FF0CBEF85
:103F90001FF0A8EF20F0DC0EE36AE32AE10EE12433
:103FA000D96EFF0EE220DA6E010EDF6EEA0EE1241A
:103FB000D96EFF0EE220DA6EDF6AE20EE124D96EDE
:103FC000FF0EE220DA6EEB0E6F008FFFDFFF080EB0
:103FD000396EE150EB0FD96EE250DA6EFF0EDA2245
:103FE0003928DE5203EF20F0DE52DE52DE52DE527E
:103FF000DE52DE52D890DD32DD32DD32DD32DD32AE
:10400000DD32DD32DE32E82EF4EF1FF0E30EE12484
:10401000D96EFF0EE220DA6EEB0E6F008FFFDFFF2E
:10402000080E396EE150EB0FD96EE250DA6EFF0EDA
:10403000DA223928DE522CEF20F0DE52DE52DE5238
:10404000DE52DE52DE52D890DD32DD32DD32DD323C
:10405000DD32DD32DD32DE32E82E1DEF20F0E40EFF
:10406000E124D96EFF0EE220DA6EEB0E6F008FFFB7
:10407000DFFF080E396EE150EB0FD96EE250DA6EB9
:10408000FF0EDA223928DE5255EF20F0DE52DE52E2
:10409000DE52DE52DE52DE52D890DD32DD32DD32CB
:1040A000DD32DD32DD32DD32DE32E82E46EF20F069
:1040B000E50EE124D96EFF0EE220DA6EEB0E6F0002
:1040C0008FFFDFFF080E396EE150EB0FD96EE25023
:1040D000DA6EFF0EDA223928DE527EEF20F0DE5251
:1040E000DE52DE52DE52DE52DE52D890DD32DD325A
:1040F000DD32DD32DD32DD32DD32DE32E82E6FEFF1
:1041000020F0E150EB0FD96EE250DA6EFF0EDA22AA
:10411000DD0EE124E96EFF0EE220EA6E6F007BFF08
:10412000EEFF6F007BFFEEFF6F007BFFEEFF6F0087
:104130007BFFEEFFDC0EE1242E6EFF0EE2202F6EE1
:104140006000BBF0E6FF6000BFF0E6FFF6EC37F082
:10415000DA0E6F008FFFD9FFDB0E6F008FFFDAFFE3
:10416000DF50100AD8A4B7EF20F0B9EF20F095EF98
:1041700021F0DC0EE36AE32AE10EE124D96EFF0EA2
:10418000E220DA6EDF6AEA0EE124D96EFF0EE22049
:10419000DA6EDF6AE20EE124D96EFF0EE220DA6EFB
:1041A000EB0E6F008FFFDFFF080E396EE150EB0F53
:1041B000D96EE250DA6EFF0EDA223928DE52F0EFC5
:1041C00020F0DE52DE52DE52DE52DE52DE52D89057
:1041D000DD32DD32DD32DD32DD32DD32DD32DE3266
:1041E000E82EE1EF20F0E30EE124D96EFF0EE2208D
:1041F000DA6EEB0E6F008FFFDFFF080E396EE150B5
:10420000EB0FD96EE250DA6EFF0EDA223928DE5259
:1042100019EF21F0DE52DE52DE52DE52DE52DE5265
:10422000D890DD32DD32DD32DD32DD32DD32DD32BD
:10423000DE32E82E0AEF21F0E40EE124D96EFF0E03
:10424000E220DA6EEB0E6F008FFFDFFF080E396E93
:10425000E150EB0FD96EE250DA6EFF0EDA22392808
:10426000DE5242EF21F0DE52DE52DE52DE52DE52EC
:10427000DE52D890DD32DD32DD32DD32DD32DD324C
:10428000DD32DE32E82E33EF21F0E50EE124D96E87
:10429000FF0EE220DA6EEB0E6F008FFFDFFF080EDD
:1042A000396EE150EB0FD96EE250DA6EFF0EDA2272
:1042B0003928DE526BEF21F0DE52DE52DE52DE5242
:1042C000DE52DE52D890DD32DD32DD32DD32DD32DB
:1042D000DD32DD32DE32E82E5CEF21F0E150EB0F13
:1042E000D96EE250DA6EFF0EDA22DD0EE124E96EBD
:1042F000FF0EE220EA6E6F007BFFEEFF6F007BFF98
:10430000EEFF6F007BFFEEFF6F007BFFEEFFDC0E2A
:10431000E1242E6EFF0EE2202F6E6000BBF0E6FF60
:104320006000BFF0E6FFF6EC37F0DA0E6F008FFFAB
:10433000D9FFDB0E6F008FFFDAFFDF50110AD8A420
:10434000A4EF21F0A6EF21F0B0EF22F0DC0EE36A3B
:10435000E32AE10EE124D96EFF0EE220DA6EDF6A75
:10436000EA0EE124D96EFF0EE220DA6E010EDF6E56
:10437000E20EE124D96EFF0EE220DA6EEB0E6F0042
:104380008FFFDFFF080E396EE150EB0FD96EE25060
:10439000DA6EFF0EDA223928DE52DEEF21F0DE522D
:1043A000DE52DE52DE52DE52DE52D890DD32DD3297
:1043B000DD32DD32DD32DD32DD32DE32E82ECFEFCE
:1043C00021F0E30EE124D96EFF0EE220DA6EEB0E4F
:1043D0006F008FFFDFFF080E396EE150EB0FD96ED3
:1043E000E250DA6EFF0EDA223928DE5207EF22F0B1
:1043F000DE52DE52DE52DE52DE52DE52D890DD3226
:10440000DD32DD32DD32DD32DD32DD32DE32E82E2C
:10441000F8EF21F0E40EE124D96EFF0EE220DA6E0F
:10442000EB0E6F008FFFDFFF080E396EE150EB0FD0
:10443000D96EE250DA6EFF0EDA223928DE5230EF02
:1044400022F0DE52DE52DE52DE52DE52DE52D890D2
:10445000DD32DD32DD32DD32DD32DD32DD32DE32E3
:10446000E82E21EF22F0E50EE124D96EFF0EE220C6
:10447000DA6EEB0E6F008FFFDFFF080E396EE15032
:10448000EB0FD96EE250DA6EFF0EDA223928DE52D7
:1044900059EF22F0DE52DE52DE52DE52DE52DE52A2
:1044A000D890DD32DD32DD32DD32DD32DD32DD323B
:1044B000DE32E82E4AEF22F0E150EB0FD96EE250E7
:1044C000DA6EFF0EDA22DD0EE124E96EFF0EE22045
:1044D000EA6E6F007BFFEEFF6F007BFFEEFF6F0069
:1044E0007BFFEEFF6F007BFFEEFFDC0EE1242E6E04
:1044F000FF0EE2202F6E6000BBF0E6FF6000BFF011
:10450000E6FFF6EC37F0B0EF22F0FB0E6F008FFF06
:10451000F6FFFC0E6F008FFFF7FF000EF86E0F0E18
:10452000F76403D00800F55007D06F00DBFFE9FF08
:104530006F00DFFFEAFFEF50386E396A3950000A2A
:10454000D8B4A5EF22F0B0EF22F038500A0AD8B460
:1045500074EF1BF0010AD8B4A0EF1BF0B0EF22F00B
:10456000FF0E6F008CFF39F0FB0E6F008FFFF6FF20
:10457000FC0E6F008FFFF7FF000EF86E0F0EF76452
:1045800003D00800F55007D06F00DBFFE9FF6F0094
:10459000DFFFEAFFEF503918D8B4D1EF22F0D3EFA4
:1045A00022F014EF23F0FF0EE350386E396A3950D1
:1045B000000AD8B4DEEF22F0E9EF22F038500A0A00
:1045C000D8B4E9EF22F0010AD8B4E9EF22F0E9EF1C
:1045D00022F0FB0E6F008FFFF6FFFC0E6F008FFFC7
:1045E000F7FF000EF86E0F0EF76403D00800F550C9
:1045F00007D06F00DBFFE9FF6F00DFFFEAFFEF503E
:10460000386E396A3950000AD8B409EF23F014EF34
:1046100023F038500A0AD8B414EF23F0010AD8B4B2
:1046200014EF23F014EF23F0DA0EE126FF0EE2225E
:1046300012000A0EE126000EE222EF0E6F008CFF40
:1046400036F0F00E6F008CFF37F0F10E6F008CFF2C
:1046500038F0F20E6F008CFF39F0F60E6000DBF0E0
:10466000E3FFF70E6000DFF0E3FFF80E6000E3F019
:10467000E3FFF90E6000E7F0E3FFF90EE124D96EE5
:10468000FF0EE220DA6EDF50396EFA0E6000E7F0BE
:10469000E3FFF80EE124D96EFF0EE220DA6EFB0E86
:1046A000E124E96EFF0EE220EA6E6F007FFFEFFF6C
:1046B000F70EE124D96EFF0EE220DA6EFC0EE12443
:1046C000E96EFF0EE220EA6E6F007FFFEFFFFD0E46
:1046D000E124D96EFF0EE220DA6EF60E6F008FFF36
:1046E000DFFFEF0E6F008CFF2EF0FE0E6000BBF0C0
:1046F000E3FFF00E6F008CFF2EF0FF0E6000BBF0AA
:10470000E3FF41EF29F0F40EE350D8A48AEF23F041
:104710008CEF23F0DEEF23F0F70EE124D96EFF0ECD
:10472000E220DA6EDF50D8B498EF23F09AEF23F04E
:104730009CEF23F0DCEC64F0F60E6F008CFF01F0D0
:10474000F90EE124D96EFF0EE220DA6EDF50026E20
:104750000150E66E010EE66EFFEC63F00250E66E6D
:10476000020EE66EFFEC63F00250E66ED3EC64F0EE
:104770006000BBF0E6FF6000BFF0E6FF54EC60F0C5
:10478000000EE66E000EE66E000EE66E000EE66EA1
:10479000000EE66E000EE66E000EE66E000EE66E91
:1047A000000EE66E000EE66ED3EC64F06000BBF027
:1047B000E6FF6000BFF0E6FFE5EC5CF0F40EE3041A
:1047C000D8A4E5EF23F0E7EF23F00AEF24F0E1505F
:1047D000FA0FD96EE250DA6EFF0EDA226F0078FF20
:1047E00003F06F0078FF04F06F0078FF05F06F00B2
:1047F00078FF06F060000FF0E6FF600013F0E6FFC0
:10480000600017F0E6FF60001BF0E6FF030EE66EA7
:10481000DBEC57F0F40E6F008CFF2EF0020E2E181A
:10482000D8A415EF24F017EF24F04CEF24F0E1505A
:10483000FA0FD96EE250DA6EFF0EDA226F0078FFBF
:1048400007F06F0078FF08F06F0078FF09F06F0045
:1048500078FF0AF060001FF0E6FF600023F0E6FF3B
:10486000600027F0E6FF60002BF0E6FF070EE66E23
:10487000DBEC57F060001FF0E6FF600023F0E6FF7E
:10488000600027F0E6FF60002BF0E6FF050EE66E05
:10489000000EE66E59EC3BF0F40E6F008CFF2EF02C
:1048A000030E2E18D8A457EF24F059EF24F07CEF14
:1048B00024F0E150FA0FD96EE250DA6EFF0EDA22E0
:1048C0006F0078FF0BF06F0078FF0CF06F0078FF3F
:1048D0000DF06F0078FF0EF060002FF0E6FF600033
:1048E00033F0E6FF600037F0E6FF60003BF0E6FFE4
:1048F0000B0EE66EDBEC57F0F40E6F008CFF2EF023
:10490000040E2E18D8A487EF24F089EF24F0A1EF2D
:1049100024F0F60E6F008CFF0FF0F70EE124D96E35
:10492000FF0EE220DA6EDF50106E0F50E66E0F0EB3
:10493000E66EFFEC63F01050E66E100EE66EFFECD4
:1049400063F0F40E6F008CFF2EF0050E2E18D8A425
:10495000ACEF24F0AEEF24F0D2EF24F0F60E6F00AF
:104960008CFF15F0F70EE124D96EFF0EE220DA6E0F
:10497000DF50196E1550E66E150EE66EFFEC63F013
:104980001950E66E190EE66EFFEC63F0000EE66E4F
:10499000000EE66EA7EC60F0020EE66E100EE66EFC
:1049A00064EC52F0F40E6F008CFF2EF0060E2E1801
:1049B000D8A4DDEF24F0DFEF24F043EF25F0F60E6E
:1049C0006F008CFF11F0F70EE124D96EFF0EE2208C
:1049D000DA6EDF50126EF80EE124D96EFF0EE2207F
:1049E000DA6EDF50136EF90EE124D96EFF0EE2206D
:1049F000DA6EDF50146E1150E66E110EE66EFFECAB
:104A000063F01250E66E120EE66EFFEC63F0135088
:104A1000E66E130EE66EFFEC63F01450E66E140EB5
:104A2000E66EFFEC63F01450E66ECAEC64F06000D2
:104A3000BBF0E6FF6000BFF0E6FF54EC60F0000E54
:104A4000E66E000EE66E000EE66E000EE66E000EDE
:104A5000E66E000EE66E000EE66E000EE66E000ECE
:104A6000E66E000EE66ECAEC64F06000BBF0E6FF96
:104A70006000BFF0E6FFE5EC5CF0000EE66E000EB5
:104A8000E66E5FEC5AF0F40E6F008CFF2EF0070E0E
:104A90002E18D8A44EEF25F050EF25F0AEEF25F0FC
:104AA000F60E6F008CFF18F0F70EE124D96EFF0EA2
:104AB000E220DA6EDF50166EF80EE124D96EFF0E9A
:104AC000E220DA6EDF50176E1850E66E180EE66EB2
:104AD000FFEC63F01650E66E160EE66EFFEC63F028
:104AE0001750E66E170EE66EFFEC63F01850E66E98
:104AF000B8EC64F0010E2E26000E2F226000BBF0F1
:104B0000E6FF6000BFF0E6FF54EC60F0000EE66EDA
:104B1000000EE66E000EE66E000EE66E000EE66E0D
:104B2000000EE66E000EE66E000EE66E000EE66EFD
:104B3000000EE66EB8EC64F0010E2E26000E2F2259
:104B40006000BBF0E6FF6000BFF0E6FFE5EC5CF064
:104B5000030EE66E100EE66E2EEC59F0F40E6F00AA
:104B60008CFF2EF0080E2E18D8A4B9EF25F0BBEF5D
:104B700025F0F5EF25F0F60E6F008CFF1AF0F70E1A
:104B8000E124D96EFF0EE220DA6EDF501B6EF80EC4
:104B9000E124D96EFF0EE220DA6EDF501C6EF90EB2
:104BA000E124D96EFF0EE220DA6EDF501D6E1A503E
:104BB000E66E1A0EE66EFFEC63F01B50E66E1B0EFF
:104BC000E66EFFEC63F01C50E66E1C0EE66EFFEC2A
:104BD00063F01D50E66E1D0EE66EFFEC63F0000EF6
:104BE000E66E000EE66E24EC5AF0F40E6F008CFFB9
:104BF0002EF0090E2E18D8A400EF26F002EF26F0B2
:104C00006BEF29F0F60E6F008CFF1EF0F70EE1241B
:104C1000D96EFF0EE220DA6EDF501F6E1E50E66E78
:104C20001E0EE66EFFEC63F01F50E66E1F0EE66E82
:104C3000FFEC63F06BEF29F0F40EE304D8A423EF4C
:104C400026F025EF26F04FEF26F0F70EE124D96E7F
:104C5000FF0EE220DA6EDF50E66EB2EC41F0F60EA7
:104C6000E350E66EB2EC44F0F80EE124D96EFF0E8C
:104C7000E220DA6EDF50D8A440EF26F043EF26F0B2
:104C8000010E44EF26F0000ED36FA6EC64F0600036
:104C9000BBF0E6FF6000BFF0E6FF71EC5CF0F40EE5
:104CA0006F008CFF2EF00F0E2E18D8A45AEF26F0AE
:104CB0005CEF26F06BEF29F0CAEC64F06000BBF00B
:104CC000E6FF6000BFF0E6FFC9EC63F0CAEC64F0F9
:104CD0006000BBF0D9FF6000BFF0DAFF180EDE18ED
:104CE000D8A475EF26F077EF26F06BEF29F0110EC0
:104CF000E66EC1EC64F02E50116E120EE66EC1EC41
:104D000064F02E50126E130EE66EC1EC64F02E505D
:104D1000136E140EE66EC1EC64F02E50146E145037
:104D2000E66ECAEC64F06000BBF0E6FF6000BFF026
:104D3000E6FF54EC60F0000EE66E000EE66E000E2C
:104D4000E66E000EE66E000EE66E000EE66E000EDB
:104D5000E66E000EE66E000EE66E000EE66ECAEC23
:104D600064F06000BBF0E6FF6000BFF0E6FF1FEC00
:104D70005DF0000EE66E000EE66E000EE66E000EB2
:104D8000E66E000EE66E000EE66E000EE66E000E9B
:104D9000E66E000EE66E000EE66ECAEC64F0600091
:104DA000BBF0E6FF6000BFF0E6FF93EC5DF0000EA5
:104DB000E66E000EE66E000EE66E000EE66E000E6B
:104DC000E66E000EE66E000EE66E000EE66E000E5B
:104DD000E66E000EE66ECAEC64F06000BBF0E6FF23
:104DE0006000BFF0E6FF59EC5DF06BEF29F0F40EC8
:104DF0006F008CFF2EF00F0E2E18D8A402EF27F0B4
:104E000004EF27F06BEF29F0F60E6F008CFFD6F061
:104E10000001D651D8A40FEF27F011EF27F019EFBA
:104E200027F0030EE66E100EE66E64EC61F06BEF99
:104E300029F0040EE66E100EE66E64EC61F06BEF86
:104E400029F0F40EE350D8A428EF27F02AEF27F03A
:104E500043EF27F0FA0E6F008FFFE6FF6F008FFF22
:104E6000E6FF6F008FFFE6FF6F008FFFE6FF20EC8D
:104E70004FF0B8EC64F06000BBF0E6FF6000BFF0FC
:104E8000E6FFABEC5CF0F40E6F008CFF2EF00F0E23
:104E90002E18D8A44EEF27F050EF27F06BEF29F033
:104EA000B8EC64F0010E2E26000E2F226000BBF03D
:104EB000E6FF6000BFF0E6FFC9EC63F0B8EC64F019
:104EC000010E2E24D96E000E2F20DA6E180EDE1879
:104ED000D8A46DEF27F06FEF27F06BEF29F0160ED7
:104EE000E66EC1EC64F02E50166E170EE66EC1EC45
:104EF00064F02E50176E180EE66EC1EC64F02E5062
:104F0000186E000EE66E000EE66E000EE66E000EE7
:104F1000E66E000EE66E000EE66E000EE66E000E09
:104F2000E66E000EE66E000EE66EB8EC64F0010E62
:104F30002E26000E2F226000BBF0E6FF6000BFF0BF
:104F4000E6FF1FEC5DF0000EE66E000EE66E000E52
:104F5000E66E000EE66E000EE66E000EE66E000EC9
:104F6000E66E000EE66E000EE66E000EE66EB8EC23
:104F700064F0010E2E26000E2F226000BBF0E6FF2B
:104F80006000BFF0E6FF93EC5DF06BEF29F0F40EEC
:104F9000E304D8A4CEEF27F0D0EF27F005EF28F0F8
:104FA000E150FA0FD96EE250DA6EFF0EDA226F008E
:104FB00078FFCBF06F0078FFCCF06F0078FFCDF07A
:104FC0006F0078FFCEF0000EE66E000EE66E000E6B
:104FD000E66E000EE66E000EE66E000EE66E000E49
:104FE000E66E000EE66E000EE66E000EE66EA6ECB5
:104FF00064F0010E2E26000E2F226000BBF0E6FFAB
:105000006000BFF0E6FF59EC5DF0F40E6F008CFF1E
:105010002EF00E0E2E18D8A410EF28F012EF28F064
:105020001FEF28F0F60EE350D8A419EF28F01CEF7C
:1050300028F0010E1DEF28F0000E0001D56FF40ED0
:105040006F008CFF2EF00F0E2E18D8A42AEF28F038
:105050002CEF28F06BEF29F0A6EC64F0010E2E2661
:10506000000E2F226000BBF0E6FF6000BFF0E6FFFD
:10507000C9EC63F0A6EC64F0010E2E24D96E000E8C
:105080002F20DA6E180EDE18D8A449EF28F04BEF67
:1050900028F095EF28F0190EE66EC1EC64F02E5062
:1050A000196E000EE66E000EE66E000EE66E000E45
:1050B000E66E000EE66E000EE66E000EE66E000E68
:1050C000E66EF40EE66E010EE66EA6EC64F0010EDE
:1050D0002E26000E2F226000BBF0E6FF6000BFF01E
:1050E000E6FF1FEC5DF0000EE66E000EE66E000EB1
:1050F000E66E000EE66E000EE66E000EE66E000E28
:10510000E66E000EE66EE80EE66E030EE66EA6ECA8
:1051100064F0010E2E26000E2F226000BBF0E6FF89
:105120006000BFF0E6FF93EC5DF0E150FE0FD96E3A
:10513000E250DA6EFF0EDA22DFA8A1EF28F0A3EF2B
:1051400028F06BEF29F0A6EC64F0010E2E24D96E46
:10515000000E2F20DA6E160EDE18D8A4B2EF28F05B
:10516000B4EF28F06BEF29F0000EE66E000EE66E4D
:10517000000EE66E000EE66E000EE66E000EE66EA7
:10518000000EE66E000EE66EE80EE66E030EE66EAC
:10519000A6EC64F0010E2E26000E2F226000BBF05C
:1051A000E6FF6000BFF0E6FF59EC5DF06BEF29F021
:1051B000F40E6F008CFF2EF0040E2E18D8A4E3EF2F
:1051C00028F0E5EF28F06BEF29F0B8EC64F0600010
:1051D000BBF0E6FF6000BFF0E6FFF4EC60F0A6EC89
:1051E00064F06000BBF0E6FF6000BFF0E6FFCEECCD
:1051F00060F0CAEC64F06000BBF0E6FF6000BFF056
:10520000E6FF63EC5FF0000EE66E000EE66E000E49
:10521000E66E000EE66E000EE66E000EE66E000E06
:10522000E66E000EE66E640EE66E000EE66ECAECEA
:1052300064F06000BBF0E6FF6000BFF0E6FF93ECB7
:105240005DF0000EE66E000EE66E000EE66E000EDD
:10525000E66E000EE66E000EE66E000EE66E000EC6
:10526000E66EC80EE66E000EE66ECAEC64F06000F4
:10527000BBF0E6FF6000BFF0E6FF59EC5DF06BEFBE
:1052800029F0F50EE350386E396A3950000AD8B467
:105290004CEF29F06BEF29F03850000AD8B483EFB7
:1052A00023F0020AD8B41CEF26F0010AD8B4F7EFB5
:1052B00026F0070AD8B421EF27F0010AD8B4C7EFC7
:1052C00027F0030AD8B4D8EF28F0010AD8B46BEF5E
:1052D00029F06BEF29F0EF0EE126FF0EE22212001B
:1052E000E652E652E652E652FA0E6F008FFFE6FFF4
:1052F0006F008FFFE6FF25EC63F0FD0E6000BFF04E
:10530000E3FFFC0E6000BBF0E3FFFC0E6F008FFFBD
:10531000F6FFFD0E6F008FFFF7FF000EF86E0F0E09
:10532000F76403D00800F55007D06F00DBFFE9FFFA
:105330006F00DFFFEAFFEF50396EFF0E6000E7F00D
:10534000E3FFFA0E6F008FFFE6FF6F008FFFE6FFAF
:10535000E5EC63F0FE0E6000BBF0E3FF2AEF2DF0FA
:10536000FA0E6F008FFFD9FFFB0E6F008FFFDAFF81
:10537000DF50C80AD8A4BFEF29F0C1EF29F05DEFD4
:105380002DF0FC0E6F008FFFF6FFFD0E6F008FFFFC
:10539000F7FF000EF86E0F0EF76404D0010EF56EE5
:1053A0000C0008D06F00DBFFE9FF6F00DFFFEAFFB2
:1053B000010EEF6E5DEF2DF0FC0EE350050F386E21
:1053C000FD0E6F008CFF39F0000E39226000E3F013
:1053D000F6FF6000E7F0F7FF000EF86E0F0EF764BF
:1053E00003D00800F55007D06F00DBFFE9FF6F0026
:1053F000DFFFEAFFEF50396EFC0EE350070F366E09
:10540000FD0E6F008CFF37F0000E37226000DBF0DE
:10541000F6FF6000DFF0F7FF000EF86E0F0EF76486
:1054200005D06000E7F0F5FF0C0009D06F00DBFF4E
:10543000E9FF6F00DFFFEAFF6000E7F0EFFFFE0E1D
:105440006F008CFF2EF0CA0E2E18D8A42AEF2AF077
:105450002CEF2AF09FEF2AF0FC0E6F008FFFF6FF73
:10546000FD0E6F008FFFF7FF000EF86E0F0EF76452
:1054700004D0020EF56E0C0008D06F00DBFFE9FFD0
:105480006F00DFFFEAFF020EEF6EFC0EE350060F27
:10549000386EFD0E6F008CFF39F0000E392260006F
:1054A000E3F0F6FF6000E7F0F7FF000EF86E0F0E76
:1054B000F76404D0010EF56E0C0008D06F00DBFF1E
:1054C000E9FF6F00DFFFEAFF010EEF6EFC0EE35015
:1054D000010F386EFD0E6F008CFF39F0000E39227F
:1054E0006000E3F0F6FF6000E7F0F7FF000EF86EF3
:1054F0000F0EF76409D009006F00D4FF38F00900DF
:105500006F00D4FF39F00CD06F00DBFFE9FF6F00B4
:10551000DFFFEAFF6F00B8FF38F06F00B8FF39F027
:105520006000E3F0E6FF6000E7F0E6FFFA0E6F00D0
:105530008FFFE6FF6F008FFFE6FFFEEC5FF0FE0ED1
:105540006F008CFF2EF0C90E2E18D8A4AAEF2AF0F7
:10555000ACEF2AF05DEF2DF0FC0E6F008FFFF6FF31
:10556000FD0E6F008FFFF7FF000EF86E0F0EF76451
:1055700004D0020EF56E0C0008D06F00DBFFE9FFCF
:105580006F00DFFFEAFF020EEF6EFC0EE350060F26
:10559000386EFD0E6F008CFF39F0000E392260006E
:1055A000E3F0F6FF6000E7F0F7FF000EF86E0F0E75
:1055B000F76404D0000EF56E0C0008D06F00DBFF1E
:1055C000E9FF6F00DFFFEAFF000EEF6EFC0EE35015
:1055D000010F386EFD0E6F008CFF39F0000E39227E
:1055E0006000E3F0F6FF6000E7F0F7FF000EF86EF2
:1055F0000F0EF76409D009006F00D4FF38F00900DE
:105600006F00D4FF39F00CD06F00DBFFE9FF6F00B3
:10561000DFFFEAFF6F00B8FF38F06F00B8FF39F026
:105620006000E3F0E6FF6000E7F0E6FFFA0E6F00CF
:105630008FFFE6FF6F008FFFE6FFFEEC5FF05DEF90
:105640002DF0FC0EE350060F386EFD0E6F008CFF40
:1056500039F0000E39226000E3F0F6FF6000E7F059
:10566000F7FF000EF86E0F0EF76403D00800F55038
:1056700007D06F00DBFFE9FF6F00DFFFEAFFEF50AD
:105680000009D8B446EF2BF048EF2BF08DEF2BF04C
:10569000FC0EE350070F386EFD0E6F008CFF39F0E3
:1056A000000E39226000E3F0F6FF6000E7F0F7FF3C
:1056B000000EF86E0F0EF76403D00800F55007D007
:1056C0006F00DBFFE9FF6F00DFFFEAFFEF50396E8D
:1056D000FF0E3926FC0EE350070F366EFD0E6F00ED
:1056E0008CFF37F0000E37226000DBF0F6FF600021
:1056F000DFF0F7FF000EF86E0F0EF76405D06000C4
:10570000E7F0F5FF0C0009D06F00DBFFE9FF6F0049
:10571000DFFFEAFF6000E7F0EFFFFE0E6F008CFF97
:105720002EF0CB0E2E18D8A498EF2BF09AEF2BF07A
:105730005DEF2DF0FC0E6F008FFFF6FFFD0E6F008A
:105740008FFFF7FF000EF86E0F0EF76404D0030E04
:10575000F56E0C0008D06F00DBFFE9FF6F00DFFF84
:10576000EAFF030EEF6EFC0EE350030F386EFD0EE2
:105770006F008CFF39F0000E39226000E3F0F6FF75
:105780006000E7F0F7FF000EF86E0F0EF76409D027
:1057900009006F00D4FF38F009006F00D4FF39F022
:1057A0000CD06F00DBFFE9FF6F00DFFFEAFF6F0047
:1057B000B8FF38F06F00B8FF39F06000E3F0E6FFA3
:1057C0006000E7F0E6FFFA0E6F008FFFE6FF6F0064
:1057D0008FFFE6FFFEEC5FF05DEF2DF0FE0E6F0039
:1057E0008CFF2EF0CB0E2E18D8A4F9EF2BF0FBEF88
:1057F0002BF05DEF2DF0FC0EE350070F386EFD0E21
:105800006F008CFF39F0000E39226000E3F0F6FFE4
:105810006000E7F0F7FF000EF86E0F0EF76403D09C
:105820000800F55007D06F00DBFFE9FF6F00DFFFD6
:10583000EAFFEF500009D8A420EF2CF022EF2CF063
:10584000D6EF2CF0FC0E6F008FFFF6FFFD0E6F0001
:105850008FFFF7FF000EF86E0F0EF76404D0010EF5
:10586000F56E0C0008D06F00DBFFE9FF6F00DFFF73
:10587000EAFF010EEF6EFC0EE350140F386EFD0EC2
:105880006F008CFF39F0000E39226000E3F0F6FF64
:105890006000E7F0F7FF000EF86E0F0EF76409D016
:1058A00009006F00D4FF38F009006F00D4FF39F011
:1058B0000CD06F00DBFFE9FF6F00DFFFEAFF6F0036
:1058C000B8FF38F06F00B8FF39F038503910D8B44D
:1058D0006CEF2CF06EEF2CF05DEF2DF0FC0EE35032
:1058E000160F386EFD0E6F008CFF39F0000E392256
:1058F0006000E3F0F6FF6000E7F0F7FF000EF86EDF
:105900000F0EF76409D009006F00D4FF38F00900CA
:105910006F00D4FF39F00CD06F00DBFFE9FF6F00A0
:10592000DFFFEAFF6F00B8FF38F06F00B8FF39F013
:105930006000E3F0E6FF6000E7F0E6FFFA0EE350F8
:10594000140F386EFB0E6F008CFF39F0000E3922F9
:105950006000E3F0F6FF6000E7F0F7FF000EF86E7E
:105960000F0EF76409D009006F00D4FF38F009006A
:105970006F00D4FF39F00CD06F00DBFFE9FF6F0040
:10598000DFFFEAFF6F00B8FF38F06F00B8FF39F0B3
:1059900002D8D4EF2CF00500FA6E3850FD6E395065
:1059A000FE6EFF6AFA5012005DEF2DF0FC0E6F00E4
:1059B0008FFFF6FFFD0E6F008FFFF7FF000EF86EF2
:1059C0000F0EF76404D0020EF56E0C0008D06F00C5
:1059D000DBFFE9FF6F00DFFFEAFF020EEF6EFC0E58
:1059E000E350010F386EFD0E6F008CFF39F0000E92
:1059F00039226000E3F0F6FF6000E7F0F7FF000EE9
:105A0000F86E0F0EF76409D009006F00D4FF38F06C
:105A100009006F00D4FF39F00CD06F00DBFFE9FF05
:105A20006F00DFFFEAFF6F00B8FF38F06F00B8FFCC
:105A300039F06000E3F0E6FF6000E7F0E6FFFA0E01
:105A40006F008FFFE6FF6F008FFFE6FFFEEC5FF059
:105A50005DEF2DF0FC0E6F008FFFF6FFFD0E6F0067
:105A60008FFFF7FF000EF86E0F0EF76403D00800EB
:105A7000F55007D06F00DBFFE9FF6F00DFFFEAFFA3
:105A8000EF50386E396A3950000AD8B44AEF2DF019
:105A90005DEF2DF03850000AD8B4B0EF29F0010ABC
:105AA000D8B4DCEF29F0030AD8B421EF2BF0010AB7
:105AB000D8B4EEEF2BF05DEF2DF0FF0E6F008CFFF2
:105AC00039F0FC0E6F008FFFF6FFFD0E6F008FFFA9
:105AD000F7FF000EF86E0F0EF76403D00800F550C4
:105AE00007D06F00DBFFE9FF6F00DFFFEAFFEF5039
:105AF0003918D8B47EEF2DF080EF2DF0A2EF2FF003
:105B0000FF0EE350386E396A3950000AD8B48BEF73
:105B10002DF06FEF2FF03850000AD8B46FEF2FF050
:105B2000010AD8B46FEF2FF0030AD8B46FEF2FF04B
:105B3000010AD8B46FEF2FF06FEF2FF0FC0EE35097
:105B4000080F386EFD0E6F008CFF39F0000E392201
:105B50006000E3F0F6FF6000E7F0F7FF000EF86E7C
:105B60000F0EF76409D009006F00D4FF38F0090068
:105B70006F00D4FF39F00CD06F00DBFFE9FF6F003E
:105B8000DFFFEAFF6F00B8FF38F06F00B8FF39F0B1
:105B900038503910D8B4CFEF2DF0D1EF2DF0A2EF5F
:105BA0002FF0FC0EE3500A0F386EFD0E6F008CFFD5
:105BB00039F0000E39226000E3F0F6FF6000E7F0F4
:105BC000F7FF000EF86E0F0EF76409D009006F00A2
:105BD000D4FF38F009006F00D4FF39F00CD06F000B
:105BE000DBFFE9FF6F00DFFFEAFF6F00B8FF38F06F
:105BF0006F00B8FF39F06000E3F0E6FF6000E7F007
:105C0000E6FFFA0EE350080F386EFB0E6F008CFFB4
:105C100039F0000E39226000E3F0F6FF6000E7F093
:105C2000F7FF000EF86E0F0EF76409D009006F0041
:105C3000D4FF38F009006F00D4FF39F00CD06F00AA
:105C4000DBFFE9FF6F00DFFFEAFF6F00B8FF38F00E
:105C50006F00B8FF39F002D837EF2EF00500FA6E6A
:105C60003850FD6E3950FE6EFF6AFA501200A2EFF6
:105C70002FF0FC0EE3500C0F386EFD0E6F008CFF02
:105C800039F0000E39226000E3F0F6FF6000E7F023
:105C9000F7FF000EF86E0F0EF76409D009006F00D1
:105CA000D4FF38F009006F00D4FF39F00CD06F003A
:105CB000DBFFE9FF6F00DFFFEAFF6F00B8FF38F09E
:105CC0006F00B8FF39F038503910D8B46AEF2EF0B1
:105CD0006CEF2EF0A2EF2FF0FC0EE3500E0F386E9B
:105CE000FD0E6F008CFF39F0000E39226000E3F0EA
:105CF000F6FF6000E7F0F7FF000EF86E0F0EF76496
:105D000009D009006F00D4FF38F009006F00D4FFFC
:105D100039F00CD06F00DBFFE9FF6F00DFFFEAFF17
:105D20006F00B8FF38F06F00B8FF39F06000E3F0A3
:105D3000E6FF6000E7F0E6FFFA0EE3500C0F386E66
:105D4000FB0E6F008CFF39F0000E39226000E3F08B
:105D5000F6FF6000E7F0F7FF000EF86E0F0EF76435
:105D600009D009006F00D4FF38F009006F00D4FF9C
:105D700039F00CD06F00DBFFE9FF6F00DFFFEAFFB7
:105D80006F00B8FF38F06F00B8FF39F002D8D2EFDB
:105D90002EF00500FA6E3850FD6E3950FE6EFF6A27
:105DA000FA501200A2EF2FF0FC0EE350100F386EE5
:105DB000FD0E6F008CFF39F0000E39226000E3F019
:105DC000F6FF6000E7F0F7FF000EF86E0F0EF764C5
:105DD00009D009006F00D4FF38F009006F00D4FF2C
:105DE00039F00CD06F00DBFFE9FF6F00DFFFEAFF47
:105DF0006F00B8FF38F06F00B8FF39F03850391035
:105E0000D8B405EF2FF007EF2FF0A2EF2FF0FC0E24
:105E1000E350120F386EFD0E6F008CFF39F0000E4C
:105E200039226000E3F0F6FF6000E7F0F7FF000EB4
:105E3000F86E0F0EF76409D009006F00D4FF38F038
:105E400009006F00D4FF39F00CD06F00DBFFE9FFD1
:105E50006F00DFFFEAFF6F00B8FF38F06F00B8FF98
:105E600039F06000E3F0E6FF6000E7F0E6FFFA0ECD
:105E7000E350100F386EFB0E6F008CFF39F0000EF0
:105E800039226000E3F0F6FF6000E7F0F7FF000E54
:105E9000F86E0F0EF76409D009006F00D4FF38F0D8
:105EA00009006F00D4FF39F00CD06F00DBFFE9FF71
:105EB0006F00DFFFEAFF6F00B8FF38F06F00B8FF38
:105EC00039F002D86DEF2FF00500FA6E3850FD6EF4
:105ED0003950FE6EFF6AFA501200A2EF2FF0FC0E4E
:105EE0006F008FFFF6FFFD0E6F008FFFF7FF000EB4
:105EF000F86E0F0EF76403D00800F55007D06F005E
:105F0000DBFFE9FF6F00DFFFEAFFEF50386E396A11
:105F10003950000AD8B48FEF2FF0A2EF2FF038508D
:105F2000000AD8B4A2EF2FF0010AD8B49EEF2DF0EA
:105F3000030AD8B439EF2EF0010AD8B4D4EF2EF00A
:105F4000A2EF2FF0FA0EE126FF0EE2221200E65237
:105F5000E652E652FB0E6F008FFFE6FF6F008FFFE9
:105F6000E6FF25EC63F0FE0E6000BFF0E3FFFD0EE0
:105F70006000BBF0E3FFFD0E6F008FFFF6FFFE0E2B
:105F80006F008FFFF7FF000EF86E0F0EF76403D05F
:105F90000800F55007D06F00DBFFE9FF6F00DFFF5F
:105FA000EAFFEF50396EFF0E6000E7F0E3FFFB0EF3
:105FB0006F008FFFE6FF6F008FFFE6FFE5EC63F0F9
:105FC000FB0E6F008FFFE6FF6F008FFFE6FF87EC91
:105FD00062F0F80EE126FF0EE22270EF31F0FB0EC8
:105FE0006F008FFFD9FFFC0E6F008FFFDAFFDF50CD
:105FF000640AD8A4FEEF2FF000EF30F0A3EF31F0E9
:10600000FD0E6F008FFFF6FFFE0E6F008FFFF7FF94
:10601000000EF86E0F0EF76404D0650EF56E0C00DE
:1060200008D06F00DBFFE9FF6F00DFFFEAFF650EBE
:10603000EF6EFD0EE350010F386EFE0E6F008CFF09
:1060400039F0000E39226000E3F0E6FF6000E7F06F
:10605000E6FF63EC5FF0A3EF31F0FB0E6F008FFF04
:10606000D9FFFC0E6F008FFFDAFFDF50650AD8A45E
:106070003CEF30F03EEF30F057EF30F0FD0E6F00A8
:106080008FFFF6FFFE0E6F008FFFF7FF000EF86E1A
:106090000F0EF76404D0660EF56E0C0008D06F008A
:1060A000DBFFE9FF6F00DFFFEAFF660EEF6E1850BF
:1060B000E66EFC0EE350010F386EFD0E6F008CFF94
:1060C00039F0000E39226000E3F0E6FF6000E7F0EF
:1060D000E6FF54EC60F0000EE66E000EE66E000E79
:1060E000E66E000EE66E000EE66E000EE66E000E28
:1060F000E66E000EE66E640EE66E000EE66EF30EC1
:10610000E350010F386EF40E6F008CFF39F0000E73
:1061100039226000E3F0E6FF6000E7F0E6FF93EC71
:106120005DF0000EE66E000EE66E000EE66E000EEE
:10613000E66E000EE66E000EE66E000EE66E000ED7
:10614000E66EC80EE66E000EE66EF30EE350010F2B
:10615000386EF40E6F008CFF39F0000E39226000AB
:10616000E3F0E6FF6000E7F0E6FF59EC5DF0A3EF37
:1061700031F0FB0E6F008FFFD9FFFC0E6F008FFF19
:10618000DAFFDF50660AD8A4C8EF30F0CAEF30F06B
:10619000E3EF30F0FD0E6F008FFFF6FFFE0E6F0095
:1061A0008FFFF7FF000EF86E0F0EF76404D0670E36
:1061B000F56E0C0008D06F00DBFFE9FF6F00DFFF1A
:1061C000EAFF670EEF6EFB0E6F008FFFD9FFFC0E2C
:1061D0006F008FFFDAFFDF50690AD8A4F2EF30F0CA
:1061E000F4EF30F02BEF31F0C90EE66E000EE66EE4
:1061F00090EC58F01750D8A400EF31F002EF31F0D6
:1062000004EF31F0010E176E000EE66E000EE66E22
:10621000000EE66E000EE66E000EE66E000EE66EF6
:10622000000EE66E000EE66E1750050D6F00CCFFF7
:1062300038F06F00D0FF39F06000E3F0E6FF600057
:10624000E7F0E6FFF30E6F008FFFE6FF6F008FFFB2
:10625000E6FF37EC5CF0FB0E6F008FFFD9FFFC0E02
:106260006F008FFFDAFFDF50680AD8A43AEF31F0F1
:106270003CEF31F0A3EF31F0D40EE66E000EE66E87
:106280006DEC59F0A3EF31F0FB0E6F008FFFD9FFDB
:10629000FC0E6F008FFFDAFFDF50670AD8A453EFC0
:1062A00031F055EF31F0A3EF31F0FD0E6F008FFFAD
:1062B000F6FFFE0E6F008FFFF7FF000EF86E0F0E59
:1062C000F76404D0650EF56E0C0008D06F00DBFF9C
:1062D000E9FF6F00DFFFEAFF650EEF6EA3EF31F01D
:1062E000FD0E6F008FFFF6FFFE0E6F008FFFF7FFB2
:1062F000000EF86E0F0EF76403D00800F55007D0BB
:106300006F00DBFFE9FF6F00DFFFEAFFEF50386E41
:10631000396A3950000AD8B490EF31F0A3EF31F068
:106320003850640AD8B4EFEF2FF0010AD8B42DEF3B
:1063300030F0030AD8B4B9EF30F0010AD8B444EF12
:1063400031F0A3EF31F0FF0E6F008CFF39F0FD0E3E
:106350006F008FFFF6FFFE0E6F008FFFF7FF000E3E
:10636000F86E0F0EF76403D00800F55007D06F00E9
:10637000DBFFE9FF6F00DFFFEAFFEF503918D8B409
:10638000C4EF31F0C6EF31F019EF34F0FF0EE350F7
:10639000386E396A3950000AD8B4D1EF31F0E6EFDF
:1063A00033F03850640AD8B4E6EF33F0010AD8B4B9
:1063B000E6EF33F0030AD8B4E6EF33F0010AD8B4BD
:1063C000E6EF33F0E6EF33F0FD0EE350380F386EB2
:1063D000FE0E6F008CFF39F0000E39226000E3F0F2
:1063E000F6FF6000E7F0F7FF000EF86E0F0EF7649F
:1063F00009D009006F00D4FF38F009006F00D4FF06
:1064000039F00CD06F00DBFFE9FF6F00DFFFEAFF20
:106410006F00B8FF38F06F00B8FF39F0385039100E
:10642000D8B415EF32F017EF32F019EF34F0FD0E5B
:10643000E3503A0F386EFE0E6F008CFF39F0000EFD
:1064400039226000E3F0F6FF6000E7F0F7FF000E8E
:10645000F86E0F0EF76409D009006F00D4FF38F012
:1064600009006F00D4FF39F00CD06F00DBFFE9FFAB
:106470006F00DFFFEAFF6F00B8FF38F06F00B8FF72
:1064800039F06000E3F0E6FF6000E7F0E6FFFB0EA6
:10649000E350380F386EFC0E6F008CFF39F0000EA1
:1064A00039226000E3F0F6FF6000E7F0F7FF000E2E
:1064B000F86E0F0EF76409D009006F00D4FF38F0B2
:1064C00009006F00D4FF39F00CD06F00DBFFE9FF4B
:1064D0006F00DFFFEAFF6F00B8FF38F06F00B8FF12
:1064E00039F002D87DEF32F00500FA6E3850FD6EBB
:1064F0003950FE6EFF6AFA50120019EF34F017504F
:10650000D8A485EF32F087EF32F089EF32F0010E38
:10651000176E000EE66E000EE66E000EE66E000EC2
:10652000E66E000EE66E000EE66E000EE66E000EE3
:10653000E66E1750050D6F00CCFF38F06F00D0FFEE
:1065400039F06000E3F0E6FF6000E7F0E6FFF30EED
:106550006F008FFFE6FF6F008FFFE6FF37EC5CF008
:10656000FD0EE3503C0F386EFE0E6F008CFF39F0CD
:10657000000E39226000E3F0F6FF6000E7F0F7FF5D
:10658000000EF86E0F0EF76409D009006F00D4FFFB
:1065900038F009006F00D4FF39F00CD06F00DBFF3A
:1065A000E9FF6F00DFFFEAFF6F00B8FF38F06F0010
:1065B000B8FF39F038503910D8B4E1EF32F0E3EFDA
:1065C00032F019EF34F0FD0EE3503E0F386EFE0E40
:1065D0006F008CFF39F0000E39226000E3F0F6FF07
:1065E0006000E7F0F7FF000EF86E0F0EF76409D0B9
:1065F00009006F00D4FF38F009006F00D4FF39F0B4
:106600000CD06F00DBFFE9FF6F00DFFFEAFF6F00D8
:10661000B8FF38F06F00B8FF39F06000E3F0E6FF34
:106620006000E7F0E6FFFB0EE3503C0F386EFC0E17
:106630006F008CFF39F0000E39226000E3F0F6FFA6
:106640006000E7F0F7FF000EF86E0F0EF76409D058
:1066500009006F00D4FF38F009006F00D4FF39F053
:106660000CD06F00DBFFE9FF6F00DFFFEAFF6F0078
:10667000B8FF38F06F00B8FF39F002D849EF33F0B7
:106680000500FA6E3850FD6E3950FE6EFF6AFA5002
:10669000120019EF34F0FD0EE350400F386EFE0E7D
:1066A0006F008CFF39F0000E39226000E3F0F6FF36
:1066B0006000E7F0F7FF000EF86E0F0EF76409D0E8
:1066C00009006F00D4FF38F009006F00D4FF39F0E3
:1066D0000CD06F00DBFFE9FF6F00DFFFEAFF6F0008
:1066E000B8FF38F06F00B8FF39F038503910D8B41F
:1066F0007CEF33F07EEF33F019EF34F0FD0EE35012
:10670000420F386EFE0E6F008CFF39F0000E3922FA
:106710006000E3F0F6FF6000E7F0F7FF000EF86EB0
:106720000F0EF76409D009006F00D4FF38F009009C
:106730006F00D4FF39F00CD06F00DBFFE9FF6F0072
:10674000DFFFEAFF6F00B8FF38F06F00B8FF39F0E5
:106750006000E3F0E6FF6000E7F0E6FFFB0EE350C9
:10676000400F386EFC0E6F008CFF39F0000E39229E
:106770006000E3F0F6FF6000E7F0F7FF000EF86E50
:106780000F0EF76409D009006F00D4FF38F009003C
:106790006F00D4FF39F00CD06F00DBFFE9FF6F0012
:1067A000DFFFEAFF6F00B8FF38F06F00B8FF39F085
:1067B00002D8E4EF33F00500FA6E3850FD6E395020
:1067C000FE6EFF6AFA50120019EF34F0FD0E6F00F2
:1067D0008FFFF6FFFE0E6F008FFFF7FF000EF86EC3
:1067E0000F0EF76403D00800F55007D06F00DBFFF1
:1067F000E9FF6F00DFFFEAFFEF50386E396A39506A
:10680000000AD8B406EF34F019EF34F03850640AB7
:10681000D8B419EF34F0010AD8B4E4EF31F0030A28
:10682000D8B47FEF32F0010AD8B44BEF33F019EF50
:1068300034F0FB0EE126FF0EE2221200E652E65291
:10684000E652FB0E6F008FFFE6FF6F008FFFE6FF43
:1068500025EC63F0FE0E6000BFF0E3FFFD0E60006C
:10686000BBF0E3FFFD0E6F008FFFF6FFFE0E6F0023
:106870008FFFF7FF000EF86E0F0EF76403D00800CD
:10688000F55007D06F00DBFFE9FF6F00DFFFEAFF85
:10689000EF50396EFF0E6000E7F0E3FFFB0E6F0074
:1068A0008FFFE6FF6F008FFFE6FFE5EC63F0FB0E66
:1068B0006F008FFFE6FF6F008FFFE6FF87EC62F04F
:1068C000F80EE126FF0EE2223FEF35F0FB0E6F00DF
:1068D0008FFFD9FFFC0E6F008FFFDAFFDF506E0ACB
:1068E000D8A475EF34F077EF34F072EF35F0FD0E89
:1068F0006F008FFFF6FFFE0E6F008FFFF7FF000E99
:10690000F86E0F0EF76404D06F0EF56E0C0008D011
:106910006F00DBFFE9FF6F00DFFFEAFF6F0EEF6E36
:10692000FD0EE350010F386EFE0E6F008CFF39F044
:10693000000E39226000E3F0E6FF6000E7F0E6FFBA
:1069400063EC5FF072EF35F0FB0E6F008FFFD9FF45
:10695000FC0E6F008FFFDAFFDF506F0AD8A4B3EF91
:1069600034F0B5EF34F072EF35F0FD0E6F008FFFAD
:10697000F6FFFE0E6F008FFFF7FF000EF86E0F0E92
:10698000F76404D0700EF56E0C0008D06F00DBFFCA
:10699000E9FF6F00DFFFEAFF700EEF6E72EF35F078
:1069A000FB0E6F008FFFD9FFFC0E6F008FFFDAFF29
:1069B000DF50700AD8A4DFEF34F0E1EF34F0FAEFE3
:1069C00034F0FD0E6F008FFFF6FFFE0E6F008FFF9D
:1069D000F7FF000EF86E0F0EF76404D0710EF56E1F
:1069E0000C0008D06F00DBFFE9FF6F00DFFFEAFF5C
:1069F000710EEF6EFB0E6F008FFFD9FFFC0E6F0064
:106A00008FFFDAFFDF50720AD8A409EF35F00BEFE1
:106A100035F072EF35F0CF0EE66E000EE66E67ECE5
:106A200054F072EF35F0FB0E6F008FFFD9FFFC0EB4
:106A30006F008FFFDAFFDF50710AD8A422EF35F024
:106A400024EF35F072EF35F0FD0E6F008FFFF6FF8B
:106A5000FE0E6F008FFFF7FF000EF86E0F0EF7644B
:106A600004D06F0EF56E0C0008D06F00DBFFE9FF5D
:106A70006F00DFFFEAFF6F0EEF6E72EF35F0FD0E75
:106A80006F008FFFF6FFFE0E6F008FFFF7FF000E07
:106A9000F86E0F0EF76403D00800F55007D06F00B2
:106AA000DBFFE9FF6F00DFFFEAFFEF50386E396A66
:106AB0003950000AD8B45FEF35F072EF35F0385036
:106AC0006E0AD8B466EF34F0010AD8B4A4EF34F0FB
:106AD0001F0AD8B4D0EF34F0010AD8B413EF35F060
:106AE00072EF35F0FF0E6F008CFF39F0FD0E6F0076
:106AF0008FFFF6FFFE0E6F008FFFF7FF000EF86EA0
:106B00000F0EF76403D00800F55007D06F00DBFFCD
:106B1000E9FF6F00DFFFEAFFEF503918D8B493EFB9
:106B200035F095EF35F0F1EF37F0FF0EE350386EAA
:106B3000396A3950000AD8B4A0EF35F0BEEF37F00B
:106B400038506E0AD8B4BEEF37F0010AD8B4BEEFA1
:106B500037F01F0AD8B4BEEF37F0010AD8B4BEEF41
:106B600037F0BEEF37F0FD0EE350380F386EFE0EF3
:106B70006F008CFF39F0000E39226000E3F0F6FF61
:106B80006000E7F0F7FF000EF86E0F0EF76409D013
:106B900009006F00D4FF38F009006F00D4FF39F00E
:106BA0000CD06F00DBFFE9FF6F00DFFFEAFF6F0033
:106BB000B8FF38F06F00B8FF39F038503910D8B44A
:106BC000E4EF35F0E6EF35F04CEF36F0FD0EE35034
:106BD0003A0F386EFE0E6F008CFF39F0000E39222E
:106BE0006000E3F0F6FF6000E7F0F7FF000EF86EDC
:106BF0000F0EF76409D009006F00D4FF38F00900C8
:106C00006F00D4FF39F00CD06F00DBFFE9FF6F009D
:106C1000DFFFEAFF6F00B8FF38F06F00B8FF39F010
:106C20006000E3F0E6FF6000E7F0E6FFFB0EE350F4
:106C3000380F386EFC0E6F008CFF39F0000E3922D1
:106C40006000E3F0F6FF6000E7F0F7FF000EF86E7B
:106C50000F0EF76409D009006F00D4FF38F0090067
:106C60006F00D4FF39F00CD06F00DBFFE9FF6F003D
:106C7000DFFFEAFF6F00B8FF38F06F00B8FF39F0B0
:106C800002D84CEF36F00500FA6E3850FD6E3950E0
:106C9000FE6EFF6AFA5012001950E66EFC0EE350C9
:106CA000010F386EFD0E6F008CFF39F0000E392297
:106CB0006000E3F0E6FF6000E7F0E6FF54EC60F010
:106CC000000EE66E000EE66E000EE66E000EE66E3C
:106CD000000EE66E000EE66E000EE66E000EE66E2C
:106CE000F40EE66E010EE66EF30EE350010F386E01
:106CF000F40E6F008CFF39F0000E39226000E3F0D3
:106D0000E6FF6000E7F0E6FF93EC5DF0F1EF37F0AF
:106D1000FD0EE3503C0F386EFE0E6F008CFF39F015
:106D2000000E39226000E3F0F6FF6000E7F0F7FFA5
:106D3000000EF86E0F0EF76409D009006F00D4FF43
:106D400038F009006F00D4FF39F00CD06F00DBFF82
:106D5000E9FF6F00DFFFEAFF6F00B8FF38F06F0058
:106D6000B8FF39F038503910D8B4B9EF36F0BBEF6E
:106D700036F0F1EF37F0FD0EE3503E0F386EFE0EA9
:106D80006F008CFF39F0000E39226000E3F0F6FF4F
:106D90006000E7F0F7FF000EF86E0F0EF76409D001
:106DA00009006F00D4FF38F009006F00D4FF39F0FC
:106DB0000CD06F00DBFFE9FF6F00DFFFEAFF6F0021
:106DC000B8FF38F06F00B8FF39F06000E3F0E6FF7D
:106DD0006000E7F0E6FFFB0EE3503C0F386EFC0E60
:106DE0006F008CFF39F0000E39226000E3F0F6FFEF
:106DF0006000E7F0F7FF000EF86E0F0EF76409D0A1
:106E000009006F00D4FF38F009006F00D4FF39F09B
:106E10000CD06F00DBFFE9FF6F00DFFFEAFF6F00C0
:106E2000B8FF38F06F00B8FF39F002D821EF37F023
:106E30000500FA6E3850FD6E3950FE6EFF6AFA504A
:106E40001200F1EF37F0FD0EE350400F386EFE0EEA
:106E50006F008CFF39F0000E39226000E3F0F6FF7E
:106E60006000E7F0F7FF000EF86E0F0EF76409D030
:106E700009006F00D4FF38F009006F00D4FF39F02B
:106E80000CD06F00DBFFE9FF6F00DFFFEAFF6F0050
:106E9000B8FF38F06F00B8FF39F038503910D8B467
:106EA00054EF37F056EF37F0F1EF37F0FD0EE350C7
:106EB000420F386EFE0E6F008CFF39F0000E392243
:106EC0006000E3F0F6FF6000E7F0F7FF000EF86EF9
:106ED0000F0EF76409D009006F00D4FF38F00900E5
:106EE0006F00D4FF39F00CD06F00DBFFE9FF6F00BB
:106EF000DFFFEAFF6F00B8FF38F06F00B8FF39F02E
:106F00006000E3F0E6FF6000E7F0E6FFFB0EE35011
:106F1000400F386EFC0E6F008CFF39F0000E3922E6
:106F20006000E3F0F6FF6000E7F0F7FF000EF86E98
:106F30000F0EF76409D009006F00D4FF38F0090084
:106F40006F00D4FF39F00CD06F00DBFFE9FF6F005A
:106F5000DFFFEAFF6F00B8FF38F06F00B8FF39F0CD
:106F600002D8BCEF37F00500FA6E3850FD6E39508C
:106F7000FE6EFF6AFA501200F1EF37F0FD0E6F005F
:106F80008FFFF6FFFE0E6F008FFFF7FF000EF86E0B
:106F90000F0EF76403D00800F55007D06F00DBFF39
:106FA000E9FF6F00DFFFEAFFEF50386E396A3950B2
:106FB000000AD8B4DEEF37F0F1EF37F038506E0A40
:106FC000D8B4F1EF37F0010AD8B4B3EF35F01F0AA7
:106FD000D8B488EF36F0010AD8B423EF37F0F1EFD8
:106FE00037F0FB0EE126FF0EE2221200E652E652D7
:106FF000E652E652FF0EE36AFE0EE36AFD0EE36A16
:10700000FC0EE36A3701E0B708EF38F00AEF38F01A
:107010001EEF39F0FC0EE1242E6EFF0EE2202F6EE3
:107020006000BBF0E6FF6000BFF0E6FFFB0EE1246E
:107030002E6EFF0EE2202F6E6000BBF0E6FF6000B8
:10704000BFF0E6FFFA0EE1242E6EFF0EE2202F6E57
:107050006000BBF0E6FF6000BFF0E6FFF90EE12440
:107060002E6EFF0EE2202F6E6000BBF0E6FF600088
:10707000BFF0E6FFF20E6F008FFFD9FFF30E6F0037
:107080008FFFDAFFDF50E66EF10E6F008CFF38F0F5
:10709000F20E6F008CFF39F0010E3824D96E000E0D
:1070A0003920DA6E6F007BFFE6FF6F007BFFE6FFA3
:1070B0006F007BFFE6FF6F007BFFE6FF8AEC47F087
:1070C000FF0E6F008FFFE3F7FE0E6F008FFFE4F7F8
:1070D000FD0E6F008FFFE1F7FC0E6F008FFFE2F7F0
:1070E000FA0E6F008CFF38F0FB0E6F008CFF39F04A
:1070F000050E3824D96E000E3920DA6EDF50396E55
:10710000FA0E6F008CFF36F0FB0E6F008CFF37F02D
:107110000E0E3624D96E000E3720DA6EDF50386E30
:10712000060E2E6ED89038362E2E92EF38F038504C
:1071300039103701E56FFA0E6F008CFF38F0FB0E47
:107140006F008CFF39F0060E3824D96E000E3920FE
:10715000DA6EDF50E66FFA0E6F008CFF38F0FB0E30
:107160006F008CFF39F0070E3824D96E000E3920DD
:10717000DA6EDF50E76FFA0E6F008CFF38F0FB0E0F
:107180006F008CFF39F0080E3824D96E000E3920BC
:10719000DA6EDF50E86FFA0E6F008CFF38F0FB0EEE
:1071A0006F008CFF39F0090E3824D96E000E39209B
:1071B000DA6EDF50E96FFA0E6F008CFF38F0FB0ECD
:1071C0006F008CFF39F00A0E3824D96E000E39207A
:1071D000DA6EDF50EA6FFA0E6F008CFF38F0FB0EAC
:1071E0006F008CFF39F00B0E3824D96E000E392059
:1071F000DA6EDF50EB6FFA0E6F008CFF38F0FB0E8B
:107200006F008CFF39F00C0E3824D96E000E392037
:10721000DA6EDF50EC6FFA0E6F008CFF38F0FB0E69
:107220006F008CFF39F00D0E3824D96E000E392016
:10723000DA6EDF50ED6FE08754EF3BF0D0B723EF0D
:1072400039F025EF39F039EF3AF0FC0EE1242E6EDB
:10725000FF0EE2202F6E6000BBF0E6FF6000BFF083
:10726000E6FFFB0EE1242E6EFF0EE2202F6E600083
:10727000BBF0E6FF6000BFF0E6FFFA0EE1242E6EE1
:10728000FF0EE2202F6E6000BBF0E6FF6000BFF053
:10729000E6FFF90EE1242E6EFF0EE2202F6E600055
:1072A000BBF0E6FF6000BFF0E6FFF20E6F008FFF5D
:1072B000D9FFF30E6F008FFFDAFFDF50E66EF10E9D
:1072C0006F008CFF38F0F20E6F008CFF39F0010E6A
:1072D0003824D96E000E3920DA6E6F007BFFE6FF8E
:1072E0006F007BFFE6FF6F007BFFE6FF6F007BFF19
:1072F000E6FF8AEC47F0FF0E6F008FFFD3F7FE0E1C
:107300006F008FFFD4F7FD0E6F008FFFD1F7FC0EDB
:107310006F008FFFD2F7FA0E6F008CFF38F0FB0E74
:107320006F008CFF39F0050E3824D96E000E39201D
:10733000DA6EDF50396EFA0E6F008CFF36F0FB0EFE
:107340006F008CFF37F00E0E3624D96E000E3720FA
:10735000DA6EDF50386E060E2E6ED89038362E2E2E
:10736000ADEF39F0385039103701D56FFA0E6F0094
:107370008CFF38F0FB0E6F008CFF39F0060E3824BE
:10738000D96E000E3920DA6EDF50D66FFA0E6F001C
:107390008CFF38F0FB0E6F008CFF39F0070E38249D
:1073A000D96E000E3920DA6EDF50D76FFA0E6F00FB
:1073B0008CFF38F0FB0E6F008CFF39F0080E38247C
:1073C000D96E000E3920DA6EDF50D86FFA0E6F00DA
:1073D0008CFF38F0FB0E6F008CFF39F0090E38245B
:1073E000D96E000E3920DA6EDF50D96FFA0E6F00B9
:1073F0008CFF38F0FB0E6F008CFF39F00A0E38243A
:10740000D96E000E3920DA6EDF50DA6FFA0E6F0097
:107410008CFF38F0FB0E6F008CFF39F00B0E382418
:10742000D96E000E3920DA6EDF50DB6FFA0E6F0076
:107430008CFF38F0FB0E6F008CFF39F00C0E3824F7
:10744000D96E000E3920DA6EDF50DC6FFA0E6F0055
:107450008CFF38F0FB0E6F008CFF39F00D0E3824D6
:10746000D96E000E3920DA6EDF50DD6FD0871CEF49
:1074700039F0C0B73EEF3AF040EF3AF054EF3BF04E
:10748000FC0EE1242E6EFF0EE2202F6E6000BBF09A
:10749000E6FF6000BFF0E6FFFB0EE1242E6EFF0E5C
:1074A000E2202F6E6000BBF0E6FF6000BFF0E6FF59
:1074B000FA0EE1242E6EFF0EE2202F6E6000BBF06C
:1074C000E6FF6000BFF0E6FFF90EE1242E6EFF0E2E
:1074D000E2202F6E6000BBF0E6FF6000BFF0E6FF29
:1074E000F20E6F008FFFD9FFF30E6F008FFFDAFFF0
:1074F000DF50E66EF10E6F008CFF38F0F20E6F0079
:107500008CFF39F0010E3824D96E000E3920DA6E66
:107510006F007BFFE6FF6F007BFFE6FF6F007BFFE6
:10752000E6FF6F007BFFE6FF8AEC47F0FF0E6F007F
:107530008FFFC3F7FE0E6F008FFFC4F7FD0E6F00C5
:107540008FFFC1F7FC0E6F008FFFC2F7FA0E6F00BE
:107550008CFF38F0FB0E6F008CFF39F0050E3824DD
:10756000D96E000E3920DA6EDF50396EFA0E6F00D8
:107570008CFF36F0FB0E6F008CFF37F00E0E3624BA
:10758000D96E000E3720DA6EDF50386E060E2E6E82
:10759000D89038362E2EC8EF3AF0385039103701CF
:1075A000C56FFA0E6F008CFF38F0FB0E6F008CFF7A
:1075B00039F0060E3824D96E000E3920DA6EDF500D
:1075C000C66FFA0E6F008CFF38F0FB0E6F008CFF59
:1075D00039F0070E3824D96E000E3920DA6EDF50EC
:1075E000C76FFA0E6F008CFF38F0FB0E6F008CFF38
:1075F00039F0080E3824D96E000E3920DA6EDF50CB
:10760000C86FFA0E6F008CFF38F0FB0E6F008CFF16
:1076100039F0090E3824D96E000E3920DA6EDF50A9
:10762000C96FFA0E6F008CFF38F0FB0E6F008CFFF5
:1076300039F00A0E3824D96E000E3920DA6EDF5088
:10764000CA6FFA0E6F008CFF38F0FB0E6F008CFFD4
:1076500039F00B0E3824D96E000E3920DA6EDF5067
:10766000CB6FFA0E6F008CFF38F0FB0E6F008CFFB3
:1076700039F00C0E3824D96E000E3920DA6EDF5046
:10768000CC6FFA0E6F008CFF38F0FB0E6F008CFF92
:1076900039F00D0E3824D96E000E3920DA6EDF5025
:1076A000CD6FC0871CEF39F0FA0EE126FF0EE22203
:1076B0001200080EE126000EE2226000ACF03EF05F
:1076C0003F6A406A416A426A436A446A456AF80E00
:1076D0006000FBF0E3FFF90E6000FFF0E3FFFA0E3D
:1076E000600003F1E3FFFB0E600007F1E3FFFC0E17
:1076F00060000BF1E3FFFD0E60000FF1E3FFFE0EF3
:10770000600013F1E3FFFF0E600017F1E3FFF80ED6
:107710006F008CFF3EF0F90E6F008CFF3FF0FA0E09
:107720006F008CFF40F0FB0E6F008CFF41F0FC0EF1
:107730006F008CFF42F0FD0E6F008CFF43F0FE0ED9
:107740006F008CFF44F0FF0E6F008CFF45F0040EBD
:10775000D8903E363F364036413642364336443680
:107760004536E82EA8EF3BF0F70EE3503E10466E8C
:107770003F50476E4050486E4150496E42504A6EED
:1077800043504B6E44504C6E45504D6EF80E6000A9
:107790001BF1E3FFF90E60001FF1E3FFFA0E60003A
:1077A00023F1E3FFFB0E600027F1E3FFFC0E600016
:1077B0002BF1E3FFFD0E60002FF1E3FFFE0E6000F2
:1077C00033F1E3FFFF0E600037F1E3FFF80E6F00C7
:1077D0008CFF3EF0F90E6F008CFF3FF0FA0E6F0049
:1077E0008CFF40F0FB0E6F008CFF41F0FC0E6F0031
:1077F0008CFF42F0FD0E6F008CFF43F0FE0E6F0019
:107800008CFF44F0FF0E6F008CFF45F0040ED89003
:107810003E363F36403641364236433644364536AC
:10782000E82E07EF3CF0F60EE3503E10466E3F5058
:10783000476E4050486E4150496E42504A6E435028
:107840004B6E44504C6E45504D6EF80E60001BF16F
:10785000E3FFF90E60001FF1E3FFFA0E600023F171
:10786000E3FFFB0E600027F1E3FFFC0E60002BF14D
:10787000E3FFFD0E60002FF1E3FFFE0E600033F129
:10788000E3FFFF0E600037F1E3FFF20E6F008CFFA5
:1078900036F0F30E6F008CFF37F0F40E6F008CFFA4
:1078A00038F0F50E6F008CFF39F036503E6E3750D1
:1078B0003F6E3850406E3950416E426A436A446AA6
:1078C000456AF80E6F008CFF46F0F90E6F008CFFD2
:1078D00047F0FA0E6F008CFF48F0FB0E6F008CFF34
:1078E00049F0FC0E6F008CFF4AF0FD0E6F008CFF1C
:1078F0004BF0FE0E6F008CFF4CF0FF0E6F008CFF04
:107900004DF0200ED89046364736483649364A362E
:107910004B364C364D36E82E82EF3CF03E5046104A
:10792000366E3F504710376E40504810386E415009
:107930004910396E42504A103A6E43504B103B6E1C
:1079400044504C103C6E45504D103D6EF80E60009A
:10795000DBF0E3FFF90E6000DFF0E3FFFA0E6000FA
:10796000E3F0E3FFFB0E6000E7F0E3FFFC0E6000D6
:10797000EBF0E3FFFD0E6000EFF0E3FFFE0E6000B2
:10798000F3F0E3FFFF0E6000F7F0E3FFE150F80FC4
:10799000D96EE250DA6EFF0EDA226F007BFFE6FF4F
:1079A0006F007BFFE6FF6F007BFFE6FF6F007BFF52
:1079B000E6FF6F007BFFE6FF6F007BFFE6FF6F00D7
:1079C0007BFFE6FF6F007BFFE6FF000EE66E000E1A
:1079D000E66E0D0EE66E9E0EE66E350EE66E2A0E15
:1079E000E66E000EE66E69EC4EF0F20EE126FF0E3A
:1079F000E2221200E652000EE66EC1EC64F0FF0EC9
:107A00006000BBF0E3FFFF0E6F008CFF2EF0420E14
:107A10002E18D8B40EEF3DF010EF3DF0F6EF3DF02C
:107A2000016A0A0E026E070E036EB20E046E010E9C
:107A3000056E000E066E100E076E270E086E000E05
:107A4000096E000E0A6EF00E0B6E730E0C6E550E64
:107A50000D6E000E0E6E320E0F6E190E106E116A44
:107A6000050E126E010E136E190E146E640E156E55
:107A7000140E166E0A0E176EFA0E186E640E196E3C
:107A8000320E1A6E320E1B6E320E1C6E320E1D6ED0
:107A90000A0E1E6E0A0E1F6E0150E66E010EE66E95
:107AA000FFEC63F00250E66E020EE66EFFEC63F050
:107AB00060000FF0E6FF600013F0E6FF600017F0D3
:107AC000E6FF60001BF0E6FF030EE66EDBEC57F00E
:107AD00060001FF0E6FF600023F0E6FF600027F083
:107AE000E6FF60002BF0E6FF070EE66EDBEC57F0DA
:107AF00060002FF0E6FF600033F0E6FF600037F033
:107B0000E6FF60003BF0E6FF0B0EE66EDBEC57F0A5
:107B10000F50E66E0F0EE66EFFEC63F01050E66E4F
:107B2000100EE66EFFEC63F01150E66E110EE66E7D
:107B3000FFEC63F01250E66E120EE66EFFEC63F09F
:107B40001350E66E130EE66EFFEC63F01450E66E13
:107B5000140EE66EFFEC63F01550E66E150EE66E41
:107B6000FFEC63F01650E66E160EE66EFFEC63F067
:107B70001750E66E170EE66EFFEC63F01850E66ED7
:107B8000180EE66EFFEC63F01950E66E190EE66E05
:107B9000FFEC63F01A50E66E1A0EE66EFFEC63F02F
:107BA0001B50E66E1B0EE66EFFEC63F01C50E66E9B
:107BB0001C0EE66EFFEC63F01D50E66E1D0EE66EC9
:107BC000FFEC63F01F50E66E1F0EE66EFFEC63F0F5
:107BD0001E50E66E1E0EE66EFFEC63F0420EE66E81
:107BE000000EE66EFFEC63F098EF3EF0010EE66EDD
:107BF000C1EC64F02E50016E020EE66EC1EC64F032
:107C00002E50026E030EE66E3DEC58F06000B8F0A8
:107C100003F06000BCF004F06000C0F005F060000C
:107C2000C4F006F0070EE66E3DEC58F06000B8F0C8
:107C300007F06000BCF008F06000C0F009F06000E0
:107C4000C4F00AF00B0EE66E3DEC58F06000B8F0A0
:107C50000BF06000BCF00CF06000C0F00DF06000B4
:107C6000C4F00EF00F0EE66EC1EC64F02E500F6EF5
:107C7000100EE66EC1EC64F02E50106E110EE66E22
:107C8000C1EC64F02E50116E120EE66EC1EC64F081
:107C90002E50126E130EE66EC1EC64F02E50136E71
:107CA000140EE66EC1EC64F02E50146E150EE66EE6
:107CB000C1EC64F02E50156E160EE66EC1EC64F049
:107CC0002E50166E170EE66EC1EC64F02E50176E35
:107CD000180EE66EC1EC64F02E50186E190EE66EAA
:107CE000C1EC64F02E50196E1A0EE66EC1EC64F011
:107CF0002E501A6E1B0EE66EC1EC64F02E501B6EF9
:107D00001C0EE66EC1EC64F02E501C6E1D0EE66E6D
:107D1000C1EC64F02E501D6E1F0EE66EC1EC64F0D7
:107D20002E501F6E1E0EE66EC1EC64F02E501E6EBD
:107D3000E55212000001606B030E616F050E626F69
:107D4000070E636F0A0E646F0C0E656F0E0E666F82
:107D5000100E676F120E686F140E696F160E6A6F41
:107D6000180E6B6F190E6C6F1B0E6D6F1C0E6E6F05
:107D70001E0E6F6F1F0E706F210E716F220E726FCD
:107D8000240E736F250E746F260E756F270E766F97
:107D9000280E776F290E786F2A0E796F2B0E7A6F67
:107DA0002C0E7B6F2D0E7C6F2E0E7D6F2F0E7E6F37
:107DB0002F0E7F6F300E806F310E816F320E826F0B
:107DC000320E836F330E846F330E856F340E866FE1
:107DD000350E876F350E886F350E896F360E8A6FB8
:107DE000360E8B6F370E8C6F370E8D6F380E8E6F91
:107DF000380E8F6F380E906F390E916F390E926F6B
:107E00003A0E936F3A0E946F3A0E956F3B0E966F43
:107E10003B0E976F3B0E986F3C0E996F3C0E9A6F1E
:107E20003C0E9B6F3D0E9C6F3D0E9D6F3E0E9E6FF8
:107E30003E0E9F6F3E0EA06F3F0EA16F3F0EA26FD2
:107E4000400EA36F400EA46F410EA56F410EA66FAA
:107E5000420EA76F430EA86F430EA96F440EAA6F80
:107E6000450EAB6F450EAC6F460EAD6F470EAE6F55
:107E7000480EAF6F480EB06F490EB16F4A0EB26F29
:107E80004B0EB36F4C0EB46F4D0EB56F4E0EB66FFA
:107E9000500EB76F510EB86F520EB96F530EBA6FC6
:107EA000550EBB6F560EBC6F580EBD6F590EBE6F90
:107EB0005B0EBF6F5D0EC06F5E0EC16F600EC26F56
:107EC000620EC36F640EC46F0101006B016B026B25
:107ED000036B046B010E056F010E066F010E076F39
:107EE000020E086F020E096F030E0A6F030E0B6F6E
:107EF000040E0C6F050E0D6F050E0E6F060E0F6F44
:107F0000070E106F080E116F090E126F090E136F16
:107F10000A0E146F0B0E156F0C0E166F0D0E176FE9
:107F20000F0E186F100E196F110E1A6F120E1B6FB5
:107F3000130E1C6F140E1D6F160E1E6F170E1F6F83
:107F4000180E206F190E216F1B0E226F1C0E236F4F
:107F50001E0E246F1F0E256F200E266F220E276F18
:107F6000230E286F250E296F260E2A6F280E2B6FE1
:107F7000290E2C6F2B0E2D6F2C0E2E6F2E0E2F6FA9
:107F80002F0E306F310E316F320E326F330E336F72
:107F9000350E346F360E356F380E366F390E376F3B
:107FA0003B0E386F3C0E396F3E0E3A6F3F0E3B6F03
:107FB000410E3C6F420E3D6F440E3E6F450E3F6FCB
:107FC000460E406F480E416F490E426F4B0E436F95
:107FD0004C0E446F4D0E456F4E0E466F500E476F60
:107FE000510E486F520E496F530E4A6F540E4B6F2D
:107FF000550E4C6F570E4D6F580E4E6F590E4F6FFA
:108000005A0E506F5B0E516F5B0E526F5C0E536FCA
:108010005D0E546F5E0E556F5F0E566F5F0E576F9D
:10802000600E586F610E596F610E5A6F620E5B6F72
:10803000620E5C6F630E5D6F630E5E6F630E5F6F4B
:10804000640E606F640E616F640E626F640E636F26
:10805000640E646F1200170EE126000EE222E90E94
:10806000E1242E6EFF0EE2202F6E6000BBF0E6FFD3
:108070006000BFF0E6FFC5EC11F0EA0EE124D96E16
:10808000FF0EE220DA6E6F0078FF36F06F0078FFA7
:1080900037F06F0078FF38F06F0078FF39F0365016
:1080A0003E6E37503F6E3850406E3950416E426AD6
:1080B000436A446A456AF80E6000FBF0E3FFF90E7C
:1080C0006000FFF0E3FFFA0E600003F1E3FFFB0E38
:1080D000600007F1E3FFFC0E60000BF1E3FFFD0E13
:1080E00060000FF1E3FFFE0E600013F1E3FFFF0EEF
:1080F000600017F1E3FFE150F80FD96EE250DA6E3D
:10810000FF0EDA220C0ED890DE36DE36DE36DE3694
:10811000DE36DE36DE36DD36DD52DD52DD52DD5254
:10812000DD52DD52E82E83EF40F0E150F80FD96EBA
:10813000E250DA6EFF0EDA22F20EE124E96EFF0E53
:10814000E220EA6EEF50DE12000EDE12DE12DE12C8
:10815000DE12DE12DE12DE12E150F80FD96EE250AE
:10816000DA6EFF0EDA22080ED890DE36DE36DE3604
:10817000DE36DE36DE36DE36DD36DD52DD52DD520F
:10818000DD52DD52DD52E82EB4EF40F0E150F80F41
:10819000D96EE250DA6EFF0EDA22F10EE124E96EBA
:1081A000FF0EE220EA6EEF50DE12000EDE12DE124B
:1081B000DE12DE12DE12DE12DE12E150F80FD96E90
:1081C000E250DA6EFF0EDA22080ED890DE36DE3686
:1081D000DE36DE36DE36DE36DE36DD36DD52DD52CA
:1081E000DD52DD52DD52DD52E82EE5EF40F0E15088
:1081F000F80FD96EE250DA6EFF0EDA22F00EE124AB
:10820000E96EFF0EE220EA6EEF50DE12000EDE1283
:10821000DE12DE12DE12DE12DE12DE12E150F80F86
:10822000D96EE250DA6EFF0EDA22080ED890DE36F2
:10823000DE36DE36DE36DE36DE36DE36DD36DD5284
:10824000DD52DD52DD52DD52DD52E82E16EF41F0F7
:10825000E150F80FD96EE250DA6EFF0EDA22EF0E1F
:10826000E124E96EFF0EE220EA6EEF50DE12000E0E
:10827000DE12DE12DE12DE12DE12DE12DE12F70E69
:10828000E124D96EFF0EE220DA6EDF50D8B44BEF56
:1082900041F04DEF41F07EEF41F0E150F80FD96E23
:1082A000E250DA6EFF0EDA226F007BFFE6FF6F000E
:1082B0007BFFE6FF6F007BFFE6FF6F007BFFE6FFC3
:1082C0006F007BFFE6FF6F007BFFE6FF6F007BFF29
:1082D000E6FF6F007BFFE6FF000EE66E000EE66E27
:1082E0000C0EE66E9E0EE66E350EE66E2A0EE66EFD
:1082F000000EE66E69EC4EF0ADEF41F0E150F80F84
:10830000D96EE250DA6EFF0EDA226F007BFFE6FFD5
:108310006F007BFFE6FF6F007BFFE6FF6F007BFFD8
:10832000E6FF6F007BFFE6FF6F007BFFE6FF6F005D
:108330007BFFE6FF6F007BFFE6FF000EE66E000EA0
:10834000E66E0B0EE66E9E0EE66E350EE66E2A0E9D
:10835000E66E000EE66E69EC4EF0E90EE126FF0EC9
:10836000E2221200E652E652E652E652FB0EE350DB
:10837000366E000E36BEFF0E376E386E396EFC0E4E
:108380006000DBF0E3FFFD0E6000DFF0E3FFFE0EB8
:108390006000E3F0E3FFFF0E6000E7F0E3FF020E92
:1083A0000001D619D8A4D7EF41F0D9EF41F07DEF05
:1083B00042F0FF0EE3BEDFEF41F0E1EF41F009EFE5
:1083C00042F0FC0E6F008CFF38F0FD0E6F008CFF4A
:1083D00039F0600E3824D96E000E3920DA6EDF5085
:1083E000396E6000E4F032F0336A346A356AFC0EAC
:1083F0006000CBF0E3FFFD0E6000CFF0E3FFFE0E68
:108400006000D3F0E3FFFF0E6000D7F0E3FF7DEFE5
:1084100042F0FF0EE66EFF0EE66EFF0EE66EFF0EFA
:10842000E66EF80E6F008FFFE6FF6F008FFFE6FF2E
:108430006F008FFFE6FF6F008FFFE6FFF2EC53F057
:10844000FC0E6000BBF0E3FFFD0E6000BFF0E3FF39
:10845000FE0E6000C3F0E3FFFF0E6000C7F0E3FF15
:10846000FC0E6F008CFF38F0FD0E6F008CFF39F0B2
:10847000600E3824D96E000E3920DA6EDF50396E66
:108480006000E4F032F0336A346A356AFC0E600052
:10849000CBF0E3FFFD0E6000CFF0E3FFFE0E6000C7
:1084A000D3F0E3FFFF0E6000D7F0E3FFFF0EE66EB0
:1084B000FF0EE66EFF0EE66EFF0EE66EF80E6F0024
:1084C0008FFFE6FF6F008FFFE6FF6F008FFFE6FF75
:1084D0006F008FFFE6FFF2EC53F0FC0E6000BBF084
:1084E000E3FFFD0E6000BFF0E3FFFE0E6000C3F08F
:1084F000E3FFFF0E6000C7F0E3FF60001FF0E6FF40
:10850000600023F0E6FF600027F0E6FF60002BF03C
:10851000E6FFF80E6F008FFFE6FF6F008FFFE6FFAC
:108520006F008FFFE6FF6F008FFFE6FFF2EC53F066
:10853000FC0E6000BBF0E3FFFD0E6000BFF0E3FF48
:10854000FE0E6000C3F0E3FFFF0E6000C7F0E3FF24
:10855000E80EE66E030EE66E000EE66E000EE66EA8
:10856000F80E6F008FFFE6FF6F008FFFE6FF6F00D2
:108570008FFFE6FF6F008FFFE6FFA8EC48F0FC0ED0
:108580006000BBF0E3FFFD0E6000BFF0E3FFFE0EF6
:108590006000C3F0E3FFFF0E6000C7F0E3FF0001DF
:1085A000D351D8B4D6EF42F0D8EF42F026EF43F0E3
:1085B0007E0EE66E040EE66E000EE66E000EE66EB1
:1085C000F80E6F008FFFE6FF6F008FFFE6FF6F0072
:1085D0008FFFE6FF6F008FFFE6FFF2EC53F0FC0E1B
:1085E0006000BBF0E3FFFD0E6000BFF0E3FFFE0E96
:1085F0006000C3F0E3FFFF0E6000C7F0E3FFE80E8A
:10860000E66E030EE66E000EE66E000EE66EF80EE7
:108610006F008FFFE6FF6F008FFFE6FF6F008FFF99
:10862000E6FF6F008FFFE6FFA8EC48F0FC0E60004D
:10863000BBF0E3FFFD0E6000BFF0E3FFFE0E600045
:10864000C3F0E3FFFF0E6000C7F0E3FFFC0E6F0016
:108650008CFFC9F0FD0E6F008CFFCAF0FB0EE12607
:10866000FF0EE2221200080EE126000EE222600058
:10867000ACF03EF03F6A406A416A426A436A446A2B
:10868000456AF80E6000FBF0E3FFF90E6000FFF0B2
:10869000E3FFFA0E600003F1E3FFFB0E600007F159
:1086A000E3FFFC0E60000BF1E3FFFD0E60000FF135
:1086B000E3FFFE0E600013F1E3FFFF0E600017F111
:1086C000E3FFF80E6F008CFF3EF0F90E6F008CFF99
:1086D0003FF0FA0E6F008CFF40F0FB0E6F008CFF36
:1086E00041F0FC0E6F008CFF42F0FD0E6F008CFF1E
:1086F00043F0FE0E6F008CFF44F0FF0E6F008CFF06
:1087000045F0040ED8903E363F364036413642366C
:10871000433644364536E82E82EF43F0F70EE350F9
:108720003E10466E3F50476E4050486E4150496E75
:1087300042504A6E43504B6E44504C6E45504D6E05
:10874000F80E60001BF1E3FFF90E60001FF1E3FF7C
:10875000FA0E600023F1E3FFFB0E600027F1E3FF58
:10876000FC0E60002BF1E3FFFD0E60002FF1E3FF34
:10877000FE0E600033F1E3FFFF0E600037F1E3FF10
:10878000F80E6F008CFF3EF0F90E6F008CFF3FF08B
:10879000FA0E6F008CFF40F0FB0E6F008CFF41F073
:1087A000FC0E6F008CFF42F0FD0E6F008CFF43F05B
:1087B000FE0E6F008CFF44F0FF0E6F008CFF45F043
:1087C000040ED8903E363F36403641364236433668
:1087D00044364536E82EE1EF43F0F60EE3503E1006
:1087E000466E3F50476E4050486E4150496E425071
:1087F0004A6E43504B6E44504C6E45504D6EF80ED1
:1088000060001BF1E3FFF90E60001FF1E3FFFA0EB9
:10881000600023F1E3FFFB0E600027F1E3FFFC0E95
:1088200060002BF1E3FFFD0E60002FF1E3FFFE0E71
:10883000600033F1E3FFFF0E600037F1E3FFF80E55
:108840006F008CFF3EF0F90E6F008CFF3FF0FA0EC8
:108850006F008CFF40F0FB0E6F008CFF41F0FC0EB0
:108860006F008CFF42F0FD0E6F008CFF43F0FE0E98
:108870006F008CFF44F0FF0E6F008CFF45F0200E60
:10888000D8903E363F36403641364236433644363F
:108890004536E82E40EF44F0F50EE3503E10466EAC
:1088A0003F50476E4050486E4150496E42504A6EAC
:1088B00043504B6E44504C6E45504D6EF80E600068
:1088C0001BF1E3FFF90E60001FF1E3FFFA0E6000F9
:1088D00023F1E3FFFB0E600027F1E3FFFC0E6000D5
:1088E0002BF1E3FFFD0E60002FF1E3FFFE0E6000B1
:1088F00033F1E3FFFF0E600037F1E3FFE150F80FC3
:10890000D96EE250DA6EFF0EDA226F007BFFE6FFCF
:108910006F007BFFE6FF6F007BFFE6FF6F007BFFD2
:10892000E6FF6F007BFFE6FF6F007BFFE6FF6F0057
:108930007BFFE6FF6F007BFFE6FF000EE66E000E9A
:10894000E66E0F0EE66E9E0EE66E350EE66E2A0E93
:10895000E66E000EE66E69EC4EF0F50EE126FF0EB7
:10896000E2221200E652E652E652E652FB0EE350D5
:10897000366E000E36BEFF0E376E386E396EFC0E48
:108980006000DBF0E3FFFD0E6000DFF0E3FFFE0EB2
:108990006000E3F0E3FFFF0E6000E7F0E3FFFF0E8F
:1089A000E66EFF0EE66EFF0EE66EFF0EE66EF80E4A
:1089B0006F008FFFE6FF6F008FFFE6FF6F008FFFF6
:1089C000E6FF6F008FFFE6FFF2EC53F0FC0E600055
:1089D000BBF0E3FFFD0E6000BFF0E3FFFE0E6000A2
:1089E000C3F0E3FFFF0E6000C7F0E3FF020E0001DB
:1089F000D619D8A4FEEF44F000EF45F0A4EF45F0FF
:108A0000FF0EE3BE06EF45F008EF45F030EF45F00E
:108A1000FC0E6F008CFF38F0FD0E6F008CFF39F0FC
:108A2000000E3824D96E010E3920DA6EDF50396E0F
:108A30006000E4F032F0336A346A356AFC0E60009C
:108A4000CBF0E3FFFD0E6000CFF0E3FFFE0E600011
:108A5000D3F0E3FFFF0E6000D7F0E3FFA4EF45F093
:108A6000FF0EE66EFF0EE66EFF0EE66EFF0EE66E82
:108A7000F80E6F008FFFE6FF6F008FFFE6FF6F00BD
:108A80008FFFE6FF6F008FFFE6FFF2EC53F0FC0E66
:108A90006000BBF0E3FFFD0E6000BFF0E3FFFE0EE1
:108AA0006000C3F0E3FFFF0E6000C7F0E3FFFC0EC1
:108AB0006F008CFF38F0FD0E6F008CFF39F0000E58
:108AC0003824D96E010E3920DA6EDF50396E60001D
:108AD000E4F032F0336A346A356AFC0E6000CBF0A1
:108AE000E3FFFD0E6000CFF0E3FFFE0E6000D3F069
:108AF000E3FFFF0E6000D7F0E3FFFF0EE66EFF0E10
:108B0000E66EFF0EE66EFF0EE66EF80E6F008FFF4C
:108B1000E6FF6F008FFFE6FF6F008FFFE6FF6F003D
:108B20008FFFE6FFF2EC53F0FC0E6000BBF0E3FFBA
:108B3000FD0E6000BFF0E3FFFE0E6000C3F0E3FF38
:108B4000FF0E6000C7F0E3FF60002FF0E6FF60005B
:108B500033F0E6FF600037F0E6FF60003BF0E6FF31
:108B6000F80E6F008FFFE6FF6F008FFFE6FF6F00CC
:108B70008FFFE6FF6F008FFFE6FFF2EC53F0FC0E75
:108B80006000BBF0E3FFFD0E6000BFF0E3FFFE0EF0
:108B90006000C3F0E3FFFF0E6000C7F0E3FFE80EE4
:108BA000E66E030EE66E000EE66E000EE66EF80E42
:108BB0006F008FFFE6FF6F008FFFE6FF6F008FFFF4
:108BC000E6FF6F008FFFE6FFA8EC48F0FC0E6000A8
:108BD000BBF0E3FFFD0E6000BFF0E3FFFE0E6000A0
:108BE000C3F0E3FFFF0E6000C7F0E3FFE150FC0FAE
:108BF000D96EE250DA6EFF0EDA220001CB51DE268A
:108C0000CC51DE22CD51DE22CE51DE22E150FC0FCE
:108C1000D96EE250DA6EFF0EDA226F0078FFCFF0E5
:108C20006F0078FFD0F06F0078FFD1F06F0078FF11
:108C3000D2F0FB0EE126FF0EE2221200FE0E6F00C4
:108C40008FFFD9FFFF0E6F008FFFDAFF140EDF6E6C
:108C5000FE0E6F008CFF38F0FF0E6F008CFF39F0B6
:108C60001A0E3824D96E000E3920DA6EDF6AFE0E35
:108C70006F008CFF38F0FF0E6F008CFF39F01B0E79
:108C80003824D96E000E3920DA6EDF6AFE0E6F00CE
:108C90008CFF38F0FF0E6F008CFF39F01C0E38246B
:108CA000D96E000E3920DA6EDF6AFE0E6F008CFF7F
:108CB00038F0FF0E6F008CFF39F01D0E3824D96E8E
:108CC000000E3920DA6E010EDF6EFE0E6F008CFF93
:108CD00038F0FF0E6F008CFF39F01E0E3824D96E6D
:108CE000000E3920DA6E0A0EDF6EFE0E6F008CFF6A
:108CF00038F0FF0E6F008CFF39F01F0E3824D96E4C
:108D0000000E3920DA6EDE6ADD6AFE0E6F008CFF1F
:108D100038F0FF0E6F008CFF39F0230E3824D96E27
:108D2000000E3920DA6EDE6ADD6AFE0E6F008CFFFF
:108D300038F0FF0E6F008CFF39F0270E3824D96E03
:108D4000000E3920DA6EDE6ADD6AFE0E6F008CFFDF
:108D500038F0FF0E6F008CFF39F02B0E3824D96EDF
:108D6000000E3920DA6EDE6ADD6AFE0E6F008CFFBF
:108D700038F0FF0E6F008CFF39F02F0E3824D96EBB
:108D8000000E3920DA6EDE6ADD6AFE0E6F008CFF9F
:108D900038F0FF0E6F008CFF39F0330E3824D96E97
:108DA000000E3920DA6EDE6ADD6AFD0EE350E66EF3
:108DB000FD0EE350010F386EFE0E6F008CFF39F090
:108DC000000E39226000E3F0E6FF6000E7F0E6FF06
:108DD0009BEC63F0FE0EE350010F386EFF0E6F0048
:108DE0008CFF39F0000E39226000E3F0E6FF6000EE
:108DF000E7F0E6FF24EC64F0FE0EE350020F386E5D
:108E0000FF0E6F008CFF39F0000E39226000E3F096
:108E1000E6FF6000E7F0E6FF29EC51F0320EE66E67
:108E2000000EE66EFC0EE350020F386EFD0E6F0072
:108E30008CFF39F0000E39226000E3F0E6FF60009D
:108E4000E7F0E6FF47EC62F0320EE66E000EE66EEB
:108E5000FC0EE350020F386EFD0E6F008CFF39F0F0
:108E6000000E39226000E3F0E6FF6000E7F0E6FF65
:108E700067EC62F0FE0EE350010F386EFF0E6F00DC
:108E80008CFF39F0000E39226000E3F0E6FF60004D
:108E9000E7F0E6FFB60EE66EA90EE66EFA0EE350B8
:108EA000020F386EFB0E6F008CFF39F0000E392276
:108EB0006000E3F0E6FF6000E7F0E6FF4BEC5BF0FC
:108EC000FE0EE350010F386EFF0E6F008CFF39F07D
:108ED000000E39226000E3F0E6FF6000E7F0E6FFF5
:108EE0009E0EE66EAA0EE66EFA0EE350020F386E84
:108EF000FB0E6F008CFF39F0000E39226000E3F0AA
:108F0000E6FF6000E7F0E6FF86EC5BF0E552E55235
:108F1000E5521200E652FA0E6F008CFF2EF0020EA0
:108F20002E18D8A496EF47F098EF47F071EF48F06D
:108F3000F60E6F008FFFD9FFF70E6F008FFFDAFF7D
:108F4000FB0E6F008FFFDFFFFC0EE124D96EFF0EDA
:108F5000E220DA6E6F0078FF37F06F0078FF38F0AC
:108F60006F0078FF39F03750326E3850336E395019
:108F7000346E356AFB0E6000CBF0E3FFFC0E600040
:108F8000CFF0E3FFFD0E6000D3F0E3FFFE0E6000C4
:108F9000D7F0E3FFF80E6F008FFFD9FFF90E6F00D7
:108FA0008FFFDAFFFB0E6F008FFFDFFFFC0EE12467
:108FB000D96EFF0EE220DA6E6F0078FF37F06F0097
:108FC00078FF38F06F0078FF39F03750326E385044
:108FD000336E3950346E356AFB0E6000CBF0E3FF20
:108FE000FC0E6000CFF0E3FFFD0E6000D3F0E3FF66
:108FF000FE0E6000D7F0E3FFFB0E6F008CFF39F030
:10900000030E3916FF0E6000E7F0E3FFE150FB0F9F
:10901000D96EE250DA6EFF0EDA22030ED890DE36F9
:10902000DE36DE36DD36DD52DD52E82E0EEF48F05C
:10903000FB0E6F008CFF39F0E00E3916E150FF0F88
:10904000D96EE250DA6EFF0EDA223950DF26FF0EBB
:109050006F008CFF2EF0080E2E26FF0E6000BBF076
:10906000E3FFF20E6F008FFFD9FFF30E6F008FFF4B
:10907000DAFFFF0EE350EB0BDF6EFC0EE124D96E3E
:10908000FF0EE220DA6E6F0078FF37F06F0078FF96
:1090900038F06F0078FF39F03750326E3850336E49
:1090A0003950346E356AFB0E6000CBF0E3FFFC0EE6
:1090B0006000CFF0E3FFFD0E6000D3F0E3FFFE0E93
:1090C0006000D7F0E3FFF40E6F008FFFD9FFF50EBD
:1090D0006F008FFFDAFFFB0E6F008FFFDFFFA3EF44
:1090E00048F0F80E6F008FFFD9FFF90E6F008FFF69
:1090F000DAFFDF6AF60E6F008FFFD9FFF70E6F0001
:109100008FFFDAFFDF6AE150FB0FD96EE250DA6EB3
:10911000FF0EDA22050ED890DE36DE36DE36DD367C
:10912000DD52DD52E82E8BEF48F0F20E6F008FFF1C
:10913000D9FFF30E6F008FFFDAFFFB0E6F008FFF7A
:10914000DFFF3DEF48F0F20EE126FF0EE2221200B3
:10915000060EE126000EE222FE0EE36AF50EE3BEE5
:10916000B6EF48F0B4EF48F0CAEF48F0F20EE36C07
:10917000F30EE31EF40EE31EF50EE31E08E3F30EFA
:10918000E32A05E3F40EE32A02E3F50EE32AFE0EDA
:10919000E36AE32AF90EE3BED2EF48F0D0EF48F0DD
:1091A000E5EF48F0F60EE36CF70EE31EF80EE31E53
:1091B000F90EE31E08E3F70EE32A05E3F80EE32AAF
:1091C00002E3F90EE32AFE0EE370FA0EE36AFB0EE9
:1091D000E36AFC0EE36AFD0EE36AF20EE3500FE170
:1091E000F30EE3500CE1F40EE35009E1F50EE35009
:1091F000D8B4FDEF48F0FFEF48F068EF49F0FF0EFC
:10920000E36AE32A0FEF49F0D890F20EE336F30E4B
:10921000E336F40EE336F50EE336FF0EE32AF50EE1
:10922000E3AE15EF49F017EF49F004EF49F0D8909D
:10923000FA0EE336FB0EE336FC0EE336FD0EE336A4
:10924000E150F60FD96EE250DA6EFF0EDA22F20E1E
:10925000E350DE5CF30EE350DE58F40EE350DE58CC
:10926000F50EE350DE58D8A038EF49F03AEF49F058
:109270004FEF49F0E150F60FD96EE250DA6EFF0E73
:10928000DA22F20EE350DE5EF30EE350DE5AF40E05
:10929000E350DE5AF50EE350DE5AFA0EE380D89022
:1092A000F50EE332F40EE332F30EE332F20EE33264
:1092B000FF0EE3502E6E010E2E5EFF0E6000BBF01F
:1092C000E3FFD8A466EF49F068EF49F017EF49F0E3
:1092D000FE0EE350D8B46FEF49F071EF49F082EF22
:1092E00049F0FA0EE36CFB0EE31EFC0EE31EFD0ECE
:1092F000E31E08E3FB0EE32A05E3FC0EE32A02E388
:10930000FD0EE32AFA0E6F008CFF2EF0FB0E6F00AD
:109310008CFF2FF0FC0E6F008CFF30F0FD0E6F0005
:109320008CFF31F0F20EE126FF0EE22212000A0E4F
:10933000E126000EE222F60EE36AF70EE36AF80E6B
:10934000E36AF90EE36AF20E6F008CFF39F0030E48
:109350003916FF0E6000E7F0E3FFF20E6F008CFF9E
:1093600039F0050E2E6ED89039322E2EB3EF49F01B
:10937000FE0E6000E7F0E3FFF30EE350386E396A4B
:10938000D89038363936D89038363936D89038367D
:109390003936F60E6000E3F0E3FFF70E6000E7F009
:1093A000E3FF2E6AE3BE2E68F80E6000BBF0E3FF19
:1093B000F90E6000BBF0E3FFE150F60FD96EE2500A
:1093C000DA6EFF0EDA22FE0EE350DE26000EDE22FB
:1093D000DE22DE22E150F60FD96EE250DA6EFF0E89
:1093E000DA22020ED890DE36DE36DE36DD36DD528B
:1093F000DD52E82EF2EF49F0E150F60FD96EE2505F
:10940000DA6EFF0EDA22FF0EE350DE26000EDE22B9
:10941000DE22DE22E150F60FD96EE250DA6EFF0E48
:10942000DA22080ED890DE36DE36DE36DD36DD5244
:10943000DD52E82E12EF4AF0E150F60FD96EE250FD
:10944000DA6EFF0EDA22F50EE350DE26000EDE2283
:10945000DE22DE22E150F60FD96EE250DA6EFF0E08
:10946000DA22080ED890DE36DE36DE36DD36DD5204
:10947000DD52E82E32EF4AF0E150F60FD96EE2509D
:10948000DA6EFF0EDA22F40EE350DE26000EDE2244
:10949000DE22DE22F60E6F008CFF36F0F70E6F0034
:1094A0008CFF37F0F80E6F008CFF38F0F90E6F006C
:1094B0008CFF39F0FA0E6000DBF0E3FFFB0E60007A
:1094C000DFF0E3FFFC0E6000E3F0E3FFFD0E600061
:1094D000E7F0E3FFFA0E6F008CFF2EF0FB0E6F003B
:1094E0008CFF2FF0FC0E6F008CFF30F0FD0E6F0034
:1094F0008CFF31F0F20EE126FF0EE2221200800E08
:109500008F6E8E50E00B800AD8A489EF4AF08BEF63
:109510004AF081EF4AF0900E916E3701006B3D6B7F
:10952000B90EE66E370EE66EB80EE66E370EE66ED4
:10953000BB0EE66E370EE66EBA0EE66E370EE66EC0
:10954000010EE66E700EE66E000EE66E000EE66E22
:10955000000EE66E8AEC47F0BD0EE66E370EE66E44
:10956000BC0EE66E370EE66EBF0EE66E370EE66E8A
:10957000BE0EE66E370EE66E010EE66E700EE66EFD
:10958000000EE66E000EE66E000EE66E8AEC47F008
:10959000A10EE66E370EE66EA00EE66E370EE66E94
:1095A000A30EE66E370EE66EA20EE66E370EE66E80
:1095B000010EE66E000EE66E000EE66E000EE66E22
:1095C000000EE66E8AEC47F0A50EE66E370EE66EEC
:1095D000A40EE66E370EE66EA70EE66E370EE66E4A
:1095E000A60EE66E370EE66E010EE66E100EE66E05
:1095F000000EE66E000EE66E000EE66E8AEC47F098
:10960000A90EE66E370EE66EA80EE66E370EE66E13
:10961000AB0EE66E370EE66EAA0EE66E370EE66EFF
:10962000010EE66E700EE66E000EE66E000EE66E41
:10963000000EE66E8AEC47F0070E3701066F100E3B
:10964000396F0F0E036F980E046F810E056FFA0EBF
:10965000E66EC90EE66E7DEC64F03901A593958344
:10966000040EE66ECA0EE66E67EC64F0060EE66E59
:10967000CA0EE66E72EC64F0FE0EE66EC90EE66E81
:1096800046EC64F0020EE66ECA0EE66E5CEC64F028
:10969000FC0EE66EC90EE66E3BEC64F0000EE66E64
:1096A000CA0EE66E51EC64F03901A59B958B8F6A6A
:1096B0006F0038FE39F0E00E3916D8A462EF4BF097
:1096C00064EF4BF058EF4BF01200FE0E6F008FFF6F
:1096D000D9FFFF0E6F008FFFDAFF6E0EDF6E030EF5
:1096E000E66EFD0EE350010F386EFE0E6F008CFF2C
:1096F00039F0000E39226000E3F0E6FF6000E7F089
:10970000E6FF1EEC46F0010EE66E100EE66EC80E89
:10971000E66EA40EE66EFA0EE350010F386EFB0EF5
:109720006F008CFF39F0000E39226000E3F0E6FF95
:109730006000E7F0E6FFD5EC5AF0FE0E6F008FFFF9
:10974000E6FF6F008FFFE6FF0E0EE66EBC0EE66EC4
:10975000FA0EE350010F386EFB0E6F008CFF39F0EC
:10976000000E39226000E3F0E6FF6000E7F0E6FF5C
:109770009AEC5AF0FE0E6F008FFFE6FF6F008FFF2E
:10978000E6FF9A0EE66EBB0EE66EFA0EE350010F90
:10979000386EFB0E6F008CFF39F0000E392260002E
:1097A000E3F0E6FF6000E7F0E6FFC1EC5BF0FE0EE1
:1097B0006F008FFFE6FF6F008FFFE6FF8E0EE66EF5
:1097C000C30EE66EFA0EE350010F386EFB0E6F000B
:1097D0008CFF39F0000E39226000E3F0E6FF6000F4
:1097E000E7F0E6FF10EC5BF0FE0E6F008CFF38F048
:1097F000FF0E6F008CFF39F0380E3824D96E000E42
:109800003920DA6EDE6ADD6AFE0E6F008CFF38F0FA
:10981000FF0E6F008CFF39F03C0E3824D96E000E1D
:109820003920DA6EDE6ADD6AFE0E6F008CFF38F0DA
:10983000FF0E6F008CFF39F0400E3824D96E000EF9
:109840003920DA6EDE6ADD6A980E0001CB6F8B0E6E
:10985000CC6F080ECD6F000ECE6FE552E5521200B0
:10986000FE0E6F008FFFD9FFFF0E6F008FFFDAFF34
:10987000640EDF6E020EE66EFD0EE350010F386ED1
:10988000FE0E6F008CFF39F0000E39226000E3F00D
:10989000E6FF6000E7F0E6FF1EEC46F0040EE66E21
:1098A000100EE66E5C0EE66EB20EE66EFA0EE35039
:1098B000010F386EFB0E6F008CFF39F0000E39225D
:1098C0006000E3F0E6FF6000E7F0E6FFD5EC5AF059
:1098D000FE0E6F008FFFE6FF6F008FFFE6FF6A0E40
:1098E000E66EBD0EE66EFA0EE350010F386EFB0E0B
:1098F0006F008CFF39F0000E39226000E3F0E6FFC4
:109900006000E7F0E6FF9AEC5AF0FE0E6F008FFF62
:10991000E6FF6F008FFFE6FFF60EE66EBC0EE66E0A
:10992000FA0EE350010F386EFB0E6F008CFF39F01A
:10993000000E39226000E3F0E6FF6000E7F0E6FF8A
:10994000C1EC5BF0FE0E6F008FFFE6FF6F008FFF34
:10995000E6FF820EE66EBC0EE66EFA0EE350010FD5
:10996000386EFB0E6F008CFF39F0000E392260005C
:10997000E3F0E6FF6000E7F0E6FF10EC5BF0FE0EC0
:109980006F008CFF38F0FF0E6F008CFF39F0380E3F
:109990003824D96E000E3920DA6EDE6ADD6AFE0EDA
:1099A0006F008CFF38F0FF0E6F008CFF39F03C0E1B
:1099B0003824D96E000E3920DA6EDE6ADD6AFE0EBA
:1099C0006F008CFF38F0FF0E6F008CFF39F0400EF7
:1099D0003824D96E000E3920DA6EDE6ADD6AE5526F
:1099E000E5521200E652E652FE0EE36AFF0EE36A0B
:1099F000FE0E6F008CFF38F0FF0E6F008CFF39F009
:109A00000F0E38026F00CCFF36F06F00D0FF37F03A
:109A10003902F3503726A10E3624386E040E372053
:109A2000396E6000E3F0E6FF6000E7F0E6FFE0EC8F
:109A300058F0FE0EE350010F2E6EFE0E6000BBF0DC
:109A4000E3FF2E6AFF0EE3502E202E6EFF0E600005
:109A5000BBF0E3FFFF0EE3BE3CEF4DF0FF0EE35023
:109A60000DE1FE0E6F008CFF2EF0140E2E5ED8A0BE
:109A70003CEF4DF03EEF4DF0F8EF4CF0FE0EE36A98
:109A8000FF0EE36AFE0E6F008CFF38F0FF0E6F00D2
:109A90008CFF39F0110E38026F00CCFF36F06F00EA
:109AA000D0FF37F03902F3503726F80E3624D96E3E
:109AB000020E3720DA6EDE6ADD6AFE0E6F008CFF62
:109AC00038F0FF0E6F008CFF39F0110E38026F0076
:109AD000CCFF36F06F00D0FF37F03902F350372655
:109AE000FA0E3624386E020E3720396E6000E3F02D
:109AF000E6FF6000E7F0E6FFE0EC58F0FE0EE35012
:109B0000010F2E6EFE0E6000BBF0E3FF2E6AFF0E0B
:109B1000E3502E202E6EFF0E6000BBF0E3FFFF0E21
:109B2000E3BEA1EF4DF0FF0EE3500DE1FE0E6F001E
:109B30008CFF2EF0190E2E5ED8A0A1EF4DF0A3EFF2
:109B40004DF042EF4DF0000E6F00A0FFCDF5000E7E
:109B50006F00A0FFCEF5E552E5521200E652E65244
:109B6000E652EE0EE1242E6EFF0EE2202F6E600014
:109B7000BBF0E6FF6000BFF0E6FF3CEC63F0FD0EDB
:109B80006000BBF0E3FFFE0E6000BFF0E3FFFD0EE0
:109B90006F008CFF2EF0FE0EE3502E10D8B4D3EFE2
:109BA0004DF0D5EF4DF00DEF4EF0000EE66E000ECD
:109BB000E66EEC0EE1242E6EFF0EE2202F6E6000AA
:109BC000BBF0E6FF6000BFF0E6FFE7EC61F0ED0EF2
:109BD000E350E66EED0EE124D96EFF0EE220DA6E60
:109BE0000F0E6F007BFFE6FFE82CF1EF4DF0ED0E5E
:109BF0006F008FFFE6FF6F008FFFE6FF79EC57F0F5
:109C0000EB0E6F008FFFD9FFEC0E6F008FFFDAFFB6
:109C10006000BBF0DFFF62EF4EF0ED0EE350E66E4A
:109C200018EC64F0140EE66E000EE66E21EECDF137
:109C3000DF50386E396A010E3826000E3922600076
:109C4000E3F0E6FF6000E7F0E6FFD2EC4FF0FF0E36
:109C50006000BBF0E3FF21EECEF1FF0EE350DE1813
:109C6000D8A435EF4EF037EF4EF040EF4EF0ED0E4A
:109C7000E350E66E0CEC64F0000E2E6E64EF4EF0D6
:109C8000EE0EE124D96EFF0EE220DA6E01EECDF188
:109C9000EF500F0DA10EF324E96E040EF420EA6ECE
:109CA0000E0E6F006FFFEBFFE806FBE2FF0E6F008A
:109CB0008CFF39F06000E4F0CDF5ED0EE350E66E78
:109CC0000CEC64F0010E2E6EEB0EE126FF0EE2228C
:109CD0001200100EE126000EE222190E396EFF0E60
:109CE0006000E7F0E3FFF00EE1242E6EFF0EE220AD
:109CF0002F6E6000BBF0E6FF6000BFF0E6FFE0EC17
:109D000058F0EE0E6F008FFFE6FF6F008FFFE6FF4B
:109D1000EE0EE1242E6EFF0EE2202F6E6000BBF0EF
:109D2000E6FF6000BFF0E6FF07EC62F0EC0E6F00AC
:109D30008FFFE6FF6F008FFFE6FFEE0EE1242E6E31
:109D4000FF0EE2202F6E6000BBF0E6FF6000BFF068
:109D5000E6FF27EC62F0EB0EE350E66EEF0EE12437
:109D60002E6EFF0EE2202F6E6000BBF0E6FF60005B
:109D7000BFF0E6FF8BEC63F0E90E6F008FFFE6FFAC
:109D80006F008FFFE6FFEE0EE1242E6EFF0EE22045
:109D90002F6E6000BBF0E6FF6000BFF0E6FFE7EC6F
:109DA00061F0E150E10FD96EE250DA6EFF0EDA2277
:109DB0006F007BFFE6FF6F007BFFE6FF6F007BFF1E
:109DC000E6FF6F007BFFE6FF6F007BFFE6FF6F00A3
:109DD0007BFFE6FF6F007BFFE6FF6F007BFFE6FF88
:109DE000E80EE1242E6EFF0EE2202F6E6000BBF025
:109DF000E6FF6000BFF0E6FFA3EC62F0FF0EE12497
:109E00002E6EFF0EE2202F6E6000BBF0E6FF6000BA
:109E1000BFF0E6FF000EE66EED0EE124D96EFF0EF8
:109E2000E220DA6E0F0E6F007BFFE6FFE82C13EFE7
:109E30004FF0AEEC4DF0E10EE126FF0EE2221200F3
:109E4000E652E652E652E652FB0EE3BE2AEF4FF030
:109E50002CEF4FF04EEF4FF0F80E6F008CFF36F006
:109E6000F90E6F008CFF37F0FA0E6F008CFF38F0A0
:109E7000FB0E6F008CFF39F0FC0E6000DBF0E3FF9F
:109E8000FD0E6000DFF0E3FFFE0E6000E3F0E3FF95
:109E9000FF0E6000E7F0E3FF77EF4FF0F80E6F0082
:109EA0008CFF36F0F90E6F008CFF37F0FA0E6F0062
:109EB0008CFF38F0FB0E6F008CFF39F0361E371E1A
:109EC000381E391E362A000E372238223922FC0E5F
:109ED0006000DBF0E3FFFD0E6000DFF0E3FFFE0E4D
:109EE0006000E3F0E3FFFF0E6000E7F0E3FFD00E59
:109EF000E66E070EE66E000EE66E000EE66EF80EDB
:109F00006F008FFFE6FF6F008FFFE6FF6F008FFF90
:109F1000E6FF6F008FFFE6FFF2EC53F0FC0E6000EF
:109F2000BBF0E3FFFD0E6000BFF0E3FFFE0E60003C
:109F3000C3F0E3FFFF0E6000C7F0E3FF60000FF027
:109F4000E6FF600013F0E6FF600017F0E6FF600038
:109F50001BF0E6FFF80E6F008FFFE6FF6F008FFF2C
:109F6000E6FF6F008FFFE6FF6F008FFFE6FFC8EC94
:109F700051F0FC0E6000BBF0E3FFFD0E6000BFF08F
:109F8000E3FFFE0E6000C3F0E3FFFF0E6000C7F0CA
:109F9000E3FFFC0E6F008CFFD4F0F80EE126FF0EFD
:109FA000E2221200E652E652FE0EE36AFD0EE3BE26
:109FB000DEEF4FF0DCEF4FF0E7EF4FF0FC0EE36C1D
:109FC000FD0EE31ED8B0E32AFE0EE36AE32AFB0E81
:109FD000E3BEEFEF4FF0EDEF4FF0F5EF4FF0FA0E7D
:109FE000E36CFB0EE31ED8B0E32AFA0E6F008CFF81
:109FF0002EF0FB0EE3502E10D8B401EF50F003EF1B
:10A0000050F067EF50F0FF0EE36AE32A1BEF50F0C9
:10A01000FA0EE350D890E8342E6EFA0E6000BBF0D2
:10A02000E3FFFB0EE350E8342E6EFB0E6000BBF046
:10A03000E3FFFF0EE32AFB0EE3AE21EF50F023EF28
:10A0400050F008EF50F0FA0E6F008CFF38F0FB0E66
:10A050006F008CFF39F0FC0E6F008CFF36F0FD0EA8
:10A060006F008CFF37F03850365C39503758D8A025
:10A070003CEF50F03EEF50F052EF50F0FC0EE3504A
:10A080002E6EFA0EE3502E5EFC0E6000BBF0E3FF76
:10A09000FD0EE3502E6EFB0EE3502E5AFD0E6000B7
:10A0A000BBF0E3FFD890FB0EE332FA0EE332FF0E73
:10A0B000E3502E6E010E2E5EFF0E6000BBF0E3FF3C
:10A0C000D8A465EF50F067EF50F023EF50F0FE0E8C
:10A0D000E350D8B46EEF50F070EF50F076EF50F0E0
:10A0E000FC0EE36CFD0EE31ED8B0E32AFC0E6F00FD
:10A0F0008CFF2EF0FD0E6F008CFF2FF0FA0EE12684
:10A10000FF0EE22212006F00E8FF4EF06F00ECFF3E
:10A110004FF06000B8F050F06000BCF051F060000B
:10A12000C0F052F06000C4F053F06000D8F054F07A
:10A130006000DCF055F06000E0F056F06000E4F004
:10A1400057F06000F8F058F06000FCF059F0600043
:10A1500000F15AF0600004F15BF0600008F15CF07F
:10A1600060000CF15DF0600010F15EF0600014F131
:10A170005FF012EEE8F2390193AFC1EF50F0C3EF98
:10A1800050F0CEEF50F0A3AFC8EF50F0CAEF50F050
:10A19000CEEF50F00CEC63F0F2EF50F095ABD3EF54
:10A1A00050F0D5EF50F0E0EF50F0A5ABDAEF50F003
:10A1B000DCEF50F0E0EF50F07AEC53F0F2EF50F0BB
:10A1C00095A3E5EF50F0E7EF50F0F2EF50F0A5A3C4
:10A1D000ECEF50F0EEEF50F0F2EF50F0BAEC63F02D
:10A1E000F2EF50F060007CF145F0600078F144F04F
:10A1F000600074F143F0600070F142F060006CF1B7
:10A2000041F0600068F140F0600064F13FF06000F0
:10A2100060F13EF060005CF139F0600058F138F018
:10A22000600054F137F0600050F136F060004CF1FE
:10A2300031F0600048F130F0600044F12FF0600030
:10A2400040F12EF060003FF1FBFF60003BF1FAFFB0
:10A250001100FE0E6F008FFFD9FFFF0E6F008FFF02
:10A26000DAFFDF6AFE0E6F008CFF38F0FF0E6F0022
:10A270008CFF39F0010E3824D96E000E3920DA6EC9
:10A28000F40EDE6E010EDD6EFE0E6F008CFF38F0F8
:10A29000FF0E6F008CFF39F0030E3824D96E000ECC
:10A2A0003920DA6EF40EDE6E010EDD6EFE0E6F00EA
:10A2B0008CFF38F0FF0E6F008CFF39F0050E38244C
:10A2C000D96E000E3920DA6E030EDF6EFE0E6F00BF
:10A2D0008CFF38F0FF0E6F008CFF39F0060E38242B
:10A2E000D96E000E3920DA6EDF6AFE0E6F008CFF29
:10A2F00038F0FF0E6F008CFF39F0070E3824D96E4E
:10A30000000E3920DA6E030EDF6EFE0E6F008CFF3A
:10A3100038F0FF0E6F008CFF39F0080E3824D96E2C
:10A32000000E3920DA6EDE6ADD6AFE0E6F008CFFE9
:10A3300038F0FF0E6F008CFF39F00C0E3824D96E08
:10A34000000E3920DA6EDE6ADD6AFE0E6F008CFFC9
:10A3500038F0FF0E6F008CFF39F0100E3824D96EE4
:10A36000000E3920DA6EDE6ADD6AFE0E6F008CFFA9
:10A3700038F0FF0E6F008CFF39F0140E3824D96EC0
:10A38000000E3920DA6EDE6ADD6AE552E55212000F
:10A39000050EE126000EE222FB0EE36AFC0EE36AE4
:10A3A000FD0EE36AFE0EE36AF30EE3500FE1F40ED6
:10A3B000E3500CE1F50EE35009E1F60EE350D8B49A
:10A3C000E4EF51F0E6EF51F04FEF52F0FF0EE36A89
:10A3D000E32AF6EF51F0D890F30EE336F40EE336AD
:10A3E000F50EE336F60EE336FF0EE32AF60EE3AE85
:10A3F000FCEF51F0FEEF51F0EBEF51F0D890FB0E77
:10A40000E336FC0EE336FD0EE336FE0EE336E15096
:10A41000F70FD96EE250DA6EFF0EDA22F30EE35038
:10A42000DE5CF40EE350DE58F50EE350DE58F60E17
:10A43000E350DE58D8A01FEF52F021EF52F036EF74
:10A4400052F0E150F70FD96EE250DA6EFF0EDA22C9
:10A45000F30EE350DE5EF40EE350DE5AF50EE350E9
:10A46000DE5AF60EE350DE5AFB0EE380D890F60E6D
:10A47000E332F50EE332F40EE332F30EE332FF0E75
:10A48000E3502E6E010E2E5EFF0E6000BBF0E3FF68
:10A49000D8A44DEF52F04FEF52F0FEEF51F0FB0E0B
:10A4A0006F008CFF2EF0FC0E6F008CFF2FF0FD0E66
:10A4B0006F008CFF30F0FE0E6F008CFF31F0F30E5A
:10A4C000E126FF0EE2221200050EE126000EE22236
:10A4D000F90E6F008FFFF6FFFA0E6F008FFFF7FF88
:10A4E000000EF86E0F0EF76403D00800F55007D089
:10A4F0006F00DBFFE9FF6F00DFFFEAFFEF50396E0F
:10A50000FF0E6000E7F0E3FFBCEF52F0FB0EE36AE2
:10A51000E32AFC0EE124D96EFF0EE220DA6EDF6A38
:10A52000FD0EE124D96EFF0EE220DA6EDF6AD6EF6F
:10A5300052F0FB0EE36AFC0EE124D96EFF0EE2201E
:10A54000DA6E010EDF6E90EF52F0FB0EE36AFC0E46
:10A55000E124D96EFF0EE220DA6EDF6AFD0EE124FF
:10A56000D96EFF0EE220DA6E010EDF6ED6EF52F0EA
:10A57000FB0EE36A89EF52F0FF0EE350386E396A42
:10A580003950000AD8B4C7EF52F0B8EF52F0385043
:10A59000010AD8B486EF52F0030AD8B499EF52F00A
:10A5A000010AD8B4A5EF52F0B8EF52F0FE0EE12444
:10A5B000D96EFF0EE220DA6E600067F0DFFFFB0E5F
:10A5C0006F008FFFE6FF6F008FFFE6FF6F008FFFCA
:10A5D000E6FF6F008FFFE6FF000EE66E050EE66EEB
:10A5E00059EC3BF0F90EE126FF0EE2221200E65292
:10A5F000E652FF0EE36AFF0EE350110DFA0EF3244C
:10A60000D96E020EF420DA6EDF50D8B40AEF53F0A0
:10A610000CEF53F069EF53F0FF0EE350110DF80EFD
:10A62000F324D96E020EF420DA6E0A0EDE5E000EFE
:10A63000DD5AFF0EE350110DF80EF324D96E020E11
:10A64000F420DA6EDE50DE10D8A429EF53F02BEFA1
:10A6500053F069EF53F0FE0EE1242E6EFF0EE22060
:10A660002F6E6000BBF0E6FF6000BFF0E6FF010E5A
:10A67000E66EFC0EE350110DFA0EF324D96E020EB5
:10A68000F420DA6E0F0E6F007BFFE6FFE82C43EF3D
:10A6900053F0AEEC4DF02E04D8A451EF53F053EF2D
:10A6A00053F05CEF53F0010EE66EFE0EE350E66EE3
:10A6B0007EEC60F069EF53F0FF0EE350110DF80EE1
:10A6C000F324D96E020EF420DA6E010EDE6E000E57
:10A6D000DD6EFF0EE32AFF0E6F008CFF2EF0180ECA
:10A6E0002E6475EF53F077EF53F0FBEF52F0E55225
:10A6F000E552120090AC7FEF53F081EF53F08EEFF4
:10A7000053F002D88DEF53F00500FA6E2650FD6E1F
:10A710002750FE6EFF6AFA501200909C90AA93EFA9
:10A7200053F095EF53F0A1EF53F002D8A1EF53F09F
:10A730000500FA6E2450FD6E2550FE6EFF6AFA5039
:10A74000120090A8A6EF53F0A8EF53F0B4EF53F027
:10A7500002D8B4EF53F00500FA6E2250FD6E23507C
:10A76000FE6EFF6AFA50120090A6B9EF53F0BBEFED
:10A7700053F0C7EF53F002D8C7EF53F00500FA6E5D
:10A780002050FD6E2150FE6EFF6AFA50120090A418
:10A79000CCEF53F0CEEF53F0DBEF53F002D8DBEF0A
:10A7A00053F00500FA6E0001C751FD6EC851FE6EF0
:10A7B000FF6AFA50120090A2E0EF53F0E2EF53F07C
:10A7C000EFEF53F002D8EFEF53F00500FA6E0001FF
:10A7D000C551FD6EC651FE6EFF6AFA501200390176
:10A7E000A59B1200E652E652E652E652FC0EE36AE0
:10A7F000FD0EE36AFE0EE36AFF0EE36AF80EE3A0C5
:10A8000004EF54F006EF54F02EEF54F0FC0EE3503A
:10A810002E6EF40EE3502E26FC0E6000BBF0E3FF1C
:10A82000FD0EE3502E6EF50EE3502E22FD0E60005D
:10A83000BBF0E3FFFE0EE3502E6EF60EE3502E2229
:10A84000FE0E6000BBF0E3FFFF0EE3502E6EF70E2E
:10A85000E3502E22FF0E6000BBF0E3FFD890F40E11
:10A86000E336F50EE336F60EE336F70EE336D89010
:10A87000FB0EE332FA0EE332F90EE332F80EE33266
:10A88000F80EE3500DE1F90EE3500AE1FA0EE35041
:10A8900007E1FB0EE350D8A450EF54F052EF54F010
:10A8A000FEEF53F0FC0E6F008CFF2EF0FD0E6F00DC
:10A8B0008CFF2FF0FE0E6F008CFF30F0FF0E6F004C
:10A8C0008CFF31F0F40EE126FF0EE2221200080E9A
:10A8D000E126000EE222F60E6F008FFFD9FFF70E81
:10A8E0006F008FFFDAFF6F0078FF36F06F0078FFA0
:10A8F00037F06F0078FF38F06F0078FF39F0FC0E0A
:10A900006000DBF0E3FFFD0E6000DFF0E3FFFE0E12
:10A910006000E3F0E3FFFF0E6000E7F0E3FFFF0EEF
:10A92000E124D96EFF0EE220DA6EDF50396EF80EA8
:10A930006000E7F0E3FFFE0EE124D96EFF0EE22097
:10A94000DA6EF90EE124E96EFF0EE220EA6E6F0086
:10A950007FFFEFFFFD0EE124D96EFF0EE220DA6EDD
:10A96000FA0EE124E96EFF0EE220EA6E6F007FFF2F
:10A97000EFFFFB0EE124D96EFF0EE220DA6EFC0E33
:10A980006F008FFFDFFFF80E6F008FFFE6FF6F0095
:10A990008FFFE6FF6F008FFFE6FF6F008FFFE6FF80
:10A9A000010EE66E050EE66E59EC3BF0F60EE12662
:10A9B000FF0EE2221200E652E652FC0E6F008CFF00
:10A9C00038F0FD0E6F008CFF39F0FF0E6000E7F0ED
:10A9D000E3FFFE0E6000E3F0E3FF07EF55F0BA80FF
:10A9E0004AEF55F0BA824AEF55F0BA844AEF55F073
:10A9F000BA864AEF55F0BA884AEF55F0BA8A4AEF5C
:10AA000055F0BA8C4AEF55F0BA8E4AEF55F0FE0E6B
:10AA10006F008FFFF6FFFF0E6F008FFFF7FF000E36
:10AA2000F86E0F0EF76403D00800F55007D06F00E2
:10AA3000DBFFE9FF6F00DFFFEAFFEF50386E396A96
:10AA40003950000AD8B427EF55F04AEF55F0385086
:10AA5000010AD8B4EFEF54F0030AD8B4F2EF54F07F
:10AA6000010AD8B4F5EF54F0070AD8B4F8EF54F05F
:10AA7000010AD8B4FBEF54F0030AD8B4FEEF54F047
:10AA8000010AD8B401EF55F00F0AD8B404EF55F01D
:10AA90004AEF55F0E552E552E552E5521200E65212
:10AAA000E652FC0E6F008CFF38F0FD0E6F008CFF3D
:10AAB00039F0FF0E6000E7F0E3FFFE0E6000E3F008
:10AAC000E3FF7BEF55F0BA90BEEF55F0BA92BEEFC0
:10AAD00055F0BA94BEEF55F0BA96BEEF55F0BA985D
:10AAE000BEEF55F0BA9ABEEF55F0BA9CBEEF55F0E6
:10AAF000BA9EBEEF55F0FE0E6F008FFFF6FFFF0E01
:10AB00006F008FFFF7FF000EF86E0F0EF76403D093
:10AB10000800F55007D06F00DBFFE9FF6F00DFFF93
:10AB2000EAFFEF50386E396A3950000AD8B49BEF0B
:10AB300055F0BEEF55F03850010AD8B463EF55F028
:10AB4000030AD8B466EF55F0010AD8B469EF55F09E
:10AB5000070AD8B46CEF55F0010AD8B46FEF55F07E
:10AB6000030AD8B472EF55F0010AD8B475EF55F066
:10AB70000F0AD8B478EF55F0BEEF55F0E552E55224
:10AB8000E552E5521200080EE126000EE222F70E11
:10AB9000E350386E396AD89038363936D89038361E
:10ABA0003936D89038363936F80E6000E3F0E3FFD6
:10ABB000F90E6000E7F0E3FF2E6AE3BE2E68FA0E9E
:10ABC0006000BBF0E3FFFB0E6000BBF0E3FFE15071
:10ABD000F80FD96EE250DA6EFF0EDA22F60E6F0031
:10ABE0008CFF39F0050E2E6ED89039322E2EF4EFF0
:10ABF00055F03950DE26000EDE22DE22DE22F80E6F
:10AC00006F008CFF36F0F90E6F008CFF37F0FA0EF4
:10AC10006F008CFF38F0FB0E6F008CFF39F0FC0EDC
:10AC20006000DBF0E3FFFD0E6000DFF0E3FFFE0EEF
:10AC30006000E3F0E3FFFF0E6000E7F0E3FFFC0ECF
:10AC40006F008CFF2EF0FD0E6F008CFF2FF0FE0EBC
:10AC50006F008CFF30F0FF0E6F008CFF31F0F60EAE
:10AC6000E126FF0EE22212001D0EE126000EE22276
:10AC7000F10EE36AF40EE124D96EFF0EE220DA6EE3
:10AC8000DE6ADD6AF20EE124D96EFF0EE220DA6E92
:10AC9000DE6ADD6AE20EE350E66E18EC64F021EE47
:10ACA000CEF101EECDF1DE50EE18D8A45AEF56F0F9
:10ACB0005CEF56F072EF56F0E20EE350E66E0CECED
:10ACC00064F0F10EE124D96EFF0EE220DA6E0F0E71
:10ACD0002E6EE20E6F007BFFE3FFE8282E2EFAD7E0
:10ACE0009FEF56F021EECEF1DF500F0DA10EF324B1
:10ACF000D96E040EF420DA6E0F0E2E6EF10E6F0078
:10AD00007BFFE3FFE8282E2EFAD7140EE66E000E26
:10AD1000E66E21EECEF1DF50386E396A010E38262C
:10AD2000000E39226000E3F0E6FF6000E7F0E6FF86
:10AD3000D2EC4FF06000B8F0CEF55CEF56F0F10EBB
:10AD4000E126FF0EE2221200070EE66EF5EC64F03B
:10AD50006000BBF0E6FF6000BFF0E6FF9BEC63F035
:10AD6000080EE66EAFEC64F06000BBF0E6FF60003A
:10AD7000BFF0E6FF9BEC63F0F5EC64F06000BBF025
:10AD8000E6FF6000BFF0E6FF24EC64F0AFEC64F097
:10AD90006000BBF0E6FF6000BFF0E6FF24EC64F06B
:10ADA000EFEC64F0010EE66EE9EC64F0FAEC3CF0D6
:10ADB0009AEC3EF0050EE66ED3EC64F06000BBF05A
:10ADC000E6FF6000BFF0E6FF1EEC46F00250E66EC4
:10ADD000D3EC64F06000BBF0E6FF6000BFF0E6FF7C
:10ADE00054EC60F0010EE66ECAEC64F06000BBF05B
:10ADF000E6FF6000BFF0E6FF1EEC46F0B8EC64F042
:10AE00006000BBF0E6FF6000BFF0E6FF30EC4CF006
:10AE1000A6EC64F06000BBF0E6FF6000BFF0E6FF68
:10AE200065EC4BF012000F0EE126000EE222000E40
:10AE3000E66E34EC56F0F10EE124D96EFF0EE220FE
:10AE4000DA6E0F0E2E6EDD50E552E750DF6E2E2EBD
:10AE5000FAD7F10EE350D8B430EF57F032EF57F095
:10AE600074EF57F0F40EE124D96EFF0EE220DA6E93
:10AE7000DE50DE10D8B43FEF57F041EF57F074EFDB
:10AE800057F0F20EE124D96EFF0EE220DA6EDE50AA
:10AE9000DE10D8B44EEF57F050EF57F074EF57F084
:10AEA000F10EE1242E6EFF0EE2202F6E6000BBF04B
:10AEB000E6FF6000BFF0E6FFF00EE124D96EFF0E62
:10AEC000E220DA6E6F0078FF38F06F0074FF39F01F
:10AED00002D874EF57F00500FA6E3850FD6E395005
:10AEE000FE6EFF6AFA501200F10EE126FF0EE2221A
:10AEF0001200E652ED0EE350E66E18EC64F0FF0E21
:10AF0000E36AFF0EE350110DFA0EF324D96E020E20
:10AF1000F420DA6EDF50D8A490EF57F092EF57F09C
:10AF2000BFEF57F0E150FD0FD96EE250DA6EFF0E21
:10AF3000DA22FF0EE350110DF80EF324E96E020E33
:10AF4000F420EA6E6F007BFFEEFF6F0077FFEDFFEE
:10AF5000EE0EE124D96EFF0EE220DA6EFF0EE35012
:10AF6000110DFA0EF324E96E020EF420EA6E0E0EB5
:10AF70006F006FFFEBFFE806FBE2CDEF57F0FF0E2F
:10AF8000E32AFF0E6F008CFF2EF0180E2E64CBEF1D
:10AF900057F0CDEF57F081EF57F0ED0EE350E66E2E
:10AFA0000CEC64F0FF0E6F008CFF2EF0ED0EE1262E
:10AFB000FF0EE2221200060EE126000EE222F50E3E
:10AFC0006F008CFF36F0F60E6F008CFF37F0F70E37
:10AFD0006F008CFF38F0F80E6F008CFF39F0FC0E1C
:10AFE0006000DBF0E3FFFD0E6000DFF0E3FFFE0E2C
:10AFF0006000E3F0E3FFFF0E6000E7F0E3FFFB0E0D
:10B00000E36AF90E6F008CFF2EF0FA0E6000BBF0C1
:10B01000E3FFFA0EE3502E6EFB0EE3502E26FA0EDF
:10B020006000BBF0E3FFFB0E6F008CFF39F0FC0EFD
:10B03000E124366EFF0EE220376E39503624D96E89
:10B04000000E3720DA6EDF50E66EF90EE350E66E42
:10B05000FFEC63F0FB0EE32AFB0E6F008CFF2EF07B
:10B06000030E2E6436EF58F038EF58F001EF58F029
:10B07000F50EE126FF0EE2221200060EE126000E7A
:10B08000E222FB0EE36AF90E6F008CFF2EF0FA0E3F
:10B090006000BBF0E3FFFA0EE3502E6EFB0EE350B0
:10B0A0002E26FA0E6000BBF0E3FFFA0EE350E66EC8
:10B0B000C1EC64F0FB0E6F008CFF39F0FC0EE12454
:10B0C000366EFF0EE220376E39503624D96E000EF0
:10B0D0003720DA6E6000BBF0DFFFFB0EE32AFB0EC9
:10B0E0006F008CFF2EF0030E2E6479EF58F07BEF8B
:10B0F00058F043EF58F0FC0E6F008CFF2EF0FD0E61
:10B100006F008CFF2FF0FE0E6F008CFF30F0FF0EF3
:10B110006F008CFF31F0F90EE126FF0EE2221200E3
:10B12000060EE126000EE222F80E6F008FFFE9FF07
:10B13000F90E6F008FFFEAFFFE0E6F00BBFFE3FF0B
:10B14000FF0E6F00B7FFE3FFFF0EE124D96EFF0E85
:10B15000E220DA6EDF50396EFA0E6000E7F0E3FFAE
:10B16000FB0EE124D96EFF0EE220DA6EFE0E6F00B8
:10B170008FFFDFFFFC0EE124D96EFF0EE220DA6EB6
:10B18000DF6AFD0EE124D96EFF0EE220DA6EDF6A7F
:10B19000FA0E6F008FFFE6FF6F008FFFE6FF6F0074
:10B1A0008FFFE6FF6F008FFFE6FF010EE66E040ED5
:10B1B000E66E59EC3BF0F80EE126FF0EE22212009B
:10B1C000FE0E6F008FFFD9FFFF0E6F008FFFDAFFBB
:10B1D000DF6AFE0E6F008CFF38F0FF0E6F008CFFF1
:10B1E00039F0050E3824D96E000E3920DA6EDE6A89
:10B1F000DD6AFE0E6F008CFF38F0FF0E6F008CFFD3
:10B2000039F0030E3824D96E000E3920DA6EDE6A6A
:10B21000DD6AFE0E6F008CFF38F0FF0E6F008CFFB2
:10B2200039F0070E3824D96E000E3920DA6E070E79
:10B23000DE6AE806FDE2FE0E6F008CFF38F0FF0EBE
:10B240006F008CFF39F0010E3824D96E000E3920C2
:10B25000DA6EDE6ADD6AE552E5521200E652E65227
:10B26000E652E652FA0E6F008CFF2EF0FC0E6000E4
:10B27000BBF0E3FFFD0EE124D96EFF0EE220DA6E93
:10B2800060005BF0DFFFFE0EE124D96EFF0EE220CE
:10B29000DA6E60005FF0DFFFFF0EE124D96EFF0E73
:10B2A000E220DA6E600063F0DFFFFC0E6F008FFFBC
:10B2B000E6FF6F008FFFE6FF6F008FFFE6FF6F0076
:10B2C0008FFFE6FF000EE66E040EE66E59EC3BF0D3
:10B2D000FA0EE126FF0EE2221200E652E652E65294
:10B2E000E652FC0EE36AFA0E6F008FFFD9FFFB0EE9
:10B2F0006F008FFFDAFFFD0EE124E96EFF0EE22002
:10B30000EA6E6F007FFFEFFFFE0EE124D96EFF0EA5
:10B31000E220DA6EDF6AFF0EE124D96EFF0EE22032
:10B32000DA6EDF6AFC0E6F008FFFE6FF6F008FFFA3
:10B33000E6FF6F008FFFE6FF6F008FFFE6FF020E54
:10B34000E66E030EE66E59EC3BF0FA0EE126FF0EB8
:10B35000E2221200E652D2BEB0EF59F0B4EF59F03B
:10B36000396A392AB5EF59F0396AFF0E6000E7F003
:10B37000E3FFFE0EE124D96EFF0EE220DA6EDF500D
:10B38000030B3901E16FFD0E6F008FFFE0F9FC0E3A
:10B390006F008FFFE3F93F0EE517E585D29E550E4E
:10B3A000E66FAA0EE66FE583E5B3D9EF59F0DBEF60
:10B3B00059F0D4EF59F0E595FF0EE3B002D0D29EDC
:10B3C00001D0D28EE552E552E552E5521200560EFA
:10B3D000E66E800EE66E7DEC64F0320EE66E460E92
:10B3E000E66E88EC64F0000EE66E000EE66ED20E9D
:10B3F000E66EC60EE66ED3EC64F06000BBF0E6FFCE
:10B400006000BFF0E6FFFCEC5BF01450E66ECAECA7
:10B4100064F06000BBF0E6FF6000BFF0E6FF54ECB4
:10B4200060F0000EE66E000EE66EAE0EE66EC70E23
:10B43000E66ECAEC64F06000BBF0E6FF6000BFF0AF
:10B44000E6FFC1EC5BF01200E652E652E652E6522D
:10B45000FC0E60006BF0E3FFFD0EE124D96EFF0EE1
:10B46000E220DA6E60006FF0DFFFFE0EE124D96E9D
:10B47000FF0EE220DA6E600073F0DFFFFF0EE124C2
:10B48000D96EFF0EE220DA6E600077F0DFFFFC0E6F
:10B490006F008FFFE6FF6F008FFFE6FF6F008FFFEB
:10B4A000E6FF6F008FFFE6FF000EE66E060EE66E0B
:10B4B00059EC3BF0FA0EE126FF0EE2221200E652B2
:10B4C000E652E652E652FC0E600047F0E3FFFD0E46
:10B4D000E124D96EFF0EE220DA6E60004BF0DFFF50
:10B4E000FE0EE124D96EFF0EE220DA6E60004FF00E
:10B4F000DFFFFF0EE124D96EFF0EE220DA6E60005E
:10B5000053F0DFFFFC0E6F008FFFE6FF6F008FFF31
:10B51000E6FF6F008FFFE6FF6F008FFFE6FF000E74
:10B52000E66E020EE66E59EC3BF0FA0EE126FF0ED7
:10B53000E2221200E150FC0FD96EE250DA6EFF0EEB
:10B54000DA22FE0E6F008CFF38F0FF0E6F008CFFCA
:10B5500039F0270E3824E96E000E3920EA6E6F00AC
:10B560007BFFEEFF6F0077FFEDFFE150FA0FD96E22
:10B57000E250DA6EFF0EDA22FE0E6F008CFF38F01A
:10B58000FF0E6F008CFF39F0290E3824E96E000E93
:10B590003920EA6E6F007BFFEEFF6F0077FFEDFF53
:10B5A000FA0EE126FF0EE2221200E150FC0FD96EE6
:10B5B000E250DA6EFF0EDA22FE0E6F008CFF38F0DA
:10B5C000FF0E6F008CFF39F01F0E3824E96E000E5D
:10B5D0003920EA6E6F007BFFEEFF6F0077FFEDFF13
:10B5E000E150FA0FD96EE250DA6EFF0EDA22FE0E4B
:10B5F0006F008CFF38F0FF0E6F008CFF39F0210ECA
:10B600003824E96E000E3920EA6E6F007BFFEEFFF2
:10B610006F0077FFEDFFFA0EE126FF0EE222120027
:10B62000E150FC0FD96EE250DA6EFF0EDA22FE0E08
:10B630006F008CFF38F0FF0E6F008CFF39F0230E87
:10B640003824E96E000E3920EA6E6F007BFFEEFFB2
:10B650006F0077FFEDFFE150FA0FD96EE250DA6E1E
:10B66000FF0EDA22FE0E6F008CFF38F0FF0E6F0027
:10B670008CFF39F0250E3824E96E000E3920EA6E71
:10B680006F007BFFEEFF6F0077FFEDFFFA0EE12604
:10B69000FF0EE2221200E150FC0FD96EE250DA6E8A
:10B6A000FF0EDA22FE0E6F008CFF38F0FF0E6F00E7
:10B6B0008CFF39F00C0E3824E96E000E3920EA6E4A
:10B6C0006F007BFFEEFF6F0077FFEDFFE150FA0F99
:10B6D000D96EE250DA6EFF0EDA22FE0E6F008CFF9A
:10B6E00038F0FF0E6F008CFF39F00E0E3824E96E33
:10B6F000000E3920EA6E6F007BFFEEFF6F0077FFD0
:10B70000EDFFFA0EE126FF0EE2221200E150FC0FDF
:10B71000D96EE250DA6EFF0EDA22FE0E6F008CFF59
:10B7200038F0FF0E6F008CFF39F0100E3824E96EF0
:10B73000000E3920EA6E6F007BFFEEFF6F0077FF8F
:10B74000EDFFE150FA0FD96EE250DA6EFF0EDA2209
:10B75000FE0E6F008CFF38F0FF0E6F008CFF39F08B
:10B76000120E3824E96E000E3920EA6E6F007BFF5E
:10B77000EEFF6F0077FFEDFFFA0EE126FF0EE222EB
:10B780001200E150FC0FD96EE250DA6EFF0EDA22A1
:10B79000FE0E6F008CFF38F0FF0E6F008CFF39F04B
:10B7A0002B0E3824E96E000E3920EA6E6F007BFF05
:10B7B000EEFF6F0077FFEDFFE150FA0FD96EE25018
:10B7C000DA6EFF0EDA22FE0E6F008CFF38F0FF0EED
:10B7D0006F008CFF39F02D0E3824E96E000E3920F1
:10B7E000EA6E6F007BFFEEFF6F0077FFEDFFFA0E52
:10B7F000E126FF0EE2221200E150FC0FD96EE2506A
:10B80000DA6EFF0EDA22FE0E6F008CFF38F0FF0EAC
:10B810006F008CFF39F02F0E3824E96E000E3920AE
:10B82000EA6E6F007BFFEEFF6F0077FFEDFFE150E8
:10B83000FA0FD96EE250DA6EFF0EDA22FE0E6F00BA
:10B840008CFF38F0FF0E6F008CFF39F0310E38247A
:10B85000E96E000E3920EA6E6F007BFFEEFF6F008D
:10B8600077FFEDFFFA0EE126FF0EE2221200E15013
:10B87000F40FD96EE250DA6EFF0EDA226F007BFF12
:10B88000E6FF6F007BFFE6FF6F007BFFE6FF6F00C8
:10B890007BFFE6FF6F007BFFE6FF6F007BFFE6FFAD
:10B8A0006F007BFFE6FF6F007BFFE6FFF40E6F008B
:10B8B0008FFFE6FF6F008FFFE6FF690EE66E4E0E0C
:10B8C000E66E5F0EE66EF10E6F008FFFE6FF6F0013
:10B8D0008FFFE6FF69EC4EF0F40EE126FF0EE22248
:10B8E0001200E652E652FC0E6F008CFF38F0FD0E9F
:10B8F0006F008CFF39F0FF0E6000E7F0E3FFFE0EF3
:10B900006000E3F0E3FF000EE66E000EE66E000E50
:10B91000E66E000EE66E000EE66E000EE66E000E9F
:10B92000E66E000EE66E000EE66E000EE66E720E1D
:10B93000E66E3C0EE66E680EE66EF10E6F008FFF4F
:10B94000E6FF6F008FFFE6FF69EC4EF0E552E5522F
:10B95000E552E5521200E652E652FC0E6F008CFFF3
:10B9600038F0FD0E6F008CFF39F0FF0E6000E7F03D
:10B97000E3FFFE0E6000E3F0E3FF000EE66E000E54
:10B98000E66E000EE66E000EE66E000EE66E000E2F
:10B99000E66E000EE66E000EE66E000EE66E000E1F
:10B9A000E66E680EE66E4E0EE66E5F0EE66EF10E09
:10B9B0006F008FFFE6FF6F008FFFE6FF69EC4EF030
:10B9C000E552E552E552E5521200E150F40FD96E0E
:10B9D000E250DA6EFF0EDA226F007BFFE6FF6F00A7
:10B9E0007BFFE6FF6F007BFFE6FF6F007BFFE6FF5C
:10B9F0006F007BFFE6FF6F007BFFE6FF6F007BFFC2
:10BA0000E6FF6F007BFFE6FFF40E6F008FFFE6FF9F
:10BA10006F008FFFE6FF190EE66E060EE66E100E43
:10BA2000E66EF10E6F008FFFE6FF6F008FFFE6FFFF
:10BA300069EC4EF0F40EE126FF0EE2221200E15016
:10BA4000F40FD96EE250DA6EFF0EDA226F007BFF40
:10BA5000E6FF6F007BFFE6FF6F007BFFE6FF6F00F6
:10BA60007BFFE6FF6F007BFFE6FF6F007BFFE6FFDB
:10BA70006F007BFFE6FF6F007BFFE6FFF40E6F00B9
:10BA80008FFFE6FF6F008FFFE6FF1A0EE66E060ED1
:10BA9000E66E100EE66EF10E6F008FFFE6FF6F0090
:10BAA0008FFFE6FF69EC4EF0F40EE126FF0EE22276
:10BAB0001200E150F40FD96EE250DA6EFF0EDA2276
:10BAC0006F007BFFE6FF6F007BFFE6FF6F007BFFF1
:10BAD000E6FF6F007BFFE6FF6F007BFFE6FF6F0076
:10BAE0007BFFE6FF6F007BFFE6FF6F007BFFE6FF5B
:10BAF000F40E6F008FFFE6FF6F008FFFE6FF170E5B
:10BB0000E66E060EE66E100EE66EF10E6F008FFF0B
:10BB1000E6FF6F008FFFE6FF69EC4EF0F40EE126C2
:10BB2000FF0EE2221200E150F40FD96EE250DA6EFD
:10BB3000FF0EDA226F007BFFE6FF6F007BFFE6FF60
:10BB40006F007BFFE6FF6F007BFFE6FF6F007BFF70
:10BB5000E6FF6F007BFFE6FF6F007BFFE6FF6F00F5
:10BB60007BFFE6FFF40E6F008FFFE6FF6F008FFF95
:10BB7000E6FF160EE66E060EE66E100EE66EF10E8F
:10BB80006F008FFFE6FF6F008FFFE6FF69EC4EF05E
:10BB9000F40EE126FF0EE2221200E652E652FC0EFF
:10BBA0006F008CFF38F0FD0E6F008CFF39F0FF0E38
:10BBB0006000E7F0E3FFFE0E6000E3F0E3FF000E3D
:10BBC000E66E000EE66E000EE66E000EE66E000EED
:10BBD000E66E000EE66E000EE66E000EE66E000EDD
:10BBE000E66E000EE66E700EE66E3C0EE66E680EB9
:10BBF000E66EF10E6F008FFFE6FF6F008FFFE6FF2E
:10BC000069EC4EF0E552E552E552E5521200E6527B
:10BC1000E652FC0E6F008CFF38F0FD0E6F008CFFBB
:10BC200039F0FF0E6000E7F0E3FFFE0E6000E3F086
:10BC3000E3FF000EE66E000EE66E000EE66E000EEE
:10BC4000E66E000EE66E000EE66E000EE66E000E6C
:10BC5000E66E000EE66E000EE66E6F0EE66E3C0EB1
:10BC6000E66E680EE66EF10E6F008FFFE6FF6F0066
:10BC70008FFFE6FF69EC4EF0E552E552E552E552E2
:10BC80001200E652E652FC0E6F008CFF38F0FD0EFB
:10BC90006F008CFF39F0FF0E6000E7F0E3FFFE0E4F
:10BCA0006000E3F0E3FF000EE66E000EE66E000EAD
:10BCB000E66E000EE66E000EE66E000EE66E000EFC
:10BCC000E66E000EE66E000EE66E000EE66E670E85
:10BCD000E66E4E0EE66E5F0EE66EF10E6F008FFFA3
:10BCE000E6FF6F008FFFE6FF69EC4EF0E552E5528C
:10BCF000E552E5521200E652E652FC0E6F008CFF50
:10BD000038F0FD0E6F008CFF39F0FF0E6000E7F099
:10BD1000E3FFFE0E6000E3F0E3FF000EE66E000EB0
:10BD2000E66E000EE66E000EE66E000EE66E000E8B
:10BD3000E66E000EE66E000EE66E000EE66E000E7B
:10BD4000E66E660EE66E4E0EE66E5F0EE66EF10E67
:10BD50006F008FFFE6FF6F008FFFE6FF69EC4EF08C
:10BD6000E552E552E552E5521200E652E652FC0E6B
:10BD70006F008CFF38F0FD0E6F008CFF39F0FF0E66
:10BD80006000E7F0E3FFFE0E6000E3F0E3FF000E6B
:10BD9000E66E000EE66E000EE66E000EE66E000E1B
:10BDA000E66E000EE66E000EE66E000EE66E000E0B
:10BDB000E66E000EE66E650EE66E4E0EE66E5F0EE9
:10BDC000E66EF10E6F008FFFE6FF6F008FFFE6FF5C
:10BDD00069EC4EF0E552E552E552E5521200E652AA
:10BDE000E652FC0E6F008CFF38F0FD0E6F008CFFEA
:10BDF00039F0FF0E6000E7F0E3FFFE0E6000E3F0B5
:10BE0000E3FF000EE66E000EE66E000EE66E000E1C
:10BE1000E66E000EE66E000EE66E000EE66E000E9A
:10BE2000E66E000EE66E000EE66E710EE66E3C0EDD
:10BE3000E66E680EE66EF10E6F008FFFE6FF6F0094
:10BE40008FFFE6FF69EC4EF0E552E552E552E55210
:10BE50001200E150F40FD96EE250DA6EFF0EDA22D2
:10BE60006F007BFFE6FF6F007BFFE6FF6F007BFF4D
:10BE7000E6FF6F007BFFE6FF6F007BFFE6FF6F00D2
:10BE80007BFFE6FF6F007BFFE6FF6F007BFFE6FFB7
:10BE9000F40E6F008FFFE6FF6F008FFFE6FF180EB6
:10BEA000E66E060EE66E100EE66EF10E6F008FFF68
:10BEB000E6FF6F008FFFE6FF69EC4EF0F40EE1261F
:10BEC000FF0EE2221200FE0EE350020F386EFF0E4C
:10BED0006F008CFF39F0000E39226000E3F0E6FFBE
:10BEE0006000E7F0E6FF1AEC61F0000EE66E000E6F
:10BEF000E66E000EE66E000EE66E000EE66E000EBA
:10BF0000E66E000EE66E000EE66E0A0EE66E000E9F
:10BF1000E66E140EE66E060EE66E100EE66EF10E7E
:10BF20006F008FFFE6FF6F008FFFE6FF69EC4EF0BA
:10BF3000E552E5521200FE0EE350020F386EFF0E7E
:10BF40006F008CFF39F0000E39226000E3F0E6FF4D
:10BF50006000E7F0E6FF1AEC61F0000EE66E000EFE
:10BF6000E66E000EE66E000EE66E000EE66E000E49
:10BF7000E66E000EE66E000EE66E0A0EE66E000E2F
:10BF8000E66E150EE66E060EE66E100EE66EF10E0D
:10BF90006F008FFFE6FF6F008FFFE6FF69EC4EF04A
:10BFA000E552E552120000EEF8F220EED7F2EE6A0A
:10BFB000DD50D950FCE1DA50FAE100EE00F2F80E63
:10BFC000EE6AE806FDE100EE00F1650EEE6AE806B5
:10BFD000FDE100EE60F0770EEE6AE806FDE100EEAE
:10BFE00001F02D0EEE6AE806FDE1080ED56E000E9A
:10BFF000D66E000ED76E0001DAEF62F0000EE66E2C
:10C00000000EE66E000EE66E000EE66E000EE66EA8
:10C01000000EE66E000EE66E000EE66EF40E6F0089
:10C020008FFFE6FF6F008FFFE6FFCB0EE66EE00EA0
:10C03000E66E520EE66EF10E6F008FFFE6FF6F00A8
:10C040008FFFE6FF69EC4EF0E552E552E552E5520E
:10C050001200000EE66E000EE66E000EE66E000E9A
:10C06000E66E000EE66E000EE66E000EE66E000E48
:10C07000E66EF40E6F008FFFE6FF6F008FFFE6FFA6
:10C08000C90EE66EE00EE66E520EE66EF10E6F0021
:10C090008FFFE6FF6F008FFFE6FF69EC4EF0E55281
:10C0A000E552E552E5521200FE0EE3501E0F386EC7
:10C0B000FF0E6F008CFF39F0000E39226000E3F0B4
:10C0C000F6FF6000E7F0F7FF000EF86EFD0EE3509C
:10C0D000396E0F0EF76405D06000E7F0F5FF0C0035
:10C0E00009D06F00DBFFE9FF6F00DFFFEAFF6000B0
:10C0F000E7F0EFFFE552E552E5521200FE0EE35085
:10C10000E66E18EC64F0FF0EE350110DF80EF32408
:10C11000D96E020EF420DA6EDE6ADD6AFF0EE3509D
:10C12000110DFA0EF324386E020EF420396E600001
:10C13000E3F0E6FF6000E7F0E6FFE0EC58F0FE0E0B
:10C14000E350E66E0CEC64F0E552E5521200E65264
:10C15000E652E652E652FC0EE36AFF0EE124D96E87
:10C16000FF0EE220DA6E600057F0DFFFFC0E6F007A
:10C170008FFFE6FF6F008FFFE6FF6F008FFFE6FF88
:10C180006F008FFFE6FF000EE66E030EE66E59ECC1
:10C190003BF0FA0EE126FF0EE2221200000EE66EE0
:10C1A000000EE66E000EE66E000EE66E000EE66E07
:10C1B000000EE66E000EE66E000EE66EB80EE66E3F
:10C1C0000B0EE66E6E0EE66E3C0EE66E680EE66ECA
:10C1D000F10E6F008FFFE6FF6F008FFFE6FF69EC47
:10C1E0004EF0E552E5521200000EE66E000EE66ECD
:10C1F000000EE66E000EE66E000EE66E000EE66EB7
:10C20000000EE66E000EE66EB80EE66E0B0EE66EE3
:10C21000640EE66E4E0EE66E5F0EE66EF10E6F0079
:10C220008FFFE6FF6F008FFFE6FF69EC4EF0E552EF
:10C23000E5521200000EE66E000EE66E000EE66E8F
:10C24000000EE66E000EE66E000EE66E000EE66E66
:10C25000000EE66E000EE66E000EE66EC80EE66E8E
:10C26000E00EE66E520EE66EF10E6F008FFFE6FFF7
:10C270006F008FFFE6FF69EC4EF0E552E5521200C9
:10C28000FE0EE350070F386EFF0E6F008CFF39F083
:10C29000000E39226000E3F0F6FF6000E7F0F7FFE0
:10C2A000000EF86E0F0EF76404D0000EF56E0C0051
:10C2B00008D06F00DBFFE9FF6F00DFFFEAFF000E31
:10C2C000EF6EE552E5521200E652E150FD0FD96ED5
:10C2D000E250DA6EFF0EDA226F007BFFF6FF6F008E
:10C2E00077FFF7FFF86A0800FF0E6F00D7FFE3FF44
:10C2F000FF0EE350E66E040EE66E000EE66E33ECC3
:10C3000043F0E552E552E5521200BA6ABB6ABC6AD4
:10C31000C26AF60EC36EC4683A016069EE0E506FD1
:10C32000406B816B516B800E416F616B426B526B46
:10C33000626B436953696369446954696469080EAF
:10C34000846F0C0EED6F330E0B6F1200000EE66E55
:10C35000000EE66E000EE66E000EE66E000EE66E55
:10C36000000EE66E000EE66E000EE66E000EE66E45
:10C37000000EE66E0A0EE66E9E0EE66E350EE66E58
:10C380002A0EE66E000EE66E69EC4EF01200E652E2
:10C39000E652FC0E6F008CFF38F0FD0E6F008CFF34
:10C3A00039F0FF0E6000E7F0E3FFFE0E6000E3F0FF
:10C3B000E3FFFE0E6F008FFFE6FF6F008FFFE6FFCB
:10C3C000EFEC5EF0E552E552E552E5521200E15025
:10C3D000FC0FD96EE250DA6EFF0EDA22FE0E6F000D
:10C3E0008CFF38F0FF0E6F008CFF39F0050E3824FB
:10C3F000E96E000E3920EA6E6F007BFFEEFF6F00E2
:10C4000077FFEDFFE552E552E552E5521200E150AB
:10C41000FC0FD96EE250DA6EFF0EDA22FE0E6F00CC
:10C420008CFF38F0FF0E6F008CFF39F0030E3824BC
:10C43000E96E000E3920EA6E6F007BFFEEFF6F00A1
:10C4400077FFEDFFE552E552E552E5521200E1506B
:10C45000FC0FD96EE250DA6EFF0EDA22FE0E6F008C
:10C460008CFF38F0FF0E6F008CFF39F0010E38247E
:10C47000E96E000E3920EA6E6F007BFFEEFF6F0061
:10C4800077FFEDFFE552E552E552E5521200E1502B
:10C49000FC0FD96EE250DA6EFF0EDA22FE0E6F004C
:10C4A0008CFF38F0FF0E6F008CFF39F0010E38243E
:10C4B000E96E000E3920EA6E6F007BFFEEFF6F0021
:10C4C00077FFEDFFE552E552E552E5521200E150EB
:10C4D000FC0FD96EE250DA6EFF0EDA22FE0E6F000C
:10C4E0008CFF38F0FF0E6F008CFF39F0030E3824FC
:10C4F000E96E000E3920EA6E6F007BFFEEFF6F00E1
:10C5000077FFEDFFE552E552E552E5521200060EC7
:10C51000E126000EE222F80E6F008CFF38F0F90ED3
:10C520006F008CFF39F0070E3824D96E000E3920C9
:10C53000DA6E080E2E6EF80E6F007BFFE3FFE82820
:10C540002E2EFAD71200FE0E6F008CFF38F0FF0E71
:10C550006F008CFF39F0070E3824D96E000E392099
:10C56000DA6E070E2E6EF60E6F008FFFDEFFE82AE2
:10C570002E06FAE2F60EE126FF0EE2221200E65245
:10C58000D2BEC5EF62F0C9EF62F0396A392ACAEF4C
:10C5900062F0396AFF0E6000E7F0E3FFD29E3901D6
:10C5A0005B510400FF0EE3B002D0D29E01D0D28EC8
:10C5B000E5521200ABEC63F0F2EC4CF0A4EC56F058
:10C5C000E7EC59F0F2EC63F0EE0EE66EA50EE66EC7
:10C5D00030EC64F0D28EBFEC62F013EC57F0EBEF6E
:10C5E00062F00DEF00F0FF0EE124D96EFF0EE220A5
:10C5F000DA6EDF50030B3901E16FFE0E6F008FFF23
:10C60000E0F93F0EE517E58100F000F06E008CF7D1
:10C610002EF0E552E55212003901A39F0001D751D7
:10C62000D811D8B416EF63F018EF63F024EF63F07D
:10C6300002D824EF63F00500FA6ED751FD6ED85191
:10C64000FE6EFF6AFA5012001200FE0E6F008CFFA1
:10C6500038F0FF0E6F008CFF39F0030E3824D96ECE
:10C66000000E3920DA6E6F0078FF2EF06F0074FF35
:10C670002FF0E552E5521200FE0E6F008CFF38F0ED
:10C68000FF0E6F008CFF39F0050E3824D96E000EB6
:10C690003920DA6E6F0078FF2EF06F0074FF2FF0F4
:10C6A000E552E5521200FE0E6F008CFF38F0FF0ECF
:10C6B0006F008CFF39F01A0E3824D96E000E392025
:10C6C000DA6EFD0E6F008FFFDFFFE552E552E55297
:10C6D0001200000EE66E000EE66E000EE66E000E14
:10C6E000E66E0F0EE66E000EE66E59EC3BF0E5527C
:10C6F000E5521200460EB96EF90EB76EB66A3901F0
:10C70000A39F938FF80EE66EC90EE66E30EC64F0D0
:10C71000890EB86E1200FE0E6F008FFFD9FFFF0E5C
:10C720006F008FFFDAFFFD0E6F008FFFDFFFE55216
:10C73000E552E5521200FE0E6F008FFFD9FFFF0E8B
:10C740006F008FFFDAFFFD0E6F008FFFDFFFE552F6
:10C75000E552E5521200FAEC64F093EC64F085ECDB
:10C7600061F09DEC64F0E3EC64F07AEC63F07FEC54
:10C770004AF0120002D8C6EF63F00500FA6E2850A6
:10C78000FD6E2950FE6EFF6AFA5012003901A59322
:10C790001200010EE66EFD0E6F008FFFE6FF6F00C8
:10C7A0008FFFE6FF53EC63F0E552E5521200000103
:10C7B000C96BCA6BCBC0CFF0CCC0D0F0CDC0D1F02C
:10C7C000CEC0D2F0E552E5521200FE0E6F008FFF90
:10C7D000D9FFFF0E6F008FFFDAFFDF502E6EE5529C
:10C7E000E5521200A6EC61F0D3EC64F06000BBF0FF
:10C7F000E6FF6000BFF0E6FF9BEC5FF01200FE0E6C
:10C80000E350E66EFE0EE350E66E000EE66EAAEC16
:10C8100059F0E552E5521200FF0EE350D8A413EF91
:10C8200064F015EF64F016EF64F0D28EE55212005A
:10C83000FF0EE350D8A41FEF64F021EF64F022EF65
:10C8400064F0D29EE5521200FE0E6F008FFFE6FFED
:10C850006F008FFFE6FF4FEC55F0E552E5521200F6
:10C86000FE0E6F008CFFD7F0FF0E6F008CFFD8F02C
:10C87000E552E5521200FE0E6F008CFFC7F0FF0E6E
:10C880006F008CFFC8F0E552E5521200FE0E6F00FB
:10C890008CFF22F0FF0E6F008CFF23F0E552E55273
:10C8A0001200FE0E6F008CFFC5F0FF0E6F008CFFB4
:10C8B000C6F0E552E5521200FE0E6F008CFF20F02C
:10C8C000FF0E6F008CFF21F0E552E5521200FE0EC4
:10C8D0006F008CFF26F0FF0E6F008CFF27F0E552F3
:10C8E000E5521200FE0E6F008CFF24F0FF0E6F0069
:10C8F0008CFF25F0E552E5521200FE0E6F008CFF12
:10C9000028F0FF0E6F008CFF29F0E552E55212006F
:10C91000FE0E6F008CFF2CF0FF0E6F008CFF2DF0D1
:10C92000E552E55212003901C06BC16BC26BC36B9B
:10C93000C46BC56BC66BC76B1200600E3901D96F33
:10C94000DB6BDD6B080EDF6FDE6B1200000E2E6EF0
:10C95000020E2F6EB40E2E26000E2F221200000E95
:10C960002E6E020E2F6E010E2E26000E2F221200AA
:10C97000000E2E6E020E2F6E700E2E26000E2F222F
:10C980001200FF0EE350E66E000EE66EF3EC62F06E
:10C99000E5521200000E2E6E020E2F6E390E2E265C
:10C9A000000E2F221200000E2E6E020E2F6E020EAF
:10C9B0002E26000E2F221200000EE66E000EE66EEE
:10C9C000FFEC63F012000C0E39015B6F370E5C6FE9
:10C9D0001200FF0E6F008CFF2BF0E55212000A0EC2
:10C9E0002A6E2C6A2D6A2B6A1200000E2E6E020E21
:10C9F0002F6E1200D29A12001200120012001200C2
:08CA00001200120012001200E6
:020000040020DA
:10000000FFFFFFFFFFFFFFFFFFFFFFFFFFFFFFFF00
:020000040030CA
:0A0000008CFFF7FFA6FFFFFFFFFFD4
:00000001FF
